Component: ARM Compiler 5.06 update 4 (build 422) Tool: armlink [4d35d2]

==============================================================================

Section Cross References

    main.o(.text) refers to _printf_pad.o(.text) for _printf_pre_padding
    main.o(.text) refers to _printf_percent.o(.ARM.Collect$$_printf_percent$$00000000) for _printf_percent
    main.o(.text) refers to _printf_llu.o(.ARM.Collect$$_printf_percent$$0000000F) for _printf_llu
    main.o(.text) refers to _printf_longlong_dec.o(.text) for _printf_longlong_dec
    main.o(.text) refers to _printf_f.o(.ARM.Collect$$_printf_percent$$00000003) for _printf_f
    main.o(.text) refers to printf1.o(x$fpl$printf1) for _printf_fp_dec
    main.o(.text) refers to bsp.o(.text) for bsp_init
    main.o(.text) refers to matrix_key.o(.text) for bsp_GetKey
    main.o(.text) refers to key_scan.o(.text) for Key_Scan_Process
    main.o(.text) refers to oled_task.o(.text) for Oled_Main_Task
    main.o(.text) refers to stm32f10x_tim.o(.text) for TIM_GetCounter
    main.o(.text) refers to ec11_spin_process.o(.text) for _EC11_Spin_LableSel_Count
    main.o(.text) refers to all_lo_init.o(.text) for PLL_Out_Ctr
    main.o(.text) refers to noretval__2printf.o(.text) for __2printf
    main.o(.text) refers to ch2_freq_set.o(.text) for CH2_Freq_Set
    main.o(.text) refers to amp_set.o(.text) for Amp_ASC_to_Value
    main.o(.text) refers to feqf.o(x$fpl$feqf) for __aeabi_cfcmpeq
    main.o(.text) refers to f2d.o(x$fpl$f2d) for __aeabi_f2d
    main.o(.text) refers to frleqf.o(x$fpl$frleqf) for __aeabi_cfrcmple
    main.o(.text) refers to fleqf.o(x$fpl$fleqf) for __aeabi_cfcmple
    main.o(.text) refers to main.o(.data) for Key_ON
    main.o(.text) refers to bsp_ec11.o(.data) for EC11_Lock
    main.o(.text) refers to cw_menu.o(.data) for CW_Display_flag
    main.o(.text) refers to key_s1_process.o(.data) for Out_State
    system_stm32f10x.o(.text) refers to system_stm32f10x.o(.data) for SystemCoreClock
    led.o(.text) refers to stm32f10x_rcc.o(.text) for RCC_APB2PeriphClockCmd
    led.o(.text) refers to stm32f10x_gpio.o(.text) for GPIO_Init
    adc.o(.text) refers to stm32f10x_rcc.o(.text) for RCC_APB2PeriphClockCmd
    adc.o(.text) refers to stm32f10x_gpio.o(.text) for GPIO_Init
    adc.o(.text) refers to stm32f10x_adc.o(.text) for ADC_DeInit
    adc.o(.text) refers to misc.o(.text) for NVIC_Init
    adc.o(.text) refers to dflt_clz.o(x$fpl$dfltu) for __aeabi_ui2d
    adc.o(.text) refers to pow.o(i.pow) for pow
    adc.o(.text) refers to daddsub_clz.o(x$fpl$dadd) for __aeabi_dadd
    adc.o(.text) refers to ddiv.o(x$fpl$ddiv) for __aeabi_ddiv
    adc.o(.text) refers to sqrt.o(i.sqrt) for sqrt
    adc.o(.text) refers to dfixu.o(x$fpl$dfixu) for __aeabi_d2uiz
    adc.o(.text) refers to daddsub_clz.o(x$fpl$dsub) for __aeabi_dsub
    adc.o(.text) refers to dmul.o(x$fpl$dmul) for __aeabi_dmul
    adc.o(.text) refers to adc.o(.data) for iLastData
    timer.o(.text) refers to stm32f10x_rcc.o(.text) for RCC_APB1PeriphClockCmd
    timer.o(.text) refers to stm32f10x_tim.o(.text) for TIM_TimeBaseInit
    timer.o(.text) refers to misc.o(.text) for NVIC_Init
    timer.o(.text) refers to matrix_key.o(.text) for bsp_KeyScan
    timer.o(.text) refers to main.o(.data) for BEEP_SW
    timer.o(.text) refers to timer.o(.data) for beep_count
    bsp_ec11.o(.text) refers to stm32f10x_rcc.o(.text) for RCC_APB2PeriphClockCmd
    bsp_ec11.o(.text) refers to stm32f10x_gpio.o(.text) for GPIO_Init
    spi.o(.text) refers to stm32f10x_rcc.o(.text) for RCC_APB2PeriphClockCmd
    spi.o(.text) refers to stm32f10x_gpio.o(.text) for GPIO_Init
    spi.o(.text) refers to stm32f10x_spi.o(.text) for SPI_Init
    oled.o(.text) refers to stm32f10x_gpio.o(.text) for GPIO_SetBits
    oled.o(.text) refers to stm32f10x_rcc.o(.text) for RCC_APB2PeriphClockCmd
    oled.o(.text) refers to delay.o(.text) for delay_us
    oled.o(.text) refers to oled.o(.constdata) for ASC5X8
    dac.o(.text) refers to stm32f10x_rcc.o(.text) for RCC_APB2PeriphClockCmd
    dac.o(.text) refers to stm32f10x_gpio.o(.text) for GPIO_Init
    dac.o(.text) refers to stm32f10x_dac.o(.text) for DAC_Init
    dac.o(.text) refers to fflt_clz.o(x$fpl$ffltu) for __aeabi_ui2f
    dac.o(.text) refers to fdiv.o(x$fpl$fdiv) for __aeabi_fdiv
    dac.o(.text) refers to fmul.o(x$fpl$fmul) for __aeabi_fmul
    dac.o(.text) refers to ffixu.o(x$fpl$ffixu) for __aeabi_f2uiz
    matrix_key.o(.text) refers to stm32f10x_rcc.o(.text) for RCC_APB2PeriphClockCmd
    matrix_key.o(.text) refers to stm32f10x_gpio.o(.text) for GPIO_Init
    matrix_key.o(.text) refers to matrix_key.o(.bss) for s_tKey
    bsp.o(.text) refers to cw_menu.o(.text) for CW_Menu_Parameters_Init
    bsp.o(.text) refers to amp_set.o(.text) for PLL_Out_Amp
    bsp.o(.text) refers to ch2_freq_set.o(.text) for Freq_Value_to_ASCII_PLL
    bsp.o(.text) refers to all_lo_init.o(.text) for LO_LMX2592_Init_Config
    bsp.o(.text) refers to delay.o(.text) for delay_init
    bsp.o(.text) refers to misc.o(.text) for NVIC_PriorityGroupConfig
    bsp.o(.text) refers to malloc.o(.text) for mem_init
    bsp.o(.text) refers to usart.o(.text) for uart_init
    bsp.o(.text) refers to noretval__2printf.o(.text) for __2printf
    bsp.o(.text) refers to led.o(.text) for LED_Init
    bsp.o(.text) refers to bsp_ec11.o(.text) for bsp_InitEC11Hard
    bsp.o(.text) refers to timer.o(.text) for TIM8_Init
    bsp.o(.text) refers to matrix_key.o(.text) for bsp_InitKey
    bsp.o(.text) refers to dac.o(.text) for Dac1_Init
    bsp.o(.text) refers to adc.o(.text) for Adc_Init
    bsp.o(.text) refers to oled.o(.text) for OLED_Init
    bsp.o(.text) refers to main_menu.o(.text) for Main_menu_Win
    bsp.o(.text) refers to pll_spi_init.o(.text) for Soft_SPI_Init
    bsp.o(.text) refers to pe4302.o(.text) for PE4302_GPIO_Init
    bsp.o(.text) refers to hmc241.o(.text) for HMC241_GPIO_Init
    bsp.o(.text) refers to ad9912_drive.o(.text) for AD9912_GPIO_init
    bsp.o(.text) refers to main.o(.data) for PLL_Amp_dBm
    bsp.o(.text) refers to cw_menu.o(.data) for CW_Freq_Uint
    key_scan.o(.text) refers to noretval__2printf.o(.text) for __2printf
    key_scan.o(.text) refers to key_s1_process.o(.text) for Key_S1_Down_Process_Other
    key_scan.o(.text) refers to key_s2_process.o(.text) for Key_S2_Down_Process
    key_scan.o(.text) refers to key_s3_process.o(.text) for Key_S3_Down_Process
    key_scan.o(.text) refers to ec11_key_process.o(.text) for EC11_Key_Down
    key_scan.o(.text) refers to main.o(.data) for BEEP_SW
    key_scan.o(.text) refers to cw_menu.o(.data) for CW_Display_flag
    key_scan.o(.text) refers to timer.o(.data) for oled_refresh
    key_scan.o(.text) refers to bsp_ec11.o(.data) for EC11_Lock
    delay.o(.text) refers to misc.o(.text) for SysTick_CLKSourceConfig
    delay.o(.text) refers to system_stm32f10x.o(.data) for SystemCoreClock
    delay.o(.text) refers to delay.o(.data) for fac_us
    usart.o(.text) refers (Special) to use_no_semi_2.o(.text) for __use_no_semihosting
    usart.o(.text) refers to stm32f10x_rcc.o(.text) for RCC_APB2PeriphClockCmd
    usart.o(.text) refers to stm32f10x_gpio.o(.text) for GPIO_Init
    usart.o(.text) refers to misc.o(.text) for NVIC_Init
    usart.o(.text) refers to stm32f10x_usart.o(.text) for USART_Init
    usart.o(.bss) refers (Special) to use_no_semi_2.o(.text) for __use_no_semihosting
    usart.o(.data) refers (Special) to use_no_semi_2.o(.text) for __use_no_semihosting
    startup_stm32f10x_hd.o(STACK) refers (Special) to heapauxi.o(.text) for __use_two_region_memory
    startup_stm32f10x_hd.o(HEAP) refers (Special) to heapauxi.o(.text) for __use_two_region_memory
    startup_stm32f10x_hd.o(RESET) refers (Special) to heapauxi.o(.text) for __use_two_region_memory
    startup_stm32f10x_hd.o(RESET) refers to startup_stm32f10x_hd.o(STACK) for __initial_sp
    startup_stm32f10x_hd.o(RESET) refers to startup_stm32f10x_hd.o(.text) for Reset_Handler
    startup_stm32f10x_hd.o(RESET) refers to stm32f10x_it.o(.text) for NMI_Handler
    startup_stm32f10x_hd.o(RESET) refers to adc.o(.text) for ADC1_2_IRQHandler
    startup_stm32f10x_hd.o(RESET) refers to timer.o(.text) for TIM2_IRQHandler
    startup_stm32f10x_hd.o(.text) refers (Special) to heapauxi.o(.text) for __use_two_region_memory
    startup_stm32f10x_hd.o(.text) refers to system_stm32f10x.o(.text) for SystemInit
    startup_stm32f10x_hd.o(.text) refers to __main.o(!!!main) for __main
    startup_stm32f10x_hd.o(.text) refers to startup_stm32f10x_hd.o(HEAP) for Heap_Mem
    startup_stm32f10x_hd.o(.text) refers to startup_stm32f10x_hd.o(STACK) for Stack_Mem
    main_menu.o(.text) refers to oled.o(.text) for Asc5_8_advant
    main_menu.o(.text) refers to main_menu.o(.data) for Main_menu_S1_Name
    main_menu.o(.text) refers to key_s1_process.o(.data) for Out_State
    main_menu.o(.text) refers to cw_menu.o(.data) for CW_menu_S1_Name0
    main_menu.o(.text) refers to power_menu.o(.data) for POWER_menu_S1_Name
    cw_menu.o(.text) refers to amp_set.o(.text) for Amp_Value_to_ASCII
    cw_menu.o(.text) refers to oled.o(.text) for Asc5_8_advant
    cw_menu.o(.text) refers to main_menu.o(.text) for Fun_KEY_Display
    cw_menu.o(.text) refers to main.o(.data) for PLL_Amp_dBm
    cw_menu.o(.text) refers to cw_menu.o(.data) for CW_Freq_Uint
    cw_menu.o(.text) refers to cw_menu.o(.bss) for CW_PLL_Freq_Show_Buf
    power_menu.o(.text) refers to _printf_pad.o(.text) for _printf_pre_padding
    power_menu.o(.text) refers to _printf_percent.o(.ARM.Collect$$_printf_percent$$00000000) for _printf_percent
    power_menu.o(.text) refers to _printf_f.o(.ARM.Collect$$_printf_percent$$00000003) for _printf_f
    power_menu.o(.text) refers to printf1.o(x$fpl$printf1) for _printf_fp_dec
    power_menu.o(.text) refers to fleqf.o(x$fpl$fleqf) for __aeabi_cfcmple
    power_menu.o(.text) refers to frleqf.o(x$fpl$frleqf) for __aeabi_cfrcmple
    power_menu.o(.text) refers to f2d.o(x$fpl$f2d) for __aeabi_f2d
    power_menu.o(.text) refers to noretval__2sprintf.o(.text) for __2sprintf
    power_menu.o(.text) refers to oled.o(.text) for Asc12_24_advant
    power_menu.o(.text) refers to main_menu.o(.text) for Fun_KEY_Display
    power_menu.o(.text) refers to adl5513.o(.data) for ADL5513_dBm_buf
    power_menu.o(.text) refers to cw_menu.o(.data) for dBm_Label
    power_menu.o(.text) refers to power_menu.o(.data) for Power_Display_flag
    oled_task.o(.text) refers to oled.o(.text) for Asc5_8_Single
    oled_task.o(.text) refers to adl5513.o(.text) for ADL5513_dBm_Out
    oled_task.o(.text) refers to feqf.o(x$fpl$feqf) for __aeabi_cfcmpeq
    oled_task.o(.text) refers to power_menu.o(.text) for Power_menu_dBm_show
    oled_task.o(.text) refers to main_menu.o(.text) for Fun_KEY_Display
    oled_task.o(.text) refers to cw_menu.o(.text) for CW_menu_Win
    oled_task.o(.text) refers to timer.o(.data) for tim_1s_count
    oled_task.o(.text) refers to main.o(.data) for Menu_Type
    oled_task.o(.text) refers to adl5513.o(.data) for ADL5513_dBm
    key_s1_process.o(.text) refers to main.o(.data) for Menu_Type
    key_s1_process.o(.text) refers to cw_menu.o(.data) for CW_Display_flag
    key_s1_process.o(.text) refers to timer.o(.data) for oled_refresh
    key_s1_process.o(.text) refers to key_s1_process.o(.data) for Key_S1_Down_Count
    key_s3_process.o(.text) refers to bsp.o(.text) for PLL_Freq_Amp_Init
    key_s3_process.o(.text) refers to main.o(.data) for Menu_Type
    key_s3_process.o(.text) refers to power_menu.o(.data) for Power_Display_flag
    key_s3_process.o(.text) refers to timer.o(.data) for oled_refresh
    key_s3_process.o(.text) refers to cw_menu.o(.data) for CW_Edit_Sel
    key_s3_process.o(.text) refers to key_s1_process.o(.data) for Out_State
    ec11_key_process.o(.text) refers to main.o(.data) for Menu_Type
    ec11_key_process.o(.text) refers to cw_menu.o(.data) for CW_Display_flag
    ec11_key_process.o(.text) refers to timer.o(.data) for oled_refresh
    ec11_spin_process.o(.text) refers to amp_set.o(.text) for Amp_ASC_to_Value
    ec11_spin_process.o(.text) refers to faddsub_clz.o(x$fpl$fadd) for __aeabi_fadd
    ec11_spin_process.o(.text) refers to frleqf.o(x$fpl$frleqf) for __aeabi_cfrcmple
    ec11_spin_process.o(.text) refers to noretval__2printf.o(.text) for __2printf
    ec11_spin_process.o(.text) refers to fleqf.o(x$fpl$fleqf) for __aeabi_cfcmple
    ec11_spin_process.o(.text) refers to ch2_freq_set.o(.text) for Freq_ASC_to_Value
    ec11_spin_process.o(.text) refers to main.o(.data) for EC11_Direct
    ec11_spin_process.o(.text) refers to cw_menu.o(.data) for CW_Edit_Sel
    ec11_spin_process.o(.text) refers to timer.o(.data) for oled_refresh
    ec11_spin_process.o(.text) refers to cw_menu.o(.bss) for CW_Freq_Show_Position_Anti
    ec11_spin_process.o(.text) refers to bsp_ec11.o(.data) for Out_Process
    ec11_spin_process.o(.text) refers to faddsub_clz.o(x$fpl$fsub) for __aeabi_fsub
    pll_spi_init.o(.text) refers to stm32f10x_rcc.o(.text) for RCC_APB2PeriphClockCmd
    pll_spi_init.o(.text) refers to stm32f10x_gpio.o(.text) for GPIO_Init
    pll_spi_init.o(.text) refers to delay.o(.text) for delay_us
    pll_spi_init.o(.text) refers to noretval__2printf.o(.text) for __2printf
    all_lo_init.o(.text) refers to delay.o(.text) for delay_ms
    all_lo_init.o(.text) refers to pll_spi_init.o(.text) for Soft_SPI_WriteByte
    all_lo_init.o(.text) refers to noretval__2printf.o(.text) for __2printf
    all_lo_init.o(.text) refers to all_lo_init.o(.constdata) for LO_LMX2582_Default_Reg3
    all_lo_init.o(.text) refers to all_lo_init.o(.data) for LMX2592_R0_Value
    lo_lmx2592_freq_set.o(.text) refers to dflt_clz.o(x$fpl$dfltu) for __aeabi_ui2d
    lo_lmx2592_freq_set.o(.text) refers to ddiv.o(x$fpl$ddiv) for __aeabi_ddiv
    lo_lmx2592_freq_set.o(.text) refers to dfixu.o(x$fpl$dfixu) for __aeabi_d2uiz
    lo_lmx2592_freq_set.o(.text) refers to dmul.o(x$fpl$dmul) for __aeabi_dmul
    lo_lmx2592_freq_set.o(.text) refers to ad9912_drive.o(.text) for AD9912_SetFreq_Hz
    lo_lmx2592_freq_set.o(.text) refers to pll_spi_init.o(.text) for Soft_SPI_WriteByte
    lo_lmx2592_freq_set.o(.text) refers to lo_lmx2592_freq_set.o(.data) for LMX2592_N
    lo_lmx2592_freq_set.o(.text) refers to dleqf.o(x$fpl$dleqf) for __aeabi_cdcmple
    lo_lmx2592_freq_set.o(.text) refers to drleqf.o(x$fpl$drleqf) for __aeabi_cdrcmple
    ad9912_drive.o(.text) refers to stm32f10x_rcc.o(.text) for RCC_APB2PeriphClockCmd
    ad9912_drive.o(.text) refers to stm32f10x_gpio.o(.text) for GPIO_Init
    ad9912_drive.o(.text) refers to delay.o(.text) for delay_ms
    ad9912_drive.o(.text) refers to spi.o(.text) for SPI2_Init
    ad9912_drive.o(.text) refers to dflt_clz.o(x$fpl$dfltu) for __aeabi_ui2d
    ad9912_drive.o(.text) refers to dmul.o(x$fpl$dmul) for __aeabi_dmul
    ad9912_drive.o(.text) refers to dfixull.o(x$fpl$llufromd) for __aeabi_d2ulz
    ad9912_drive.o(.text) refers to dfixu.o(x$fpl$dfixu) for __aeabi_d2uiz
    ad9912_drive.o(.text) refers to ad9912_drive.o(.data) for AD9912_Part_ID
    pe4302.o(.text) refers to stm32f10x_rcc.o(.text) for RCC_APB2PeriphClockCmd
    pe4302.o(.text) refers to stm32f10x_gpio.o(.text) for GPIO_PinRemapConfig
    pe4302.o(.text) refers to delay.o(.text) for delay_us
    hmc241.o(.text) refers to stm32f10x_rcc.o(.text) for RCC_APB2PeriphClockCmd
    hmc241.o(.text) refers to stm32f10x_gpio.o(.text) for GPIO_PinRemapConfig
    ad8310.o(.text) refers to adc.o(.text) for Get_Adc_Average
    ad8310.o(.text) refers to fflt_clz.o(x$fpl$ffltu) for __aeabi_ui2f
    ad8310.o(.text) refers to fmul.o(x$fpl$fmul) for __aeabi_fmul
    ad8310.o(.text) refers to faddsub_clz.o(x$fpl$fsub) for __aeabi_fsub
    ad8310.o(.text) refers to f2d.o(x$fpl$f2d) for __aeabi_f2d
    ad8310.o(.text) refers to dleqf.o(x$fpl$dleqf) for __aeabi_cdcmple
    ad8310.o(.text) refers to drleqf.o(x$fpl$drleqf) for __aeabi_cdrcmple
    ad8310.o(.text) refers to faddsub_clz.o(x$fpl$fadd) for __aeabi_fadd
    ad8310.o(.text) refers to ad8310.o(.data) for AD8310_Offset_60_80
    adl5513.o(.text) refers to adc.o(.text) for Get_Adc_Average
    adl5513.o(.text) refers to fdiv.o(x$fpl$fdiv) for __aeabi_fdiv
    adl5513.o(.text) refers to fflt_clz.o(x$fpl$ffltu) for __aeabi_ui2f
    adl5513.o(.text) refers to fmul.o(x$fpl$fmul) for __aeabi_fmul
    adl5513.o(.text) refers to frleqf.o(x$fpl$frleqf) for __aeabi_cfrcmple
    adl5513.o(.text) refers to fleqf.o(x$fpl$fleqf) for __aeabi_cfcmple
    adl5513.o(.text) refers to faddsub_clz.o(x$fpl$fsub) for __aeabi_fsub
    adl5513.o(.text) refers to faddsub_clz.o(x$fpl$fadd) for __aeabi_fadd
    adl5513.o(.text) refers to adl5513.o(.data) for ADC_Ref
    amp_set.o(.text) refers to _printf_pad.o(.text) for _printf_pre_padding
    amp_set.o(.text) refers to _printf_percent.o(.ARM.Collect$$_printf_percent$$00000000) for _printf_percent
    amp_set.o(.text) refers to _printf_f.o(.ARM.Collect$$_printf_percent$$00000003) for _printf_f
    amp_set.o(.text) refers to printf1.o(x$fpl$printf1) for _printf_fp_dec
    amp_set.o(.text) refers to faddsub_clz.o(x$fpl$frsb) for __aeabi_frsub
    amp_set.o(.text) refers to fleqf.o(x$fpl$fleqf) for __aeabi_cfcmple
    amp_set.o(.text) refers to faddsub_clz.o(x$fpl$fadd) for __aeabi_fadd
    amp_set.o(.text) refers to noretval__2printf.o(.text) for __2printf
    amp_set.o(.text) refers to frleqf.o(x$fpl$frleqf) for __aeabi_cfrcmple
    amp_set.o(.text) refers to f2d.o(x$fpl$f2d) for __aeabi_f2d
    amp_set.o(.text) refers to dleqf.o(x$fpl$dleqf) for __aeabi_cdcmple
    amp_set.o(.text) refers to hmc241.o(.text) for HMC241_Set
    amp_set.o(.text) refers to ffixu.o(x$fpl$ffixu) for __aeabi_f2uiz
    amp_set.o(.text) refers to dflt_clz.o(x$fpl$dfltu) for __aeabi_ui2d
    amp_set.o(.text) refers to daddsub_clz.o(x$fpl$dadd) for __aeabi_dadd
    amp_set.o(.text) refers to drleqf.o(x$fpl$drleqf) for __aeabi_cdrcmple
    amp_set.o(.text) refers to pe4302.o(.text) for PE4302_Set
    amp_set.o(.text) refers to faddsub_clz.o(x$fpl$fsub) for __aeabi_fsub
    amp_set.o(.text) refers to atof.o(i.atof) for atof
    amp_set.o(.text) refers to d2f.o(x$fpl$d2f) for __aeabi_d2f
    amp_set.o(.text) refers to main.o(.data) for DDS_Freq_Hz
    amp_set.o(.text) refers to amp_set.o(.constdata) for Cal_Bypass_ATT0
    amp_set.o(.text) refers to amp_set.o(.data) for DATT_Set
    amp_set.o(.text) refers to cw_menu.o(.data) for CW_Amp_Show_Buf
    amp_set.o(.text) refers to noretval__2sprintf.o(.text) for __2sprintf
    ch2_freq_set.o(.text) refers to _printf_pad.o(.text) for _printf_pre_padding
    ch2_freq_set.o(.text) refers to _printf_percent.o(.ARM.Collect$$_printf_percent$$00000000) for _printf_percent
    ch2_freq_set.o(.text) refers to _printf_u.o(.ARM.Collect$$_printf_percent$$0000000A) for _printf_u
    ch2_freq_set.o(.text) refers to _printf_dec.o(.text) for _printf_int_dec
    ch2_freq_set.o(.text) refers to _printf_llu.o(.ARM.Collect$$_printf_percent$$0000000F) for _printf_llu
    ch2_freq_set.o(.text) refers to _printf_longlong_dec.o(.text) for _printf_longlong_dec
    ch2_freq_set.o(.text) refers to atoi.o(.text) for atoi
    ch2_freq_set.o(.text) refers to atof.o(i.atof) for atof
    ch2_freq_set.o(.text) refers to dfixull.o(x$fpl$llufromd) for __aeabi_d2ulz
    ch2_freq_set.o(.text) refers to noretval__2sprintf.o(.text) for __2sprintf
    ch2_freq_set.o(.text) refers to dfltll_clz.o(x$fpl$dfltull) for __aeabi_ul2d
    ch2_freq_set.o(.text) refers to drleqf.o(x$fpl$drleqf) for __aeabi_cdrcmple
    ch2_freq_set.o(.text) refers to dleqf.o(x$fpl$dleqf) for __aeabi_cdcmple
    ch2_freq_set.o(.text) refers to ddiv.o(x$fpl$ddiv) for __aeabi_ddiv
    ch2_freq_set.o(.text) refers to lo_lmx2592_freq_set.o(.text) for Set_LMX2592_Freq_RealTime
    ch2_freq_set.o(.text) refers to cw_menu.o(.bss) for CW_DDS_Freq_Show_Buf
    stmflash.o(.text) refers to stm32f10x_flash.o(.text) for FLASH_ProgramHalfWord
    stmflash.o(.text) refers to stmflash.o(.bss) for STMFLASH_BUF
    malloc.o(.text) refers to malloc.o(.data) for mallco_dev
    malloc.o(.data) refers to malloc.o(.text) for mem_init
    malloc.o(.data) refers to malloc.o(.bss) for membase
    stm32f10x_gpio.o(.text) refers to stm32f10x_rcc.o(.text) for RCC_APB2PeriphResetCmd
    stm32f10x_rcc.o(.text) refers to stm32f10x_rcc.o(.data) for APBAHBPrescTable
    stm32f10x_usart.o(.text) refers to stm32f10x_rcc.o(.text) for RCC_APB2PeriphResetCmd
    stm32f10x_adc.o(.text) refers to stm32f10x_rcc.o(.text) for RCC_APB2PeriphResetCmd
    stm32f10x_bkp.o(.text) refers to stm32f10x_rcc.o(.text) for RCC_BackupResetCmd
    stm32f10x_pwr.o(.text) refers to stm32f10x_rcc.o(.text) for RCC_APB1PeriphResetCmd
    stm32f10x_tim.o(.text) refers to stm32f10x_rcc.o(.text) for RCC_APB2PeriphResetCmd
    stm32f10x_spi.o(.text) refers to stm32f10x_rcc.o(.text) for RCC_APB2PeriphResetCmd
    stm32f10x_dac.o(.text) refers to stm32f10x_rcc.o(.text) for RCC_APB1PeriphResetCmd
    use_no_semi_2.o(.text) refers (Special) to use_no_semi.o(.text) for __use_no_semihosting_swi
    __2printf.o(.text) refers to _printf_char_file.o(.text) for _printf_char_file
    __2printf.o(.text) refers to usart.o(.data) for __stdout
    __2sprintf.o(.text) refers to _printf_char_common.o(.text) for _printf_char_common
    __2sprintf.o(.text) refers to _sputc.o(.text) for _sputc
    noretval__2printf.o(.text) refers to _printf_char_file.o(.text) for _printf_char_file
    noretval__2printf.o(.text) refers to usart.o(.data) for __stdout
    noretval__2sprintf.o(.text) refers to _printf_char_common.o(.text) for _printf_char_common
    noretval__2sprintf.o(.text) refers to _sputc.o(.text) for _sputc
    __printf.o(.text) refers to _printf_percent.o(.ARM.Collect$$_printf_percent$$00000000) for _printf_percent
    _printf_dec.o(.text) refers to _printf_intcommon.o(.text) for _printf_int_common
    _printf_longlong_dec.o(.text) refers to lludiv10.o(.text) for _ll_udiv10
    _printf_longlong_dec.o(.text) refers to _printf_intcommon.o(.text) for _printf_int_common
    __printf_flags.o(.text) refers to _printf_percent.o(.ARM.Collect$$_printf_percent$$00000000) for _printf_percent
    __printf_flags.o(.text) refers to __printf_flags.o(.constdata) for .constdata
    __printf_ss.o(.text) refers to _printf_percent.o(.ARM.Collect$$_printf_percent$$00000000) for _printf_percent
    __printf_flags_ss.o(.text) refers to _printf_percent.o(.ARM.Collect$$_printf_percent$$00000000) for _printf_percent
    __printf_flags_ss.o(.text) refers to __printf_flags_ss.o(.constdata) for .constdata
    __printf_wp.o(.text) refers to __printf_wp.o(i._is_digit) for _is_digit
    __printf_wp.o(.text) refers to _printf_percent.o(.ARM.Collect$$_printf_percent$$00000000) for _printf_percent
    __printf_flags_wp.o(.text) refers to __printf_wp.o(i._is_digit) for _is_digit
    __printf_flags_wp.o(.text) refers to _printf_percent.o(.ARM.Collect$$_printf_percent$$00000000) for _printf_percent
    __printf_flags_wp.o(.text) refers to __printf_flags_wp.o(.constdata) for .constdata
    __printf_ss_wp.o(.text) refers to __printf_wp.o(i._is_digit) for _is_digit
    __printf_ss_wp.o(.text) refers to _printf_percent.o(.ARM.Collect$$_printf_percent$$00000000) for _printf_percent
    __printf_flags_ss_wp.o(.text) refers to __printf_wp.o(i._is_digit) for _is_digit
    __printf_flags_ss_wp.o(.text) refers to _printf_percent.o(.ARM.Collect$$_printf_percent$$00000000) for _printf_percent
    __printf_flags_ss_wp.o(.text) refers to __printf_flags_ss_wp.o(.constdata) for .constdata
    _printf_u.o(.ARM.Collect$$_printf_percent$$0000000A) refers (Weak) to _printf_dec.o(.text) for _printf_int_dec
    _printf_f.o(.ARM.Collect$$_printf_percent$$00000003) refers (Weak) to printf1.o(x$fpl$printf1) for _printf_fp_dec
    _printf_percent.o(.ARM.Collect$$_printf_percent$$00000000) refers (Special) to _printf_percent_end.o(.ARM.Collect$$_printf_percent$$00000017) for _printf_percent_end
    _printf_llu.o(.ARM.Collect$$_printf_percent$$0000000F) refers (Special) to _printf_ll.o(.ARM.Collect$$_printf_percent$$00000007) for _printf_ll
    _printf_llu.o(.ARM.Collect$$_printf_percent$$0000000F) refers (Weak) to _printf_longlong_dec.o(.text) for _printf_longlong_dec
    atoi.o(.text) refers to rt_errno_addr_intlibspace.o(.text) for __aeabi_errno_addr
    atoi.o(.text) refers to strtol.o(.text) for strtol
    __main.o(!!!main) refers to __rtentry.o(.ARM.Collect$$rtentry$$00000000) for __rt_entry
    d2f.o(x$fpl$d2f) refers (Special) to usenofp.o(x$fpl$usenofp) for __I$use$fp
    d2f.o(x$fpl$d2f) refers to fretinf.o(x$fpl$fretinf) for __fpl_fretinf
    d2f.o(x$fpl$d2f) refers to dnaninf.o(x$fpl$dnaninf) for __fpl_dnaninf
    daddsub_clz.o(x$fpl$dadd) refers (Special) to usenofp.o(x$fpl$usenofp) for __I$use$fp
    daddsub_clz.o(x$fpl$dadd) refers to daddsub_clz.o(x$fpl$dsub) for _dsub1
    daddsub_clz.o(x$fpl$dadd) refers to dretinf.o(x$fpl$dretinf) for __fpl_dretinf
    daddsub_clz.o(x$fpl$dadd) refers to dnaninf.o(x$fpl$dnaninf) for __fpl_dnaninf
    daddsub_clz.o(x$fpl$drsb) refers (Special) to usenofp.o(x$fpl$usenofp) for __I$use$fp
    daddsub_clz.o(x$fpl$drsb) refers to daddsub_clz.o(x$fpl$dadd) for _dadd1
    daddsub_clz.o(x$fpl$drsb) refers to daddsub_clz.o(x$fpl$dsub) for _dsub1
    daddsub_clz.o(x$fpl$dsub) refers (Special) to usenofp.o(x$fpl$usenofp) for __I$use$fp
    daddsub_clz.o(x$fpl$dsub) refers to daddsub_clz.o(x$fpl$dadd) for _dadd1
    daddsub_clz.o(x$fpl$dsub) refers to dnaninf.o(x$fpl$dnaninf) for __fpl_dnaninf
    ddiv.o(x$fpl$drdiv) refers (Special) to usenofp.o(x$fpl$usenofp) for __I$use$fp
    ddiv.o(x$fpl$drdiv) refers to ddiv.o(x$fpl$ddiv) for ddiv_entry
    ddiv.o(x$fpl$ddiv) refers (Special) to usenofp.o(x$fpl$usenofp) for __I$use$fp
    ddiv.o(x$fpl$ddiv) refers to dretinf.o(x$fpl$dretinf) for __fpl_dretinf
    ddiv.o(x$fpl$ddiv) refers to dnaninf.o(x$fpl$dnaninf) for __fpl_dnaninf
    dfixu.o(x$fpl$dfixu) refers (Special) to usenofp.o(x$fpl$usenofp) for __I$use$fp
    dfixu.o(x$fpl$dfixu) refers to dnaninf.o(x$fpl$dnaninf) for __fpl_dnaninf
    dfixu.o(x$fpl$dfixur) refers (Special) to usenofp.o(x$fpl$usenofp) for __I$use$fp
    dfixu.o(x$fpl$dfixur) refers to dnaninf.o(x$fpl$dnaninf) for __fpl_dnaninf
    dfixull.o(x$fpl$llufromd) refers (Special) to usenofp.o(x$fpl$usenofp) for __I$use$fp
    dfixull.o(x$fpl$llufromd) refers to dnaninf.o(x$fpl$dnaninf) for __fpl_dnaninf
    dfixull.o(x$fpl$llufromdr) refers (Special) to usenofp.o(x$fpl$usenofp) for __I$use$fp
    dfixull.o(x$fpl$llufromdr) refers to dnaninf.o(x$fpl$dnaninf) for __fpl_dnaninf
    dflt_clz.o(x$fpl$dfltu) refers (Special) to usenofp.o(x$fpl$usenofp) for __I$use$fp
    dflt_clz.o(x$fpl$dflt) refers (Special) to usenofp.o(x$fpl$usenofp) for __I$use$fp
    dflt_clz.o(x$fpl$dfltn) refers (Special) to usenofp.o(x$fpl$usenofp) for __I$use$fp
    dfltll_clz.o(x$fpl$dfltll) refers (Special) to usenofp.o(x$fpl$usenofp) for __I$use$fp
    dfltll_clz.o(x$fpl$dfltull) refers (Special) to usenofp.o(x$fpl$usenofp) for __I$use$fp
    dleqf.o(x$fpl$dleqf) refers (Special) to usenofp.o(x$fpl$usenofp) for __I$use$fp
    dleqf.o(x$fpl$dleqf) refers to dnaninf.o(x$fpl$dnaninf) for __fpl_dnaninf
    dleqf.o(x$fpl$dleqf) refers to dcmpi.o(x$fpl$dcmpinf) for __fpl_dcmp_Inf
    dmul.o(x$fpl$dmul) refers (Special) to usenofp.o(x$fpl$usenofp) for __I$use$fp
    dmul.o(x$fpl$dmul) refers to dretinf.o(x$fpl$dretinf) for __fpl_dretinf
    dmul.o(x$fpl$dmul) refers to dnaninf.o(x$fpl$dnaninf) for __fpl_dnaninf
    drleqf.o(x$fpl$drleqf) refers (Special) to usenofp.o(x$fpl$usenofp) for __I$use$fp
    drleqf.o(x$fpl$drleqf) refers to dleqf.o(x$fpl$dleqf) for __fpl_dcmple_InfNaN
    f2d.o(x$fpl$f2d) refers (Special) to usenofp.o(x$fpl$usenofp) for __I$use$fp
    f2d.o(x$fpl$f2d) refers to fnaninf.o(x$fpl$fnaninf) for __fpl_fnaninf
    f2d.o(x$fpl$f2d) refers to dretinf.o(x$fpl$dretinf) for __fpl_dretinf
    faddsub_clz.o(x$fpl$fadd) refers (Special) to usenofp.o(x$fpl$usenofp) for __I$use$fp
    faddsub_clz.o(x$fpl$fadd) refers to faddsub_clz.o(x$fpl$fsub) for _fsub1
    faddsub_clz.o(x$fpl$fadd) refers to fretinf.o(x$fpl$fretinf) for __fpl_fretinf
    faddsub_clz.o(x$fpl$fadd) refers to fnaninf.o(x$fpl$fnaninf) for __fpl_fnaninf
    faddsub_clz.o(x$fpl$frsb) refers (Special) to usenofp.o(x$fpl$usenofp) for __I$use$fp
    faddsub_clz.o(x$fpl$frsb) refers to faddsub_clz.o(x$fpl$fadd) for _fadd1
    faddsub_clz.o(x$fpl$frsb) refers to faddsub_clz.o(x$fpl$fsub) for _fsub1
    faddsub_clz.o(x$fpl$fsub) refers (Special) to usenofp.o(x$fpl$usenofp) for __I$use$fp
    faddsub_clz.o(x$fpl$fsub) refers to faddsub_clz.o(x$fpl$fadd) for _fadd1
    faddsub_clz.o(x$fpl$fsub) refers to fnaninf.o(x$fpl$fnaninf) for __fpl_fnaninf
    fdiv.o(x$fpl$frdiv) refers (Special) to usenofp.o(x$fpl$usenofp) for __I$use$fp
    fdiv.o(x$fpl$frdiv) refers to fdiv.o(x$fpl$fdiv) for _fdiv1
    fdiv.o(x$fpl$fdiv) refers (Special) to usenofp.o(x$fpl$usenofp) for __I$use$fp
    fdiv.o(x$fpl$fdiv) refers to fretinf.o(x$fpl$fretinf) for __fpl_fretinf
    fdiv.o(x$fpl$fdiv) refers to fnaninf.o(x$fpl$fnaninf) for __fpl_fnaninf
    feqf.o(x$fpl$feqf) refers (Special) to usenofp.o(x$fpl$usenofp) for __I$use$fp
    feqf.o(x$fpl$feqf) refers to fnaninf.o(x$fpl$fnaninf) for __fpl_fnaninf
    feqf.o(x$fpl$feqf) refers to fcmpi.o(x$fpl$fcmpinf) for __fpl_fcmp_Inf
    ffixu.o(x$fpl$ffixu) refers (Special) to usenofp.o(x$fpl$usenofp) for __I$use$fp
    ffixu.o(x$fpl$ffixu) refers to fnaninf.o(x$fpl$fnaninf) for __fpl_fnaninf
    ffixu.o(x$fpl$ffixur) refers (Special) to usenofp.o(x$fpl$usenofp) for __I$use$fp
    ffixu.o(x$fpl$ffixur) refers to fnaninf.o(x$fpl$fnaninf) for __fpl_fnaninf
    fflt_clz.o(x$fpl$ffltu) refers (Special) to usenofp.o(x$fpl$usenofp) for __I$use$fp
    fflt_clz.o(x$fpl$fflt) refers (Special) to usenofp.o(x$fpl$usenofp) for __I$use$fp
    fflt_clz.o(x$fpl$ffltn) refers (Special) to usenofp.o(x$fpl$usenofp) for __I$use$fp
    fleqf.o(x$fpl$fleqf) refers (Special) to usenofp.o(x$fpl$usenofp) for __I$use$fp
    fleqf.o(x$fpl$fleqf) refers to fnaninf.o(x$fpl$fnaninf) for __fpl_fnaninf
    fleqf.o(x$fpl$fleqf) refers to fcmpi.o(x$fpl$fcmpinf) for __fpl_fcmp_Inf
    fmul.o(x$fpl$fmul) refers (Special) to usenofp.o(x$fpl$usenofp) for __I$use$fp
    fmul.o(x$fpl$fmul) refers to fretinf.o(x$fpl$fretinf) for __fpl_fretinf
    fmul.o(x$fpl$fmul) refers to fnaninf.o(x$fpl$fnaninf) for __fpl_fnaninf
    frleqf.o(x$fpl$frleqf) refers (Special) to usenofp.o(x$fpl$usenofp) for __I$use$fp
    frleqf.o(x$fpl$frleqf) refers to fleqf.o(x$fpl$fleqf) for __fpl_fcmple_InfNaN
    printf1.o(x$fpl$printf1) refers to _printf_fp_dec.o(.text) for _printf_fp_dec_real
    atof.o(i.__softfp_atof) refers (Special) to usenofp.o(x$fpl$usenofp) for __I$use$fp
    atof.o(i.__softfp_atof) refers to _rserrno.o(.text) for __read_errno
    atof.o(i.__softfp_atof) refers to strtod.o(.text) for __strtod_int
    atof.o(i.atof) refers (Special) to usenofp.o(x$fpl$usenofp) for __I$use$fp
    atof.o(i.atof) refers to _rserrno.o(.text) for __read_errno
    atof.o(i.atof) refers to strtod.o(.text) for __strtod_int
    pow.o(i.__softfp_pow) refers (Special) to usenofp.o(x$fpl$usenofp) for __I$use$fp
    pow.o(i.__softfp_pow) refers to pow.o(i.pow) for pow
    pow.o(i.pow) refers (Special) to usenofp.o(x$fpl$usenofp) for __I$use$fp
    pow.o(i.pow) refers to dunder.o(i.__mathlib_dbl_infnan2) for __mathlib_dbl_infnan2
    pow.o(i.pow) refers to _rserrno.o(.text) for __set_errno
    pow.o(i.pow) refers to dunder.o(i.__mathlib_dbl_divzero) for __mathlib_dbl_divzero
    pow.o(i.pow) refers to ddiv.o(x$fpl$ddiv) for __aeabi_ddiv
    pow.o(i.pow) refers to sqrt.o(i.sqrt) for sqrt
    pow.o(i.pow) refers to dmul.o(x$fpl$dmul) for __aeabi_dmul
    pow.o(i.pow) refers to dflt_clz.o(x$fpl$dflt) for __aeabi_i2d
    pow.o(i.pow) refers to dunder.o(i.__mathlib_dbl_invalid) for __mathlib_dbl_invalid
    pow.o(i.pow) refers to dunder.o(i.__mathlib_dbl_overflow) for __mathlib_dbl_overflow
    pow.o(i.pow) refers to dunder.o(i.__mathlib_dbl_underflow) for __mathlib_dbl_underflow
    pow.o(i.pow) refers to daddsub_clz.o(x$fpl$dsub) for __aeabi_dsub
    pow.o(i.pow) refers to scalbn.o(x$fpl$scalbn) for __ARM_scalbn
    pow.o(i.pow) refers to daddsub_clz.o(x$fpl$drsb) for __aeabi_drsub
    pow.o(i.pow) refers to daddsub_clz.o(x$fpl$dadd) for __aeabi_dadd
    pow.o(i.pow) refers to qnan.o(.constdata) for __mathlib_zero
    pow.o(i.pow) refers to poly.o(i.__kernel_poly) for __kernel_poly
    pow.o(i.pow) refers to drleqf.o(x$fpl$drleqf) for __aeabi_cdrcmple
    pow.o(i.pow) refers to pow.o(.constdata) for .constdata
    pow.o(i.pow) refers to fpclassify.o(i.__ARM_fpclassify) for __ARM_fpclassify
    pow.o(.constdata) refers (Special) to usenofp.o(x$fpl$usenofp) for __I$use$fp
    pow_x.o(i.____softfp_pow$lsc) refers (Special) to usenofp.o(x$fpl$usenofp) for __I$use$fp
    pow_x.o(i.____softfp_pow$lsc) refers to pow_x.o(i.__pow$lsc) for __pow$lsc
    pow_x.o(i.__pow$lsc) refers (Special) to usenofp.o(x$fpl$usenofp) for __I$use$fp
    pow_x.o(i.__pow$lsc) refers to dunder.o(i.__mathlib_dbl_infnan2) for __mathlib_dbl_infnan2
    pow_x.o(i.__pow$lsc) refers to _rserrno.o(.text) for __set_errno
    pow_x.o(i.__pow$lsc) refers to ddiv.o(x$fpl$ddiv) for __aeabi_ddiv
    pow_x.o(i.__pow$lsc) refers to sqrt.o(i.sqrt) for sqrt
    pow_x.o(i.__pow$lsc) refers to dmul.o(x$fpl$dmul) for __aeabi_dmul
    pow_x.o(i.__pow$lsc) refers to dflt_clz.o(x$fpl$dflt) for __aeabi_i2d
    pow_x.o(i.__pow$lsc) refers to daddsub_clz.o(x$fpl$dsub) for __aeabi_dsub
    pow_x.o(i.__pow$lsc) refers to scalbn.o(x$fpl$scalbn) for __ARM_scalbn
    pow_x.o(i.__pow$lsc) refers to daddsub_clz.o(x$fpl$drsb) for __aeabi_drsub
    pow_x.o(i.__pow$lsc) refers to daddsub_clz.o(x$fpl$dadd) for __aeabi_dadd
    pow_x.o(i.__pow$lsc) refers to qnan.o(.constdata) for __mathlib_zero
    pow_x.o(i.__pow$lsc) refers to poly.o(i.__kernel_poly) for __kernel_poly
    pow_x.o(i.__pow$lsc) refers to drleqf.o(x$fpl$drleqf) for __aeabi_cdrcmple
    pow_x.o(i.__pow$lsc) refers to pow_x.o(.constdata) for .constdata
    pow_x.o(.constdata) refers (Special) to usenofp.o(x$fpl$usenofp) for __I$use$fp
    sqrt.o(i.__softfp_sqrt) refers (Special) to usenofp.o(x$fpl$usenofp) for __I$use$fp
    sqrt.o(i.__softfp_sqrt) refers to dsqrt_noumaal.o(x$fpl$dsqrt) for _dsqrt
    sqrt.o(i.__softfp_sqrt) refers to _rserrno.o(.text) for __set_errno
    sqrt.o(i.sqrt) refers (Special) to usenofp.o(x$fpl$usenofp) for __I$use$fp
    sqrt.o(i.sqrt) refers to dsqrt_noumaal.o(x$fpl$dsqrt) for _dsqrt
    sqrt.o(i.sqrt) refers to _rserrno.o(.text) for __set_errno
    sqrt_x.o(i.____softfp_sqrt$lsc) refers (Special) to usenofp.o(x$fpl$usenofp) for __I$use$fp
    sqrt_x.o(i.____softfp_sqrt$lsc) refers to dleqf.o(x$fpl$dleqf) for __aeabi_cdcmple
    sqrt_x.o(i.____softfp_sqrt$lsc) refers to _rserrno.o(.text) for __set_errno
    sqrt_x.o(i.____softfp_sqrt$lsc) refers to dsqrt_noumaal.o(x$fpl$dsqrt) for _dsqrt
    sqrt_x.o(i.__sqrt$lsc) refers (Special) to usenofp.o(x$fpl$usenofp) for __I$use$fp
    sqrt_x.o(i.__sqrt$lsc) refers to dleqf.o(x$fpl$dleqf) for __aeabi_cdcmple
    sqrt_x.o(i.__sqrt$lsc) refers to _rserrno.o(.text) for __set_errno
    sqrt_x.o(i.__sqrt$lsc) refers to dsqrt_noumaal.o(x$fpl$dsqrt) for _dsqrt
    __rtentry.o(.ARM.Collect$$rtentry$$00000000) refers (Special) to __rtentry2.o(.ARM.Collect$$rtentry$$0000000A) for __rt_entry_li
    __rtentry.o(.ARM.Collect$$rtentry$$00000000) refers (Special) to __rtentry2.o(.ARM.Collect$$rtentry$$0000000D) for __rt_entry_main
    __rtentry.o(.ARM.Collect$$rtentry$$00000000) refers (Special) to __rtentry2.o(.ARM.Collect$$rtentry$$0000000C) for __rt_entry_postli_1
    __rtentry.o(.ARM.Collect$$rtentry$$00000000) refers (Special) to __rtentry2.o(.ARM.Collect$$rtentry$$00000009) for __rt_entry_postsh_1
    __rtentry.o(.ARM.Collect$$rtentry$$00000000) refers (Special) to __rtentry2.o(.ARM.Collect$$rtentry$$00000002) for __rt_entry_presh_1
    __rtentry.o(.ARM.Collect$$rtentry$$00000000) refers (Special) to __rtentry4.o(.ARM.Collect$$rtentry$$00000004) for __rt_entry_sh
    rt_errno_addr.o(.text) refers to rt_errno_addr.o(.bss) for __aeabi_errno_addr_data
    rt_errno_addr_intlibspace.o(.text) refers to libspace.o(.bss) for __libspace_start
    _rserrno.o(.text) refers to rt_errno_addr_intlibspace.o(.text) for __aeabi_errno_addr
    _printf_intcommon.o(.text) refers (Weak) to _printf_pad.o(.text) for _printf_pre_padding
    _printf_intcommon.o(.text) refers (Weak) to _printf_pad.o(.text) for _printf_pre_padding
    _printf_intcommon.o(.text) refers (Weak) to _printf_pad.o(.text) for _printf_post_padding
    _printf_fp_dec.o(.text) refers (Special) to usenofp.o(x$fpl$usenofp) for __I$use$fp
    _printf_fp_dec.o(.text) refers (Special) to lc_numeric_c.o(locale$$code) for _get_lc_numeric
    _printf_fp_dec.o(.text) refers to bigflt0.o(.text) for _btod_etento
    _printf_fp_dec.o(.text) refers to btod.o(CL$$btod_d2e) for _btod_d2e
    _printf_fp_dec.o(.text) refers to btod.o(CL$$btod_ediv) for _btod_ediv
    _printf_fp_dec.o(.text) refers to btod.o(CL$$btod_emul) for _btod_emul
    _printf_fp_dec.o(.text) refers to lludiv10.o(.text) for _ll_udiv10
    _printf_fp_dec.o(.text) refers to fpclassify.o(i.__ARM_fpclassify) for __ARM_fpclassify
    _printf_fp_dec.o(.text) refers to _printf_fp_infnan.o(.text) for _printf_fp_infnan
    _printf_fp_dec.o(.text) refers (Weak) to _printf_pad.o(.text) for _printf_pre_padding
    _printf_fp_dec.o(.text) refers (Weak) to _printf_pad.o(.text) for _printf_pre_padding
    _printf_fp_dec.o(.text) refers to rt_locale_intlibspace.o(.text) for __rt_locale
    _printf_fp_dec.o(.text) refers (Weak) to _printf_pad.o(.text) for _printf_post_padding
    _printf_char_common.o(.text) refers to __printf_flags_ss_wp.o(.text) for __printf
    _printf_char_file.o(.text) refers to _printf_char_common.o(.text) for _printf_char_common
    _printf_char_file.o(.text) refers to ferror.o(.text) for ferror
    _printf_char_file.o(.text) refers to usart.o(.text) for fputc
    strtod.o(.text) refers (Special) to lc_numeric_c.o(locale$$code) for _get_lc_numeric
    strtod.o(.text) refers to scanf1.o(x$fpl$scanf1) for _scanf_real
    strtod.o(.text) refers to _sgetc.o(.text) for _sgetc
    strtod.o(.text) refers to isspace.o(.text) for isspace
    strtol.o(.text) refers to rt_ctype_table.o(.text) for __rt_ctype_table
    strtol.o(.text) refers to _strtoul.o(.text) for _strtoul
    strtol.o(.text) refers to rt_errno_addr_intlibspace.o(.text) for __aeabi_errno_addr
    dcmpi.o(x$fpl$dcmpinf) refers (Special) to usenofp.o(x$fpl$usenofp) for __I$use$fp
    dnaninf.o(x$fpl$dnaninf) refers (Special) to usenofp.o(x$fpl$usenofp) for __I$use$fp
    dretinf.o(x$fpl$dretinf) refers (Special) to usenofp.o(x$fpl$usenofp) for __I$use$fp
    dsqrt_noumaal.o(x$fpl$dsqrt) refers (Special) to usenofp.o(x$fpl$usenofp) for __I$use$fp
    dsqrt_noumaal.o(x$fpl$dsqrt) refers to dnaninf.o(x$fpl$dnaninf) for __fpl_dnaninf
    fcmpi.o(x$fpl$fcmpinf) refers (Special) to usenofp.o(x$fpl$usenofp) for __I$use$fp
    fnaninf.o(x$fpl$fnaninf) refers (Special) to usenofp.o(x$fpl$usenofp) for __I$use$fp
    fretinf.o(x$fpl$fretinf) refers (Special) to usenofp.o(x$fpl$usenofp) for __I$use$fp
    scalbn.o(x$fpl$scalbn) refers (Special) to usenofp.o(x$fpl$usenofp) for __I$use$fp
    scalbn.o(x$fpl$scalbn) refers to dcheck1.o(x$fpl$dcheck1) for __fpl_dcheck_NaN1
    dunder.o(i.__mathlib_dbl_divzero) refers to ddiv.o(x$fpl$ddiv) for __aeabi_ddiv
    dunder.o(i.__mathlib_dbl_infnan) refers to scalbn.o(x$fpl$scalbn) for __ARM_scalbn
    dunder.o(i.__mathlib_dbl_infnan2) refers to daddsub_clz.o(x$fpl$dadd) for __aeabi_dadd
    dunder.o(i.__mathlib_dbl_invalid) refers to ddiv.o(x$fpl$ddiv) for __aeabi_ddiv
    dunder.o(i.__mathlib_dbl_overflow) refers to scalbn.o(x$fpl$scalbn) for __ARM_scalbn
    dunder.o(i.__mathlib_dbl_posinfnan) refers to dmul.o(x$fpl$dmul) for __aeabi_dmul
    dunder.o(i.__mathlib_dbl_underflow) refers to scalbn.o(x$fpl$scalbn) for __ARM_scalbn
    fpclassify.o(i.__ARM_fpclassify) refers (Special) to usenofp.o(x$fpl$usenofp) for __I$use$fp
    poly.o(i.__kernel_poly) refers (Special) to usenofp.o(x$fpl$usenofp) for __I$use$fp
    poly.o(i.__kernel_poly) refers to dmul.o(x$fpl$dmul) for __aeabi_dmul
    poly.o(i.__kernel_poly) refers to daddsub_clz.o(x$fpl$dadd) for __aeabi_dadd
    qnan.o(.constdata) refers (Special) to usenofp.o(x$fpl$usenofp) for __I$use$fp
    libspace.o(.text) refers to libspace.o(.bss) for __libspace_start
    __rtentry2.o(.ARM.Collect$$rtentry$$00000008) refers to boardinit2.o(.text) for _platform_post_stackheap_init
    __rtentry2.o(.ARM.Collect$$rtentry$$0000000A) refers to libinit.o(.ARM.Collect$$libinit$$00000000) for __rt_lib_init
    __rtentry2.o(.ARM.Collect$$rtentry$$0000000B) refers to boardinit3.o(.text) for _platform_post_lib_init
    __rtentry2.o(.ARM.Collect$$rtentry$$0000000D) refers to main.o(.text) for main
    __rtentry2.o(.ARM.Collect$$rtentry$$0000000D) refers to exit.o(.text) for exit
    __rtentry2.o(.ARM.exidx) refers to __rtentry2.o(.ARM.Collect$$rtentry$$00000001) for .ARM.Collect$$rtentry$$00000001
    __rtentry2.o(.ARM.exidx) refers to __rtentry2.o(.ARM.Collect$$rtentry$$00000008) for .ARM.Collect$$rtentry$$00000008
    __rtentry2.o(.ARM.exidx) refers to __rtentry2.o(.ARM.Collect$$rtentry$$0000000A) for .ARM.Collect$$rtentry$$0000000A
    __rtentry2.o(.ARM.exidx) refers to __rtentry2.o(.ARM.Collect$$rtentry$$0000000B) for .ARM.Collect$$rtentry$$0000000B
    __rtentry2.o(.ARM.exidx) refers to __rtentry2.o(.ARM.Collect$$rtentry$$0000000D) for .ARM.Collect$$rtentry$$0000000D
    __rtentry4.o(.ARM.Collect$$rtentry$$00000004) refers to sys_stackheap_outer.o(.text) for __user_setup_stackheap
    __rtentry4.o(.ARM.exidx) refers to __rtentry4.o(.ARM.Collect$$rtentry$$00000004) for .ARM.Collect$$rtentry$$00000004
    rt_ctype_table.o(.text) refers to rt_locale_intlibspace.o(.text) for __rt_locale
    rt_ctype_table.o(.text) refers to lc_ctype_c.o(locale$$code) for _get_lc_ctype
    rt_locale.o(.text) refers to rt_locale.o(.bss) for __rt_locale_data
    rt_locale_intlibspace.o(.text) refers to libspace.o(.bss) for __libspace_start
    isspace.o(.text) refers to rt_ctype_table.o(.text) for __rt_ctype_table
    _printf_fp_infnan.o(.text) refers (Weak) to _printf_pad.o(.text) for _printf_pre_padding
    _printf_fp_infnan.o(.text) refers (Weak) to _printf_pad.o(.text) for _printf_post_padding
    _strtoul.o(.text) refers to _chval.o(.text) for _chval
    _strtoul.o(.text) refers to rt_errno_addr_intlibspace.o(.text) for __aeabi_errno_addr
    bigflt0.o(.text) refers (Special) to usenofp.o(x$fpl$usenofp) for __I$use$fp
    bigflt0.o(.text) refers to btod.o(CL$$btod_emul) for _btod_emul
    bigflt0.o(.text) refers to btod.o(CL$$btod_ediv) for _btod_ediv
    bigflt0.o(.text) refers to bigflt0.o(.constdata) for .constdata
    bigflt0.o(.constdata) refers (Special) to usenofp.o(x$fpl$usenofp) for __I$use$fp
    btod.o(CL$$btod_d2e) refers (Special) to usenofp.o(x$fpl$usenofp) for __I$use$fp
    btod.o(CL$$btod_d2e) refers to btod.o(CL$$btod_d2e_norm_op1) for _d2e_norm_op1
    btod.o(CL$$btod_d2e_norm_op1) refers (Special) to usenofp.o(x$fpl$usenofp) for __I$use$fp
    btod.o(CL$$btod_d2e_norm_op1) refers to btod.o(CL$$btod_d2e_denorm_low) for _d2e_denorm_low
    btod.o(CL$$btod_d2e_denorm_low) refers (Special) to usenofp.o(x$fpl$usenofp) for __I$use$fp
    btod.o(CL$$btod_emul) refers (Special) to usenofp.o(x$fpl$usenofp) for __I$use$fp
    btod.o(CL$$btod_emul) refers to btod.o(CL$$btod_mult_common) for __btod_mult_common
    btod.o(CL$$btod_emul) refers to btod.o(CL$$btod_e2e) for _e2e
    btod.o(CL$$btod_ediv) refers (Special) to usenofp.o(x$fpl$usenofp) for __I$use$fp
    btod.o(CL$$btod_ediv) refers to btod.o(CL$$btod_div_common) for __btod_div_common
    btod.o(CL$$btod_ediv) refers to btod.o(CL$$btod_e2e) for _e2e
    btod.o(CL$$btod_emuld) refers (Special) to usenofp.o(x$fpl$usenofp) for __I$use$fp
    btod.o(CL$$btod_emuld) refers to btod.o(CL$$btod_mult_common) for __btod_mult_common
    btod.o(CL$$btod_emuld) refers to btod.o(CL$$btod_e2d) for _e2d
    btod.o(CL$$btod_edivd) refers (Special) to usenofp.o(x$fpl$usenofp) for __I$use$fp
    btod.o(CL$$btod_edivd) refers to btod.o(CL$$btod_div_common) for __btod_div_common
    btod.o(CL$$btod_edivd) refers to btod.o(CL$$btod_e2d) for _e2d
    btod.o(CL$$btod_e2e) refers (Special) to usenofp.o(x$fpl$usenofp) for __I$use$fp
    btod.o(CL$$btod_e2d) refers (Special) to usenofp.o(x$fpl$usenofp) for __I$use$fp
    btod.o(CL$$btod_e2d) refers to btod.o(CL$$btod_e2e) for _e2e
    btod.o(CL$$btod_mult_common) refers (Special) to usenofp.o(x$fpl$usenofp) for __I$use$fp
    btod.o(CL$$btod_div_common) refers (Special) to usenofp.o(x$fpl$usenofp) for __I$use$fp
    lc_numeric_c.o(locale$$data) refers (Special) to libinit2.o(.ARM.Collect$$libinit$$00000016) for __rt_lib_init_lc_numeric_2
    lc_numeric_c.o(locale$$code) refers (Special) to libinit2.o(.ARM.Collect$$libinit$$00000016) for __rt_lib_init_lc_numeric_2
    lc_numeric_c.o(locale$$code) refers to strcmpv7m.o(.text) for strcmp
    lc_numeric_c.o(locale$$code) refers to lc_numeric_c.o(locale$$data) for __lcnum_c_name
    dcheck1.o(x$fpl$dcheck1) refers (Special) to usenofp.o(x$fpl$usenofp) for __I$use$fp
    dcheck1.o(x$fpl$dcheck1) refers to retnan.o(x$fpl$retnan) for __fpl_return_NaN
    istatus.o(x$fpl$ieeestatus) refers (Special) to usenofp.o(x$fpl$usenofp) for __I$use$fp
    scanf1.o(x$fpl$scanf1) refers to scanf_fp.o(.text) for _scanf_really_real
    sys_stackheap_outer.o(.text) refers to libspace.o(.text) for __user_perproc_libspace
    sys_stackheap_outer.o(.text) refers to startup_stm32f10x_hd.o(.text) for __user_initial_stackheap
    scanf_fp.o(.text) refers (Special) to usenofp.o(x$fpl$usenofp) for __I$use$fp
    scanf_fp.o(.text) refers (Special) to lc_numeric_c.o(locale$$code) for _get_lc_numeric
    scanf_fp.o(.text) refers to rt_errno_addr_intlibspace.o(.text) for __aeabi_errno_addr
    scanf_fp.o(.text) refers to bigflt0.o(.text) for _btod_etento
    scanf_fp.o(.text) refers to btod.o(CL$$btod_emuld) for _btod_emuld
    scanf_fp.o(.text) refers to btod.o(CL$$btod_edivd) for _btod_edivd
    scanf_fp.o(.text) refers to rt_locale_intlibspace.o(.text) for __rt_locale
    scanf_fp.o(.text) refers to scanf2.o(x$fpl$scanf2) for _scanf_infnan
    scanf_fp.o(.text) refers to __printf_wp.o(i._is_digit) for _is_digit
    scanf_fp.o(.text) refers to narrow.o(i.__mathlib_narrow) for __mathlib_narrow
    scanf_fp.o(.text) refers to fpconst.o(c$$dinf) for __huge_val
    lc_ctype_c.o(locale$$data) refers (Special) to libinit2.o(.ARM.Collect$$libinit$$00000012) for __rt_lib_init_lc_ctype_2
    lc_ctype_c.o(locale$$code) refers (Special) to libinit2.o(.ARM.Collect$$libinit$$00000012) for __rt_lib_init_lc_ctype_2
    lc_ctype_c.o(locale$$code) refers to strcmpv7m.o(.text) for strcmp
    lc_ctype_c.o(locale$$code) refers to lc_ctype_c.o(locale$$data) for __lcctype_c_name
    exit.o(.text) refers to rtexit.o(.ARM.Collect$$rtexit$$00000000) for __rt_exit
    libinit.o(.ARM.Collect$$libinit$$00000000) refers (Special) to libinit2.o(.ARM.Collect$$libinit$$0000002E) for __rt_lib_init_alloca_1
    libinit.o(.ARM.Collect$$libinit$$00000000) refers (Special) to libinit2.o(.ARM.Collect$$libinit$$0000002C) for __rt_lib_init_argv_1
    libinit.o(.ARM.Collect$$libinit$$00000000) refers (Special) to libinit2.o(.ARM.Collect$$libinit$$0000001B) for __rt_lib_init_atexit_1
    libinit.o(.ARM.Collect$$libinit$$00000000) refers (Special) to libinit2.o(.ARM.Collect$$libinit$$00000021) for __rt_lib_init_clock_1
    libinit.o(.ARM.Collect$$libinit$$00000000) refers (Special) to libinit2.o(.ARM.Collect$$libinit$$00000032) for __rt_lib_init_cpp_1
    libinit.o(.ARM.Collect$$libinit$$00000000) refers (Special) to libinit2.o(.ARM.Collect$$libinit$$00000030) for __rt_lib_init_exceptions_1
    libinit.o(.ARM.Collect$$libinit$$00000000) refers (Special) to libinit2.o(.ARM.Collect$$libinit$$00000002) for __rt_lib_init_fp_1
    libinit.o(.ARM.Collect$$libinit$$00000000) refers (Special) to libinit2.o(.ARM.Collect$$libinit$$0000001F) for __rt_lib_init_fp_trap_1
    libinit.o(.ARM.Collect$$libinit$$00000000) refers (Special) to libinit2.o(.ARM.Collect$$libinit$$00000023) for __rt_lib_init_getenv_1
    libinit.o(.ARM.Collect$$libinit$$00000000) refers (Special) to libinit2.o(.ARM.Collect$$libinit$$0000000A) for __rt_lib_init_heap_1
    libinit.o(.ARM.Collect$$libinit$$00000000) refers (Special) to libinit2.o(.ARM.Collect$$libinit$$00000011) for __rt_lib_init_lc_collate_1
    libinit.o(.ARM.Collect$$libinit$$00000000) refers (Special) to libinit2.o(.ARM.Collect$$libinit$$00000013) for __rt_lib_init_lc_ctype_1
    libinit.o(.ARM.Collect$$libinit$$00000000) refers (Special) to libinit2.o(.ARM.Collect$$libinit$$00000015) for __rt_lib_init_lc_monetary_1
    libinit.o(.ARM.Collect$$libinit$$00000000) refers (Special) to libinit2.o(.ARM.Collect$$libinit$$00000017) for __rt_lib_init_lc_numeric_1
    libinit.o(.ARM.Collect$$libinit$$00000000) refers (Special) to libinit2.o(.ARM.Collect$$libinit$$00000019) for __rt_lib_init_lc_time_1
    libinit.o(.ARM.Collect$$libinit$$00000000) refers (Special) to libinit2.o(.ARM.Collect$$libinit$$00000004) for __rt_lib_init_preinit_1
    libinit.o(.ARM.Collect$$libinit$$00000000) refers (Special) to libinit2.o(.ARM.Collect$$libinit$$0000000E) for __rt_lib_init_rand_1
    libinit.o(.ARM.Collect$$libinit$$00000000) refers (Special) to libinit2.o(.ARM.Collect$$libinit$$00000033) for __rt_lib_init_return
    libinit.o(.ARM.Collect$$libinit$$00000000) refers (Special) to libinit2.o(.ARM.Collect$$libinit$$0000001D) for __rt_lib_init_signal_1
    libinit.o(.ARM.Collect$$libinit$$00000000) refers (Special) to libinit2.o(.ARM.Collect$$libinit$$00000025) for __rt_lib_init_stdio_1
    libinit.o(.ARM.Collect$$libinit$$00000000) refers (Special) to libinit2.o(.ARM.Collect$$libinit$$0000000C) for __rt_lib_init_user_alloc_1
    libinit2.o(.ARM.Collect$$libinit$$0000000F) refers (Weak) to rt_locale_intlibspace.o(.text) for __rt_locale
    libinit2.o(.ARM.Collect$$libinit$$00000010) refers to libinit2.o(.ARM.Collect$$libinit$$0000000F) for .ARM.Collect$$libinit$$0000000F
    libinit2.o(.ARM.Collect$$libinit$$00000012) refers to libinit2.o(.ARM.Collect$$libinit$$0000000F) for .ARM.Collect$$libinit$$0000000F
    libinit2.o(.ARM.Collect$$libinit$$00000012) refers (Weak) to lc_ctype_c.o(locale$$code) for _get_lc_ctype
    libinit2.o(.ARM.Collect$$libinit$$00000014) refers to libinit2.o(.ARM.Collect$$libinit$$0000000F) for .ARM.Collect$$libinit$$0000000F
    libinit2.o(.ARM.Collect$$libinit$$00000016) refers to libinit2.o(.ARM.Collect$$libinit$$0000000F) for .ARM.Collect$$libinit$$0000000F
    libinit2.o(.ARM.Collect$$libinit$$00000016) refers (Weak) to lc_numeric_c.o(locale$$code) for _get_lc_numeric
    libinit2.o(.ARM.Collect$$libinit$$00000018) refers to libinit2.o(.ARM.Collect$$libinit$$0000000F) for .ARM.Collect$$libinit$$0000000F
    libinit2.o(.ARM.Collect$$libinit$$00000026) refers to argv_veneer.o(.emb_text) for __ARM_argv_veneer
    libinit2.o(.ARM.Collect$$libinit$$00000027) refers to argv_veneer.o(.emb_text) for __ARM_argv_veneer
    retnan.o(x$fpl$retnan) refers (Special) to usenofp.o(x$fpl$usenofp) for __I$use$fp
    retnan.o(x$fpl$retnan) refers to trapv.o(x$fpl$trapveneer) for __fpl_cmpreturn
    rtexit.o(.ARM.Collect$$rtexit$$00000000) refers (Special) to rtexit2.o(.ARM.Collect$$rtexit$$00000004) for __rt_exit_exit
    rtexit.o(.ARM.Collect$$rtexit$$00000000) refers (Special) to rtexit2.o(.ARM.Collect$$rtexit$$00000003) for __rt_exit_ls
    rtexit.o(.ARM.Collect$$rtexit$$00000000) refers (Special) to rtexit2.o(.ARM.Collect$$rtexit$$00000002) for __rt_exit_prels_1
    rtexit.o(.ARM.exidx) refers (Special) to rtexit2.o(.ARM.Collect$$rtexit$$00000004) for __rt_exit_exit
    rtexit.o(.ARM.exidx) refers (Special) to rtexit2.o(.ARM.Collect$$rtexit$$00000003) for __rt_exit_ls
    rtexit.o(.ARM.exidx) refers (Special) to rtexit2.o(.ARM.Collect$$rtexit$$00000002) for __rt_exit_prels_1
    rtexit.o(.ARM.exidx) refers to rtexit.o(.ARM.Collect$$rtexit$$00000000) for .ARM.Collect$$rtexit$$00000000
    argv_veneer.o(.emb_text) refers to no_argv.o(.text) for __ARM_get_argv
    fpconst.o(c$$dinf) refers (Special) to usenofp.o(x$fpl$usenofp) for __I$use$fp
    fpconst.o(c$$dnan) refers (Special) to usenofp.o(x$fpl$usenofp) for __I$use$fp
    fpconst.o(c$$finf) refers (Special) to usenofp.o(x$fpl$usenofp) for __I$use$fp
    scanf2.o(x$fpl$scanf2) refers to scanf_hexfp.o(.text) for _scanf_really_hex_real
    scanf2.o(x$fpl$scanf2) refers to scanf_infnan.o(.text) for _scanf_really_infnan
    scanf2b.o(x$fpl$scanf2) refers to scanf_hexfp.o(.text) for _scanf_really_hex_real
    scanf2b.o(x$fpl$scanf2) refers to scanf_infnan.o(.text) for _scanf_really_infnan
    trapv.o(x$fpl$trapveneer) refers (Special) to usenofp.o(x$fpl$usenofp) for __I$use$fp
    narrow.o(i.__mathlib_narrow) refers (Special) to usenofp.o(x$fpl$usenofp) for __I$use$fp
    narrow.o(i.__mathlib_narrow) refers to narrow.o(i.__mathlib_tofloat) for __mathlib_tofloat
    narrow.o(i.__mathlib_tofloat) refers (Special) to usenofp.o(x$fpl$usenofp) for __I$use$fp
    narrow.o(i.__mathlib_tofloat) refers to frexp.o(i.frexp) for frexp
    narrow.o(i.__mathlib_tofloat) refers to deqf.o(x$fpl$deqf) for __aeabi_cdcmpeq
    narrow.o(i.__mathlib_tofloat) refers to d2f.o(x$fpl$d2f) for __aeabi_d2f
    narrow.o(i.__mathlib_tofloat) refers to _rserrno.o(.text) for __set_errno
    narrow.o(i.__mathlib_tofloat) refers to drleqf.o(x$fpl$drleqf) for __aeabi_cdrcmple
    narrow.o(i.__softfp___mathlib_tofloat) refers (Special) to usenofp.o(x$fpl$usenofp) for __I$use$fp
    narrow.o(i.__softfp___mathlib_tofloat) refers to narrow.o(i.__mathlib_tofloat) for __mathlib_tofloat
    rtexit2.o(.ARM.Collect$$rtexit$$00000003) refers to libshutdown.o(.ARM.Collect$$libshutdown$$00000000) for __rt_lib_shutdown
    rtexit2.o(.ARM.Collect$$rtexit$$00000004) refers to usart.o(.text) for _sys_exit
    rtexit2.o(.ARM.exidx) refers to rtexit2.o(.ARM.Collect$$rtexit$$00000001) for .ARM.Collect$$rtexit$$00000001
    rtexit2.o(.ARM.exidx) refers to rtexit2.o(.ARM.Collect$$rtexit$$00000003) for .ARM.Collect$$rtexit$$00000003
    rtexit2.o(.ARM.exidx) refers to rtexit2.o(.ARM.Collect$$rtexit$$00000004) for .ARM.Collect$$rtexit$$00000004
    scanf_hexfp.o(.text) refers to _chval.o(.text) for _chval
    scanf_hexfp.o(.text) refers to llshl.o(.text) for __aeabi_llsl
    scanf_hexfp.o(.text) refers to ldexp.o(i.__support_ldexp) for __support_ldexp
    scanf_hexfp.o(.text) refers to narrow.o(i.__mathlib_narrow) for __mathlib_narrow
    _get_argv_nomalloc.o(.text) refers (Special) to hrguard.o(.text) for __heap_region$guard
    _get_argv_nomalloc.o(.text) refers to defsig_rtmem_outer.o(.text) for __rt_SIGRTMEM
    _get_argv_nomalloc.o(.text) refers to sys_command.o(.text) for _sys_command_string
    deqf.o(x$fpl$deqf) refers (Special) to usenofp.o(x$fpl$usenofp) for __I$use$fp
    deqf.o(x$fpl$deqf) refers to dnaninf.o(x$fpl$dnaninf) for __fpl_dnaninf
    deqf.o(x$fpl$deqf) refers to dcmpi.o(x$fpl$dcmpinf) for __fpl_dcmp_Inf
    frexp.o(i.__softfp_frexp) refers (Special) to usenofp.o(x$fpl$usenofp) for __I$use$fp
    frexp.o(i.__softfp_frexp) refers to scalbn.o(x$fpl$scalbn) for __ARM_scalbn
    frexp.o(i.frexp) refers (Special) to usenofp.o(x$fpl$usenofp) for __I$use$fp
    frexp.o(i.frexp) refers to scalbn.o(x$fpl$scalbn) for __ARM_scalbn
    sys_command.o(.text) refers (Special) to use_no_semi.o(.text) for __I$use$semihosting
    sys_command.o(.text) refers (Special) to indicate_semi.o(.text) for __semihosting_library_function
    defsig_rtmem_outer.o(.text) refers to defsig_rtmem_inner.o(.text) for __rt_SIGRTMEM_inner
    defsig_rtmem_outer.o(.text) refers to defsig_exit.o(.text) for __sig_exit
    defsig_rtmem_formal.o(.text) refers to rt_raise.o(.text) for __rt_raise
    libshutdown.o(.ARM.Collect$$libshutdown$$00000000) refers (Special) to libshutdown2.o(.ARM.Collect$$libshutdown$$00000002) for __rt_lib_shutdown_cpp_1
    libshutdown.o(.ARM.Collect$$libshutdown$$00000000) refers (Special) to libshutdown2.o(.ARM.Collect$$libshutdown$$00000007) for __rt_lib_shutdown_fp_trap_1
    libshutdown.o(.ARM.Collect$$libshutdown$$00000000) refers (Special) to libshutdown2.o(.ARM.Collect$$libshutdown$$0000000F) for __rt_lib_shutdown_heap_1
    libshutdown.o(.ARM.Collect$$libshutdown$$00000000) refers (Special) to libshutdown2.o(.ARM.Collect$$libshutdown$$00000010) for __rt_lib_shutdown_return
    libshutdown.o(.ARM.Collect$$libshutdown$$00000000) refers (Special) to libshutdown2.o(.ARM.Collect$$libshutdown$$0000000A) for __rt_lib_shutdown_signal_1
    libshutdown.o(.ARM.Collect$$libshutdown$$00000000) refers (Special) to libshutdown2.o(.ARM.Collect$$libshutdown$$00000004) for __rt_lib_shutdown_stdio_1
    libshutdown.o(.ARM.Collect$$libshutdown$$00000000) refers (Special) to libshutdown2.o(.ARM.Collect$$libshutdown$$0000000C) for __rt_lib_shutdown_user_alloc_1
    ldexp.o(i.__softfp_ldexp) refers (Special) to usenofp.o(x$fpl$usenofp) for __I$use$fp
    ldexp.o(i.__softfp_ldexp) refers to ldexp.o(i.ldexp) for ldexp
    ldexp.o(i.__support_ldexp) refers (Special) to usenofp.o(x$fpl$usenofp) for __I$use$fp
    ldexp.o(i.__support_ldexp) refers to ldexp.o(i.ldexp) for ldexp
    ldexp.o(i.ldexp) refers (Special) to usenofp.o(x$fpl$usenofp) for __I$use$fp
    ldexp.o(i.ldexp) refers to deqf.o(x$fpl$deqf) for __aeabi_cdcmpeq
    ldexp.o(i.ldexp) refers to scalbn.o(x$fpl$scalbn) for __ARM_scalbn
    ldexp.o(i.ldexp) refers to _rserrno.o(.text) for __set_errno
    ldexp.o(i.ldexp) refers to dunder.o(i.__mathlib_dbl_underflow) for __mathlib_dbl_underflow
    ldexp.o(i.ldexp) refers to dunder.o(i.__mathlib_dbl_overflow) for __mathlib_dbl_overflow
    ldexp_x.o(i.____softfp_ldexp$lsc) refers (Special) to usenofp.o(x$fpl$usenofp) for __I$use$fp
    ldexp_x.o(i.____softfp_ldexp$lsc) refers to ldexp_x.o(i.__ldexp$lsc) for __ldexp$lsc
    ldexp_x.o(i.____support_ldexp$lsc) refers (Special) to usenofp.o(x$fpl$usenofp) for __I$use$fp
    ldexp_x.o(i.____support_ldexp$lsc) refers to ldexp_x.o(i.__ldexp$lsc) for __ldexp$lsc
    ldexp_x.o(i.__ldexp$lsc) refers (Special) to usenofp.o(x$fpl$usenofp) for __I$use$fp
    ldexp_x.o(i.__ldexp$lsc) refers to deqf.o(x$fpl$deqf) for __aeabi_cdcmpeq
    ldexp_x.o(i.__ldexp$lsc) refers to scalbn.o(x$fpl$scalbn) for __ARM_scalbn
    ldexp_x.o(i.__ldexp$lsc) refers to _rserrno.o(.text) for __set_errno
    ldexp_x.o(i.__ldexp$lsc) refers to qnan.o(.constdata) for __mathlib_zero
    rt_raise.o(.text) refers to __raise.o(.text) for __raise
    rt_raise.o(.text) refers to usart.o(.text) for _sys_exit
    defsig_exit.o(.text) refers to usart.o(.text) for _sys_exit
    defsig_rtmem_inner.o(.text) refers to defsig_general.o(.text) for __default_signal_display
    __raise.o(.text) refers to defsig.o(CL$$defsig) for __default_signal_handler
    defsig_general.o(.text) refers to sys_wrch.o(.text) for _ttywrch
    sys_wrch.o(.text) refers (Special) to use_no_semi.o(.text) for __I$use$semihosting
    sys_wrch.o(.text) refers (Special) to indicate_semi.o(.text) for __semihosting_library_function
    defsig.o(CL$$defsig) refers to defsig_rtmem_inner.o(.text) for __rt_SIGRTMEM_inner
    defsig_abrt_inner.o(.text) refers to defsig_general.o(.text) for __default_signal_display
    defsig_fpe_inner.o(.text) refers to defsig_general.o(.text) for __default_signal_display
    defsig_rtred_inner.o(.text) refers to defsig_general.o(.text) for __default_signal_display
    defsig_stak_inner.o(.text) refers to defsig_general.o(.text) for __default_signal_display
    defsig_pvfn_inner.o(.text) refers to defsig_general.o(.text) for __default_signal_display
    defsig_cppl_inner.o(.text) refers to defsig_general.o(.text) for __default_signal_display
    defsig_segv_inner.o(.text) refers to defsig_general.o(.text) for __default_signal_display
    defsig_other.o(.text) refers to defsig_general.o(.text) for __default_signal_display


==============================================================================

Removing Unused input sections from the image.

    Removing main.o(.bss), (800 bytes).
    Removing sys.o(.emb_text), (6 bytes).
    Removing sys.o(.text), (12 bytes).
    Removing usart.o(.bss), (200 bytes).
    Removing core_cm3.o(.emb_text), (32 bytes).
    Removing ad8310.o(.text), (448 bytes).
    Removing ad8310.o(.data), (32 bytes).
    Removing ch2_freq_set.o(.data), (1 bytes).
    Removing stmflash.o(.text), (324 bytes).
    Removing stmflash.o(.bss), (2048 bytes).
    Removing malloc.o(.constdata), (12 bytes).
    Removing stm32f10x_bkp.o(.text), (196 bytes).
    Removing stm32f10x_pwr.o(.text), (204 bytes).
    Removing stm32f10x_exti.o(.text), (284 bytes).
    Removing stm32f10x_flash.o(.text), (1468 bytes).

15 unused section(s) (total 6067 bytes) removed from the image.

==============================================================================

Image Symbol Table

    Local Symbols

    Symbol Name                              Value     Ov Type        Size  Object(Section)

    ../clib/angel/boardlib.s                 0x00000000   Number         0  boardinit1.o ABSOLUTE
    ../clib/angel/boardlib.s                 0x00000000   Number         0  boardshut.o ABSOLUTE
    ../clib/angel/boardlib.s                 0x00000000   Number         0  boardinit3.o ABSOLUTE
    ../clib/angel/boardlib.s                 0x00000000   Number         0  boardinit2.o ABSOLUTE
    ../clib/angel/dczerorl2.s                0x00000000   Number         0  __dczerorl2.o ABSOLUTE
    ../clib/angel/handlers.s                 0x00000000   Number         0  __scatter_zi.o ABSOLUTE
    ../clib/angel/kernel.s                   0x00000000   Number         0  rtexit.o ABSOLUTE
    ../clib/angel/kernel.s                   0x00000000   Number         0  rtexit2.o ABSOLUTE
    ../clib/angel/kernel.s                   0x00000000   Number         0  __rtentry4.o ABSOLUTE
    ../clib/angel/kernel.s                   0x00000000   Number         0  __rtentry.o ABSOLUTE
    ../clib/angel/kernel.s                   0x00000000   Number         0  __rtentry2.o ABSOLUTE
    ../clib/angel/rt.s                       0x00000000   Number         0  rt_ctype_table.o ABSOLUTE
    ../clib/angel/rt.s                       0x00000000   Number         0  rt_locale_intlibspace.o ABSOLUTE
    ../clib/angel/rt.s                       0x00000000   Number         0  rt_raise.o ABSOLUTE
    ../clib/angel/rt.s                       0x00000000   Number         0  rt_locale.o ABSOLUTE
    ../clib/angel/rt.s                       0x00000000   Number         0  rt_errno_addr_intlibspace.o ABSOLUTE
    ../clib/angel/rt.s                       0x00000000   Number         0  rt_errno_addr.o ABSOLUTE
    ../clib/angel/scatter.s                  0x00000000   Number         0  __scatter.o ABSOLUTE
    ../clib/angel/startup.s                  0x00000000   Number         0  __main.o ABSOLUTE
    ../clib/angel/sys.s                      0x00000000   Number         0  libspace.o ABSOLUTE
    ../clib/angel/sys.s                      0x00000000   Number         0  use_no_semi.o ABSOLUTE
    ../clib/angel/sys.s                      0x00000000   Number         0  sys_stackheap_outer.o ABSOLUTE
    ../clib/angel/sys.s                      0x00000000   Number         0  indicate_semi.o ABSOLUTE
    ../clib/angel/sys.s                      0x00000000   Number         0  use_no_semi_2.o ABSOLUTE
    ../clib/angel/sysapp.c                   0x00000000   Number         0  sys_wrch.o ABSOLUTE
    ../clib/angel/sysapp.c                   0x00000000   Number         0  sys_command.o ABSOLUTE
    ../clib/armsys.c                         0x00000000   Number         0  argv_veneer.o ABSOLUTE
    ../clib/armsys.c                         0x00000000   Number         0  argv_veneer.o ABSOLUTE
    ../clib/armsys.c                         0x00000000   Number         0  _get_argv_nomalloc.o ABSOLUTE
    ../clib/armsys.c                         0x00000000   Number         0  no_argv.o ABSOLUTE
    ../clib/bigflt.c                         0x00000000   Number         0  bigflt0.o ABSOLUTE
    ../clib/btod.s                           0x00000000   Number         0  btod.o ABSOLUTE
    ../clib/ctype.c                          0x00000000   Number         0  isspace.o ABSOLUTE
    ../clib/fenv.c                           0x00000000   Number         0  _rserrno.o ABSOLUTE
    ../clib/heapalloc.c                      0x00000000   Number         0  hrguard.o ABSOLUTE
    ../clib/heapaux.c                        0x00000000   Number         0  heapauxi.o ABSOLUTE
    ../clib/libinit.s                        0x00000000   Number         0  libinit.o ABSOLUTE
    ../clib/libinit.s                        0x00000000   Number         0  libinit2.o ABSOLUTE
    ../clib/libinit.s                        0x00000000   Number         0  libshutdown.o ABSOLUTE
    ../clib/libinit.s                        0x00000000   Number         0  libshutdown2.o ABSOLUTE
    ../clib/locale.s                         0x00000000   Number         0  lc_numeric_c.o ABSOLUTE
    ../clib/locale.s                         0x00000000   Number         0  lc_ctype_c.o ABSOLUTE
    ../clib/longlong.s                       0x00000000   Number         0  lludiv10.o ABSOLUTE
    ../clib/longlong.s                       0x00000000   Number         0  llshl.o ABSOLUTE
    ../clib/memcpset.s                       0x00000000   Number         0  strcmpv7m.o ABSOLUTE
    ../clib/misc.s                           0x00000000   Number         0  printf_stubs.o ABSOLUTE
    ../clib/printf.c                         0x00000000   Number         0  _printf_longlong_dec.o ABSOLUTE
    ../clib/printf.c                         0x00000000   Number         0  __printf_flags.o ABSOLUTE
    ../clib/printf.c                         0x00000000   Number         0  __printf_ss.o ABSOLUTE
    ../clib/printf.c                         0x00000000   Number         0  __printf_flags_ss.o ABSOLUTE
    ../clib/printf.c                         0x00000000   Number         0  __printf_wp.o ABSOLUTE
    ../clib/printf.c                         0x00000000   Number         0  __printf_flags_wp.o ABSOLUTE
    ../clib/printf.c                         0x00000000   Number         0  __printf_flags_ss_wp.o ABSOLUTE
    ../clib/printf.c                         0x00000000   Number         0  _printf_pad.o ABSOLUTE
    ../clib/printf.c                         0x00000000   Number         0  _printf_fp_infnan.o ABSOLUTE
    ../clib/printf.c                         0x00000000   Number         0  __2sprintf.o ABSOLUTE
    ../clib/printf.c                         0x00000000   Number         0  __printf_nopercent.o ABSOLUTE
    ../clib/printf.c                         0x00000000   Number         0  _printf_intcommon.o ABSOLUTE
    ../clib/printf.c                         0x00000000   Number         0  __2printf.o ABSOLUTE
    ../clib/printf.c                         0x00000000   Number         0  __printf_ss_wp.o ABSOLUTE
    ../clib/printf.c                         0x00000000   Number         0  _printf_fp_dec.o ABSOLUTE
    ../clib/printf.c                         0x00000000   Number         0  _printf_char_common.o ABSOLUTE
    ../clib/printf.c                         0x00000000   Number         0  noretval__2printf.o ABSOLUTE
    ../clib/printf.c                         0x00000000   Number         0  noretval__2sprintf.o ABSOLUTE
    ../clib/printf.c                         0x00000000   Number         0  _sputc.o ABSOLUTE
    ../clib/printf.c                         0x00000000   Number         0  __printf.o ABSOLUTE
    ../clib/printf.c                         0x00000000   Number         0  _printf_char_file.o ABSOLUTE
    ../clib/printf.c                         0x00000000   Number         0  _printf_dec.o ABSOLUTE
    ../clib/printf_percent.s                 0x00000000   Number         0  _printf_llu.o ABSOLUTE
    ../clib/printf_percent.s                 0x00000000   Number         0  _printf_percent_end.o ABSOLUTE
    ../clib/printf_percent.s                 0x00000000   Number         0  _printf_ll.o ABSOLUTE
    ../clib/printf_percent.s                 0x00000000   Number         0  _printf_u.o ABSOLUTE
    ../clib/printf_percent.s                 0x00000000   Number         0  _printf_f.o ABSOLUTE
    ../clib/printf_percent.s                 0x00000000   Number         0  _printf_percent.o ABSOLUTE
    ../clib/scanf.c                          0x00000000   Number         0  atoi.o ABSOLUTE
    ../clib/scanf.c                          0x00000000   Number         0  _sgetc.o ABSOLUTE
    ../clib/scanf.c                          0x00000000   Number         0  strtol.o ABSOLUTE
    ../clib/scanf.c                          0x00000000   Number         0  strtod.o ABSOLUTE
    ../clib/scanf.c                          0x00000000   Number         0  _chval.o ABSOLUTE
    ../clib/scanf.c                          0x00000000   Number         0  scanf_fp.o ABSOLUTE
    ../clib/scanf.c                          0x00000000   Number         0  scanf_hexfp.o ABSOLUTE
    ../clib/scanf.c                          0x00000000   Number         0  scanf_infnan.o ABSOLUTE
    ../clib/scanf.c                          0x00000000   Number         0  _strtoul.o ABSOLUTE
    ../clib/signal.c                         0x00000000   Number         0  defsig_rtmem_inner.o ABSOLUTE
    ../clib/signal.c                         0x00000000   Number         0  defsig_other.o ABSOLUTE
    ../clib/signal.c                         0x00000000   Number         0  defsig_rtmem_formal.o ABSOLUTE
    ../clib/signal.c                         0x00000000   Number         0  defsig_rtmem_outer.o ABSOLUTE
    ../clib/signal.c                         0x00000000   Number         0  defsig_segv_inner.o ABSOLUTE
    ../clib/signal.c                         0x00000000   Number         0  defsig_cppl_inner.o ABSOLUTE
    ../clib/signal.c                         0x00000000   Number         0  defsig_pvfn_inner.o ABSOLUTE
    ../clib/signal.c                         0x00000000   Number         0  defsig_stak_inner.o ABSOLUTE
    ../clib/signal.c                         0x00000000   Number         0  defsig_rtred_inner.o ABSOLUTE
    ../clib/signal.c                         0x00000000   Number         0  defsig_fpe_inner.o ABSOLUTE
    ../clib/signal.c                         0x00000000   Number         0  defsig_abrt_inner.o ABSOLUTE
    ../clib/signal.c                         0x00000000   Number         0  defsig_exit.o ABSOLUTE
    ../clib/signal.c                         0x00000000   Number         0  defsig_general.o ABSOLUTE
    ../clib/signal.c                         0x00000000   Number         0  __raise.o ABSOLUTE
    ../clib/signal.s                         0x00000000   Number         0  defsig.o ABSOLUTE
    ../clib/stdio.c                          0x00000000   Number         0  ferror.o ABSOLUTE
    ../clib/stdio.c                          0x00000000   Number         0  ferror_locked.o ABSOLUTE
    ../clib/stdlib.c                         0x00000000   Number         0  exit.o ABSOLUTE
    ../fplib/d2f.s                           0x00000000   Number         0  d2f.o ABSOLUTE
    ../fplib/daddsub.s                       0x00000000   Number         0  daddsub_clz.o ABSOLUTE
    ../fplib/dcheck1.s                       0x00000000   Number         0  dcheck1.o ABSOLUTE
    ../fplib/dcmpi.s                         0x00000000   Number         0  dcmpi.o ABSOLUTE
    ../fplib/ddiv.s                          0x00000000   Number         0  ddiv.o ABSOLUTE
    ../fplib/deqf.s                          0x00000000   Number         0  deqf.o ABSOLUTE
    ../fplib/dfixu.s                         0x00000000   Number         0  dfixu.o ABSOLUTE
    ../fplib/dfixull.s                       0x00000000   Number         0  dfixull.o ABSOLUTE
    ../fplib/dflt.s                          0x00000000   Number         0  dflt_clz.o ABSOLUTE
    ../fplib/dfltll.s                        0x00000000   Number         0  dfltll_clz.o ABSOLUTE
    ../fplib/dleqf.s                         0x00000000   Number         0  dleqf.o ABSOLUTE
    ../fplib/dmul.s                          0x00000000   Number         0  dmul.o ABSOLUTE
    ../fplib/dnaninf.s                       0x00000000   Number         0  dnaninf.o ABSOLUTE
    ../fplib/dretinf.s                       0x00000000   Number         0  dretinf.o ABSOLUTE
    ../fplib/drleqf.s                        0x00000000   Number         0  drleqf.o ABSOLUTE
    ../fplib/dsqrt.s                         0x00000000   Number         0  dsqrt_noumaal.o ABSOLUTE
    ../fplib/f2d.s                           0x00000000   Number         0  f2d.o ABSOLUTE
    ../fplib/faddsub.s                       0x00000000   Number         0  faddsub_clz.o ABSOLUTE
    ../fplib/fcmpi.s                         0x00000000   Number         0  fcmpi.o ABSOLUTE
    ../fplib/fdiv.s                          0x00000000   Number         0  fdiv.o ABSOLUTE
    ../fplib/feqf.s                          0x00000000   Number         0  feqf.o ABSOLUTE
    ../fplib/ffixu.s                         0x00000000   Number         0  ffixu.o ABSOLUTE
    ../fplib/fflt.s                          0x00000000   Number         0  fflt_clz.o ABSOLUTE
    ../fplib/fleqf.s                         0x00000000   Number         0  fleqf.o ABSOLUTE
    ../fplib/fmul.s                          0x00000000   Number         0  fmul.o ABSOLUTE
    ../fplib/fnaninf.s                       0x00000000   Number         0  fnaninf.o ABSOLUTE
    ../fplib/fpconst.s                       0x00000000   Number         0  fpconst.o ABSOLUTE
    ../fplib/fpinit.s                        0x00000000   Number         0  fpinit.o ABSOLUTE
    ../fplib/fretinf.s                       0x00000000   Number         0  fretinf.o ABSOLUTE
    ../fplib/frleqf.s                        0x00000000   Number         0  frleqf.o ABSOLUTE
    ../fplib/istatus.s                       0x00000000   Number         0  istatus.o ABSOLUTE
    ../fplib/printf1.s                       0x00000000   Number         0  printf1.o ABSOLUTE
    ../fplib/retnan.s                        0x00000000   Number         0  retnan.o ABSOLUTE
    ../fplib/scalbn.s                        0x00000000   Number         0  scalbn.o ABSOLUTE
    ../fplib/scanf1.s                        0x00000000   Number         0  scanf1.o ABSOLUTE
    ../fplib/scanf2.s                        0x00000000   Number         0  scanf2.o ABSOLUTE
    ../fplib/scanf2a.s                       0x00000000   Number         0  scanf2a.o ABSOLUTE
    ../fplib/scanf2b.s                       0x00000000   Number         0  scanf2b.o ABSOLUTE
    ../fplib/trapv.s                         0x00000000   Number         0  trapv.o ABSOLUTE
    ../fplib/usenofp.s                       0x00000000   Number         0  usenofp.o ABSOLUTE
    ../mathlib/atof.c                        0x00000000   Number         0  atof.o ABSOLUTE
    ../mathlib/dunder.c                      0x00000000   Number         0  dunder.o ABSOLUTE
    ../mathlib/fpclassify.c                  0x00000000   Number         0  fpclassify.o ABSOLUTE
    ../mathlib/frexp.c                       0x00000000   Number         0  frexp.o ABSOLUTE
    ../mathlib/ldexp.c                       0x00000000   Number         0  ldexp.o ABSOLUTE
    ../mathlib/ldexp.c                       0x00000000   Number         0  ldexp_x.o ABSOLUTE
    ../mathlib/narrow.c                      0x00000000   Number         0  narrow.o ABSOLUTE
    ../mathlib/poly.c                        0x00000000   Number         0  poly.o ABSOLUTE
    ../mathlib/pow.c                         0x00000000   Number         0  pow_x.o ABSOLUTE
    ../mathlib/pow.c                         0x00000000   Number         0  pow.o ABSOLUTE
    ../mathlib/qnan.c                        0x00000000   Number         0  qnan.o ABSOLUTE
    ../mathlib/sqrt.c                        0x00000000   Number         0  sqrt_x.o ABSOLUTE
    ../mathlib/sqrt.c                        0x00000000   Number         0  sqrt.o ABSOLUTE
    ..\CORE\core_cm3.c                       0x00000000   Number         0  core_cm3.o ABSOLUTE
    ..\CORE\startup_stm32f10x_hd.s           0x00000000   Number         0  startup_stm32f10x_hd.o ABSOLUTE
    ..\HARDWARE\3_12_OLED\oled.c             0x00000000   Number         0  oled.o ABSOLUTE
    ..\HARDWARE\AD9912\AD9912_drive.c        0x00000000   Number         0  ad9912_drive.o ABSOLUTE
    ..\HARDWARE\ADC\adc.c                    0x00000000   Number         0  adc.o ABSOLUTE
    ..\HARDWARE\AMP_SET\Amp_Set.c            0x00000000   Number         0  amp_set.o ABSOLUTE
    ..\HARDWARE\BSP\bsp.c                    0x00000000   Number         0  bsp.o ABSOLUTE
    ..\HARDWARE\DAC\dac.c                    0x00000000   Number         0  dac.o ABSOLUTE
    ..\HARDWARE\Detector\AD8310.c            0x00000000   Number         0  ad8310.o ABSOLUTE
    ..\HARDWARE\Detector\ADL5513.c           0x00000000   Number         0  adl5513.o ABSOLUTE
    ..\HARDWARE\EC11\EC11_Key_Process.c      0x00000000   Number         0  ec11_key_process.o ABSOLUTE
    ..\HARDWARE\EC11\EC11_Spin_Process.c     0x00000000   Number         0  ec11_spin_process.o ABSOLUTE
    ..\HARDWARE\EC11\bsp_ec11.c              0x00000000   Number         0  bsp_ec11.o ABSOLUTE
    ..\HARDWARE\Freq_Set\CH2_Freq_Set.c      0x00000000   Number         0  ch2_freq_set.o ABSOLUTE
    ..\HARDWARE\HMC241\HMC241.c              0x00000000   Number         0  hmc241.o ABSOLUTE
    ..\HARDWARE\KEY\Key_Scan.c               0x00000000   Number         0  key_scan.o ABSOLUTE
    ..\HARDWARE\KEY\matrix_key.c             0x00000000   Number         0  matrix_key.o ABSOLUTE
    ..\HARDWARE\LED\led.c                    0x00000000   Number         0  led.o ABSOLUTE
    ..\HARDWARE\PE4302\PE4302.c              0x00000000   Number         0  pe4302.o ABSOLUTE
    ..\HARDWARE\PLL_CONFIG\ALL_LO_Init.c     0x00000000   Number         0  all_lo_init.o ABSOLUTE
    ..\HARDWARE\PLL_CONFIG\LO_LMX2592_Freq_Set.c 0x00000000   Number         0  lo_lmx2592_freq_set.o ABSOLUTE
    ..\HARDWARE\PLL_CONFIG\PLL_SPI_init.c    0x00000000   Number         0  pll_spi_init.o ABSOLUTE
    ..\HARDWARE\SPI\spi.c                    0x00000000   Number         0  spi.o ABSOLUTE
    ..\HARDWARE\STMFLASH\stmflash.c          0x00000000   Number         0  stmflash.o ABSOLUTE
    ..\HARDWARE\UI\CW_menu.c                 0x00000000   Number         0  cw_menu.o ABSOLUTE
    ..\HARDWARE\UI\Key_S1_Process.c          0x00000000   Number         0  key_s1_process.o ABSOLUTE
    ..\HARDWARE\UI\Key_S2_Process.c          0x00000000   Number         0  key_s2_process.o ABSOLUTE
    ..\HARDWARE\UI\Key_S3_Process.c          0x00000000   Number         0  key_s3_process.o ABSOLUTE
    ..\HARDWARE\UI\Main_menu.c               0x00000000   Number         0  main_menu.o ABSOLUTE
    ..\HARDWARE\UI\Oled_Task.c               0x00000000   Number         0  oled_task.o ABSOLUTE
    ..\HARDWARE\UI\Power_menu.c              0x00000000   Number         0  power_menu.o ABSOLUTE
    ..\HARDWARE\timer\timer.c                0x00000000   Number         0  timer.o ABSOLUTE
    ..\MALLOC\malloc.c                       0x00000000   Number         0  malloc.o ABSOLUTE
    ..\STM32F10x_FWLib\src\misc.c            0x00000000   Number         0  misc.o ABSOLUTE
    ..\STM32F10x_FWLib\src\stm32f10x_adc.c   0x00000000   Number         0  stm32f10x_adc.o ABSOLUTE
    ..\STM32F10x_FWLib\src\stm32f10x_bkp.c   0x00000000   Number         0  stm32f10x_bkp.o ABSOLUTE
    ..\STM32F10x_FWLib\src\stm32f10x_dac.c   0x00000000   Number         0  stm32f10x_dac.o ABSOLUTE
    ..\STM32F10x_FWLib\src\stm32f10x_exti.c  0x00000000   Number         0  stm32f10x_exti.o ABSOLUTE
    ..\STM32F10x_FWLib\src\stm32f10x_flash.c 0x00000000   Number         0  stm32f10x_flash.o ABSOLUTE
    ..\STM32F10x_FWLib\src\stm32f10x_gpio.c  0x00000000   Number         0  stm32f10x_gpio.o ABSOLUTE
    ..\STM32F10x_FWLib\src\stm32f10x_pwr.c   0x00000000   Number         0  stm32f10x_pwr.o ABSOLUTE
    ..\STM32F10x_FWLib\src\stm32f10x_rcc.c   0x00000000   Number         0  stm32f10x_rcc.o ABSOLUTE
    ..\STM32F10x_FWLib\src\stm32f10x_spi.c   0x00000000   Number         0  stm32f10x_spi.o ABSOLUTE
    ..\STM32F10x_FWLib\src\stm32f10x_tim.c   0x00000000   Number         0  stm32f10x_tim.o ABSOLUTE
    ..\STM32F10x_FWLib\src\stm32f10x_usart.c 0x00000000   Number         0  stm32f10x_usart.o ABSOLUTE
    ..\SYSTEM\delay\delay.c                  0x00000000   Number         0  delay.o ABSOLUTE
    ..\SYSTEM\sys\sys.c                      0x00000000   Number         0  sys.o ABSOLUTE
    ..\SYSTEM\usart\usart.c                  0x00000000   Number         0  usart.o ABSOLUTE
    ..\\CORE\\core_cm3.c                     0x00000000   Number         0  core_cm3.o ABSOLUTE
    ..\\SYSTEM\\sys\\sys.c                   0x00000000   Number         0  sys.o ABSOLUTE
    dc.s                                     0x00000000   Number         0  dc.o ABSOLUTE
    main.c                                   0x00000000   Number         0  main.o ABSOLUTE
    stm32f10x_it.c                           0x00000000   Number         0  stm32f10x_it.o ABSOLUTE
    system_stm32f10x.c                       0x00000000   Number         0  system_stm32f10x.o ABSOLUTE
    RESET                                    0x08000000   Section      304  startup_stm32f10x_hd.o(RESET)
    !!!main                                  0x08000130   Section        8  __main.o(!!!main)
    !!!scatter                               0x08000138   Section       52  __scatter.o(!!!scatter)
    !!dczerorl2                              0x0800016c   Section       90  __dczerorl2.o(!!dczerorl2)
    !!handler_zi                             0x080001c8   Section       28  __scatter_zi.o(!!handler_zi)
    .ARM.Collect$$_printf_percent$$00000000  0x080001e4   Section        0  _printf_percent.o(.ARM.Collect$$_printf_percent$$00000000)
    .ARM.Collect$$_printf_percent$$00000003  0x080001e4   Section        6  _printf_f.o(.ARM.Collect$$_printf_percent$$00000003)
    .ARM.Collect$$_printf_percent$$00000007  0x080001ea   Section       10  _printf_ll.o(.ARM.Collect$$_printf_percent$$00000007)
    .ARM.Collect$$_printf_percent$$0000000A  0x080001f4   Section        6  _printf_u.o(.ARM.Collect$$_printf_percent$$0000000A)
    .ARM.Collect$$_printf_percent$$0000000F  0x080001fa   Section        6  _printf_llu.o(.ARM.Collect$$_printf_percent$$0000000F)
    .ARM.Collect$$_printf_percent$$00000017  0x08000200   Section        4  _printf_percent_end.o(.ARM.Collect$$_printf_percent$$00000017)
    .ARM.Collect$$libinit$$00000000          0x08000204   Section        2  libinit.o(.ARM.Collect$$libinit$$00000000)
    .ARM.Collect$$libinit$$00000002          0x08000206   Section        0  libinit2.o(.ARM.Collect$$libinit$$00000002)
    .ARM.Collect$$libinit$$00000004          0x08000206   Section        0  libinit2.o(.ARM.Collect$$libinit$$00000004)
    .ARM.Collect$$libinit$$0000000A          0x08000206   Section        0  libinit2.o(.ARM.Collect$$libinit$$0000000A)
    .ARM.Collect$$libinit$$0000000C          0x08000206   Section        0  libinit2.o(.ARM.Collect$$libinit$$0000000C)
    .ARM.Collect$$libinit$$0000000E          0x08000206   Section        0  libinit2.o(.ARM.Collect$$libinit$$0000000E)
    .ARM.Collect$$libinit$$0000000F          0x08000206   Section        6  libinit2.o(.ARM.Collect$$libinit$$0000000F)
    .ARM.Collect$$libinit$$00000011          0x0800020c   Section        0  libinit2.o(.ARM.Collect$$libinit$$00000011)
    .ARM.Collect$$libinit$$00000012          0x0800020c   Section       12  libinit2.o(.ARM.Collect$$libinit$$00000012)
    .ARM.Collect$$libinit$$00000013          0x08000218   Section        0  libinit2.o(.ARM.Collect$$libinit$$00000013)
    .ARM.Collect$$libinit$$00000015          0x08000218   Section        0  libinit2.o(.ARM.Collect$$libinit$$00000015)
    .ARM.Collect$$libinit$$00000016          0x08000218   Section       10  libinit2.o(.ARM.Collect$$libinit$$00000016)
    .ARM.Collect$$libinit$$00000017          0x08000222   Section        0  libinit2.o(.ARM.Collect$$libinit$$00000017)
    .ARM.Collect$$libinit$$00000019          0x08000222   Section        0  libinit2.o(.ARM.Collect$$libinit$$00000019)
    .ARM.Collect$$libinit$$0000001B          0x08000222   Section        0  libinit2.o(.ARM.Collect$$libinit$$0000001B)
    .ARM.Collect$$libinit$$0000001D          0x08000222   Section        0  libinit2.o(.ARM.Collect$$libinit$$0000001D)
    .ARM.Collect$$libinit$$0000001F          0x08000222   Section        0  libinit2.o(.ARM.Collect$$libinit$$0000001F)
    .ARM.Collect$$libinit$$00000021          0x08000222   Section        0  libinit2.o(.ARM.Collect$$libinit$$00000021)
    .ARM.Collect$$libinit$$00000023          0x08000222   Section        0  libinit2.o(.ARM.Collect$$libinit$$00000023)
    .ARM.Collect$$libinit$$00000025          0x08000222   Section        0  libinit2.o(.ARM.Collect$$libinit$$00000025)
    .ARM.Collect$$libinit$$0000002C          0x08000222   Section        0  libinit2.o(.ARM.Collect$$libinit$$0000002C)
    .ARM.Collect$$libinit$$0000002E          0x08000222   Section        0  libinit2.o(.ARM.Collect$$libinit$$0000002E)
    .ARM.Collect$$libinit$$00000030          0x08000222   Section        0  libinit2.o(.ARM.Collect$$libinit$$00000030)
    .ARM.Collect$$libinit$$00000032          0x08000222   Section        0  libinit2.o(.ARM.Collect$$libinit$$00000032)
    .ARM.Collect$$libinit$$00000033          0x08000222   Section        2  libinit2.o(.ARM.Collect$$libinit$$00000033)
    .ARM.Collect$$libshutdown$$00000000      0x08000224   Section        2  libshutdown.o(.ARM.Collect$$libshutdown$$00000000)
    .ARM.Collect$$libshutdown$$00000002      0x08000226   Section        0  libshutdown2.o(.ARM.Collect$$libshutdown$$00000002)
    .ARM.Collect$$libshutdown$$00000004      0x08000226   Section        0  libshutdown2.o(.ARM.Collect$$libshutdown$$00000004)
    .ARM.Collect$$libshutdown$$00000007      0x08000226   Section        0  libshutdown2.o(.ARM.Collect$$libshutdown$$00000007)
    .ARM.Collect$$libshutdown$$0000000A      0x08000226   Section        0  libshutdown2.o(.ARM.Collect$$libshutdown$$0000000A)
    .ARM.Collect$$libshutdown$$0000000C      0x08000226   Section        0  libshutdown2.o(.ARM.Collect$$libshutdown$$0000000C)
    .ARM.Collect$$libshutdown$$0000000F      0x08000226   Section        0  libshutdown2.o(.ARM.Collect$$libshutdown$$0000000F)
    .ARM.Collect$$libshutdown$$00000010      0x08000226   Section        2  libshutdown2.o(.ARM.Collect$$libshutdown$$00000010)
    .ARM.Collect$$rtentry$$00000000          0x08000228   Section        0  __rtentry.o(.ARM.Collect$$rtentry$$00000000)
    .ARM.Collect$$rtentry$$00000002          0x08000228   Section        0  __rtentry2.o(.ARM.Collect$$rtentry$$00000002)
    .ARM.Collect$$rtentry$$00000004          0x08000228   Section        6  __rtentry4.o(.ARM.Collect$$rtentry$$00000004)
    .ARM.Collect$$rtentry$$00000009          0x0800022e   Section        0  __rtentry2.o(.ARM.Collect$$rtentry$$00000009)
    .ARM.Collect$$rtentry$$0000000A          0x0800022e   Section        4  __rtentry2.o(.ARM.Collect$$rtentry$$0000000A)
    .ARM.Collect$$rtentry$$0000000C          0x08000232   Section        0  __rtentry2.o(.ARM.Collect$$rtentry$$0000000C)
    .ARM.Collect$$rtentry$$0000000D          0x08000232   Section        8  __rtentry2.o(.ARM.Collect$$rtentry$$0000000D)
    .ARM.Collect$$rtexit$$00000000           0x0800023a   Section        2  rtexit.o(.ARM.Collect$$rtexit$$00000000)
    .ARM.Collect$$rtexit$$00000002           0x0800023c   Section        0  rtexit2.o(.ARM.Collect$$rtexit$$00000002)
    .ARM.Collect$$rtexit$$00000003           0x0800023c   Section        4  rtexit2.o(.ARM.Collect$$rtexit$$00000003)
    .ARM.Collect$$rtexit$$00000004           0x08000240   Section        6  rtexit2.o(.ARM.Collect$$rtexit$$00000004)
    .text                                    0x08000248   Section        0  main.o(.text)
    .text                                    0x08000758   Section        0  stm32f10x_it.o(.text)
    .text                                    0x08000774   Section        0  system_stm32f10x.o(.text)
    SetSysClockTo72                          0x08000775   Thumb Code   214  system_stm32f10x.o(.text)
    SetSysClock                              0x0800084b   Thumb Code     8  system_stm32f10x.o(.text)
    .text                                    0x08000954   Section        0  led.o(.text)
    .text                                    0x080009b8   Section        0  adc.o(.text)
    .text                                    0x08000c18   Section        0  timer.o(.text)
    .text                                    0x08000ee8   Section        0  bsp_ec11.o(.text)
    .text                                    0x08000f30   Section        0  spi.o(.text)
    .text                                    0x080010b0   Section        0  oled.o(.text)
    .text                                    0x08001d30   Section        0  dac.o(.text)
    .text                                    0x08001dd8   Section        0  matrix_key.o(.text)
    IsKeyDownS1                              0x08001dd9   Thumb Code    18  matrix_key.o(.text)
    IsKeyDownS2                              0x08001deb   Thumb Code    18  matrix_key.o(.text)
    IsKeyDownS3                              0x08001dfd   Thumb Code    18  matrix_key.o(.text)
    IsKeyDownS4                              0x08001e0f   Thumb Code    18  matrix_key.o(.text)
    IsKeyDownENT                             0x08001e21   Thumb Code    18  matrix_key.o(.text)
    bsp_InitKeyVar                           0x08001e33   Thumb Code   110  matrix_key.o(.text)
    bsp_InitKeyHard                          0x08001ea1   Thumb Code   136  matrix_key.o(.text)
    bsp_DetectKey                            0x08001fe1   Thumb Code   198  matrix_key.o(.text)
    .text                                    0x080020e0   Section        0  bsp.o(.text)
    .text                                    0x080022a0   Section        0  key_scan.o(.text)
    .text                                    0x0800243c   Section        0  delay.o(.text)
    .text                                    0x08002510   Section        0  usart.o(.text)
    .text                                    0x080025d0   Section       64  startup_stm32f10x_hd.o(.text)
    .text                                    0x08002610   Section        0  main_menu.o(.text)
    .text                                    0x08002758   Section        0  cw_menu.o(.text)
    .text                                    0x08002c4c   Section        0  power_menu.o(.text)
    .text                                    0x08002d2c   Section        0  oled_task.o(.text)
    .text                                    0x08002e2c   Section        0  key_s1_process.o(.text)
    .text                                    0x08002e90   Section        0  key_s2_process.o(.text)
    .text                                    0x08002e94   Section        0  key_s3_process.o(.text)
    .text                                    0x08002f4c   Section        0  ec11_key_process.o(.text)
    .text                                    0x08002ffc   Section        0  ec11_spin_process.o(.text)
    .text                                    0x08003bb4   Section        0  pll_spi_init.o(.text)
    .text                                    0x08003ed4   Section        0  all_lo_init.o(.text)
    .text                                    0x080040a8   Section        0  lo_lmx2592_freq_set.o(.text)
    .text                                    0x08004784   Section        0  ad9912_drive.o(.text)
    .text                                    0x08004f20   Section        0  pe4302.o(.text)
    .text                                    0x08005018   Section        0  hmc241.o(.text)
    .text                                    0x080050fc   Section        0  adl5513.o(.text)
    .text                                    0x080052b8   Section        0  amp_set.o(.text)
    .text                                    0x08005804   Section        0  ch2_freq_set.o(.text)
    .text                                    0x08005a40   Section        0  malloc.o(.text)
    .text                                    0x08005be0   Section        0  stm32f10x_gpio.o(.text)
    .text                                    0x08005f3c   Section        0  stm32f10x_rcc.o(.text)
    .text                                    0x080062e0   Section        0  stm32f10x_usart.o(.text)
    .text                                    0x080066e8   Section        0  misc.o(.text)
    .text                                    0x080067c4   Section        0  stm32f10x_adc.o(.text)
    .text                                    0x08006c14   Section        0  stm32f10x_tim.o(.text)
    TI4_Config                               0x080070bb   Thumb Code   130  stm32f10x_tim.o(.text)
    TI3_Config                               0x0800714f   Thumb Code   122  stm32f10x_tim.o(.text)
    TI2_Config                               0x080071e3   Thumb Code   130  stm32f10x_tim.o(.text)
    TI1_Config                               0x08007277   Thumb Code   108  stm32f10x_tim.o(.text)
    .text                                    0x08007a30   Section        0  stm32f10x_spi.o(.text)
    .text                                    0x08007d3c   Section        0  stm32f10x_dac.o(.text)
    .text                                    0x08007ec8   Section        2  use_no_semi_2.o(.text)
    .text                                    0x08007ecc   Section        0  noretval__2printf.o(.text)
    .text                                    0x08007ee4   Section        0  noretval__2sprintf.o(.text)
    .text                                    0x08007f0c   Section        0  _printf_pad.o(.text)
    .text                                    0x08007f5c   Section        0  _printf_dec.o(.text)
    .text                                    0x08007fd4   Section        0  _printf_longlong_dec.o(.text)
    .text                                    0x08008050   Section        0  __printf_flags_ss_wp.o(.text)
    .text                                    0x080081d8   Section        0  atoi.o(.text)
    .text                                    0x080081f2   Section        0  heapauxi.o(.text)
    .text                                    0x080081f8   Section        2  use_no_semi.o(.text)
    .text                                    0x080081fc   Section        8  rt_errno_addr_intlibspace.o(.text)
    .text                                    0x08008204   Section      138  lludiv10.o(.text)
    .text                                    0x0800828e   Section        0  _rserrno.o(.text)
    .text                                    0x080082a4   Section        0  _printf_intcommon.o(.text)
    .text                                    0x08008356   Section        0  _printf_fp_dec.o(.text)
    _fp_digits                               0x08008359   Thumb Code   428  _printf_fp_dec.o(.text)
    .text                                    0x08008770   Section        0  _printf_char_common.o(.text)
    _printf_input_char                       0x08008771   Thumb Code    10  _printf_char_common.o(.text)
    .text                                    0x080087a0   Section        0  _sputc.o(.text)
    .text                                    0x080087ac   Section        0  _printf_char_file.o(.text)
    .text                                    0x080087d0   Section        0  strtod.o(.text)
    _local_sscanf                            0x080087d1   Thumb Code    60  strtod.o(.text)
    .text                                    0x08008874   Section        0  strtol.o(.text)
    .text                                    0x080088e4   Section        8  libspace.o(.text)
    .text                                    0x080088ec   Section       16  rt_ctype_table.o(.text)
    .text                                    0x080088fc   Section        8  rt_locale_intlibspace.o(.text)
    .text                                    0x08008904   Section        0  isspace.o(.text)
    .text                                    0x08008918   Section        0  _printf_fp_infnan.o(.text)
    .text                                    0x08008998   Section        0  _sgetc.o(.text)
    .text                                    0x080089d8   Section        0  _strtoul.o(.text)
    .text                                    0x08008a78   Section        0  bigflt0.o(.text)
    .text                                    0x08008b54   Section        0  ferror.o(.text)
    .text                                    0x08008b5c   Section       74  sys_stackheap_outer.o(.text)
    .text                                    0x08008ba6   Section        0  _chval.o(.text)
    .text                                    0x08008bc4   Section        0  scanf_fp.o(.text)
    _fp_value                                0x08008bc5   Thumb Code   508  scanf_fp.o(.text)
    .text                                    0x08009068   Section        0  exit.o(.text)
    .text                                    0x0800907c   Section      128  strcmpv7m.o(.text)
    .text                                    0x080090fc   Section        0  scanf_hexfp.o(.text)
    .text                                    0x0800941c   Section        0  scanf_infnan.o(.text)
    .text                                    0x08009550   Section       38  llshl.o(.text)
    CL$$btod_d2e                             0x08009576   Section       62  btod.o(CL$$btod_d2e)
    CL$$btod_d2e_denorm_low                  0x080095b4   Section       70  btod.o(CL$$btod_d2e_denorm_low)
    CL$$btod_d2e_norm_op1                    0x080095fa   Section       96  btod.o(CL$$btod_d2e_norm_op1)
    CL$$btod_div_common                      0x0800965a   Section      824  btod.o(CL$$btod_div_common)
    CL$$btod_e2d                             0x08009994   Section       84  btod.o(CL$$btod_e2d)
    CL$$btod_e2e                             0x080099e8   Section      198  btod.o(CL$$btod_e2e)
    CL$$btod_ediv                            0x08009aae   Section       40  btod.o(CL$$btod_ediv)
    CL$$btod_edivd                           0x08009ad6   Section       40  btod.o(CL$$btod_edivd)
    CL$$btod_emul                            0x08009afe   Section       40  btod.o(CL$$btod_emul)
    CL$$btod_emuld                           0x08009b26   Section       40  btod.o(CL$$btod_emuld)
    CL$$btod_mult_common                     0x08009b4e   Section      580  btod.o(CL$$btod_mult_common)
    i.__ARM_fpclassify                       0x08009d92   Section        0  fpclassify.o(i.__ARM_fpclassify)
    i.__kernel_poly                          0x08009dba   Section        0  poly.o(i.__kernel_poly)
    i.__mathlib_dbl_divzero                  0x08009e64   Section        0  dunder.o(i.__mathlib_dbl_divzero)
    i.__mathlib_dbl_infnan2                  0x08009e74   Section        0  dunder.o(i.__mathlib_dbl_infnan2)
    i.__mathlib_dbl_invalid                  0x08009e78   Section        0  dunder.o(i.__mathlib_dbl_invalid)
    i.__mathlib_dbl_overflow                 0x08009e84   Section        0  dunder.o(i.__mathlib_dbl_overflow)
    i.__mathlib_dbl_underflow                0x08009e94   Section        0  dunder.o(i.__mathlib_dbl_underflow)
    i.__mathlib_narrow                       0x08009ea4   Section        0  narrow.o(i.__mathlib_narrow)
    i.__mathlib_tofloat                      0x08009eb4   Section        0  narrow.o(i.__mathlib_tofloat)
    i.__support_ldexp                        0x08009f3c   Section        0  ldexp.o(i.__support_ldexp)
    i._is_digit                              0x08009f52   Section        0  __printf_wp.o(i._is_digit)
    i.atof                                   0x08009f60   Section        0  atof.o(i.atof)
    i.frexp                                  0x08009f8c   Section        0  frexp.o(i.frexp)
    i.ldexp                                  0x08009fe4   Section        0  ldexp.o(i.ldexp)
    i.pow                                    0x0800a058   Section        0  pow.o(i.pow)
    i.sqrt                                   0x0800aa30   Section        0  sqrt.o(i.sqrt)
    locale$$code                             0x0800aa7c   Section       44  lc_numeric_c.o(locale$$code)
    locale$$code                             0x0800aaa8   Section       44  lc_ctype_c.o(locale$$code)
    x$fpl$d2f                                0x0800aad4   Section       98  d2f.o(x$fpl$d2f)
    x$fpl$dadd                               0x0800ab38   Section      336  daddsub_clz.o(x$fpl$dadd)
    _dadd1                                   0x0800ab49   Thumb Code     0  daddsub_clz.o(x$fpl$dadd)
    x$fpl$dcheck1                            0x0800ac88   Section       16  dcheck1.o(x$fpl$dcheck1)
    x$fpl$dcmpinf                            0x0800ac98   Section       24  dcmpi.o(x$fpl$dcmpinf)
    x$fpl$ddiv                               0x0800acb0   Section      688  ddiv.o(x$fpl$ddiv)
    ddiv_entry                               0x0800acb7   Thumb Code     0  ddiv.o(x$fpl$ddiv)
    x$fpl$deqf                               0x0800af60   Section      120  deqf.o(x$fpl$deqf)
    x$fpl$dfixu                              0x0800afd8   Section       90  dfixu.o(x$fpl$dfixu)
    x$fpl$dflt                               0x0800b032   Section       46  dflt_clz.o(x$fpl$dflt)
    x$fpl$dfltu                              0x0800b060   Section       38  dflt_clz.o(x$fpl$dfltu)
    x$fpl$dfltull                            0x0800b088   Section      138  dfltll_clz.o(x$fpl$dfltull)
    x$fpl$dleqf                              0x0800b114   Section      120  dleqf.o(x$fpl$dleqf)
    x$fpl$dmul                               0x0800b18c   Section      340  dmul.o(x$fpl$dmul)
    x$fpl$dnaninf                            0x0800b2e0   Section      156  dnaninf.o(x$fpl$dnaninf)
    x$fpl$dretinf                            0x0800b37c   Section       12  dretinf.o(x$fpl$dretinf)
    x$fpl$drleqf                             0x0800b388   Section      108  drleqf.o(x$fpl$drleqf)
    x$fpl$drsb                               0x0800b3f4   Section       22  daddsub_clz.o(x$fpl$drsb)
    x$fpl$dsqrt                              0x0800b40c   Section      460  dsqrt_noumaal.o(x$fpl$dsqrt)
    x$fpl$dsub                               0x0800b5d8   Section      468  daddsub_clz.o(x$fpl$dsub)
    _dsub1                                   0x0800b5e9   Thumb Code     0  daddsub_clz.o(x$fpl$dsub)
    x$fpl$f2d                                0x0800b7ac   Section       86  f2d.o(x$fpl$f2d)
    x$fpl$fadd                               0x0800b804   Section      196  faddsub_clz.o(x$fpl$fadd)
    _fadd1                                   0x0800b813   Thumb Code     0  faddsub_clz.o(x$fpl$fadd)
    x$fpl$fcmpinf                            0x0800b8c8   Section       24  fcmpi.o(x$fpl$fcmpinf)
    x$fpl$fdiv                               0x0800b8e0   Section      388  fdiv.o(x$fpl$fdiv)
    _fdiv1                                   0x0800b8e1   Thumb Code     0  fdiv.o(x$fpl$fdiv)
    x$fpl$feqf                               0x0800ba64   Section      104  feqf.o(x$fpl$feqf)
    x$fpl$ffixu                              0x0800bacc   Section       62  ffixu.o(x$fpl$ffixu)
    x$fpl$ffltu                              0x0800bb0c   Section       38  fflt_clz.o(x$fpl$ffltu)
    x$fpl$fleqf                              0x0800bb34   Section      104  fleqf.o(x$fpl$fleqf)
    x$fpl$fmul                               0x0800bb9c   Section      258  fmul.o(x$fpl$fmul)
    x$fpl$fnaninf                            0x0800bc9e   Section      140  fnaninf.o(x$fpl$fnaninf)
    x$fpl$fretinf                            0x0800bd2a   Section       10  fretinf.o(x$fpl$fretinf)
    x$fpl$frleqf                             0x0800bd34   Section       98  frleqf.o(x$fpl$frleqf)
    x$fpl$frsb                               0x0800bd96   Section       20  faddsub_clz.o(x$fpl$frsb)
    x$fpl$fsub                               0x0800bdac   Section      234  faddsub_clz.o(x$fpl$fsub)
    _fsub1                                   0x0800bdbb   Thumb Code     0  faddsub_clz.o(x$fpl$fsub)
    x$fpl$llufromd                           0x0800be98   Section      120  dfixull.o(x$fpl$llufromd)
    x$fpl$printf1                            0x0800bf10   Section        4  printf1.o(x$fpl$printf1)
    x$fpl$retnan                             0x0800bf14   Section      100  retnan.o(x$fpl$retnan)
    x$fpl$scalbn                             0x0800bf78   Section       92  scalbn.o(x$fpl$scalbn)
    x$fpl$scanf1                             0x0800bfd4   Section        4  scanf1.o(x$fpl$scanf1)
    x$fpl$scanf2                             0x0800bfd8   Section        8  scanf2.o(x$fpl$scanf2)
    x$fpl$trapveneer                         0x0800bfe0   Section       48  trapv.o(x$fpl$trapveneer)
    .constdata                               0x0800c010   Section     5376  oled.o(.constdata)
    x$fpl$usenofp                            0x0800c010   Section        0  usenofp.o(x$fpl$usenofp)
    .constdata                               0x0800d510   Section     1376  all_lo_init.o(.constdata)
    .constdata                               0x0800da70   Section      920  amp_set.o(.constdata)
    .constdata                               0x0800de08   Section       17  __printf_flags_ss_wp.o(.constdata)
    maptable                                 0x0800de08   Data          17  __printf_flags_ss_wp.o(.constdata)
    .constdata                               0x0800de20   Section      136  pow.o(.constdata)
    bp                                       0x0800de20   Data          16  pow.o(.constdata)
    dp_h                                     0x0800de30   Data          16  pow.o(.constdata)
    dp_l                                     0x0800de40   Data          16  pow.o(.constdata)
    L                                        0x0800de50   Data          48  pow.o(.constdata)
    P                                        0x0800de80   Data          40  pow.o(.constdata)
    .constdata                               0x0800dea8   Section        8  qnan.o(.constdata)
    .constdata                               0x0800deb0   Section      148  bigflt0.o(.constdata)
    tenpwrs_x                                0x0800deb0   Data          60  bigflt0.o(.constdata)
    tenpwrs_i                                0x0800deec   Data          64  bigflt0.o(.constdata)
    c$$dinf                                  0x0800df64   Section        8  fpconst.o(c$$dinf)
    locale$$data                             0x0800df6c   Section       28  lc_numeric_c.o(locale$$data)
    __lcnum_c_name                           0x0800df70   Data           2  lc_numeric_c.o(locale$$data)
    __lcnum_c_start                          0x0800df78   Data           0  lc_numeric_c.o(locale$$data)
    __lcnum_c_point                          0x0800df84   Data           0  lc_numeric_c.o(locale$$data)
    __lcnum_c_thousands                      0x0800df86   Data           0  lc_numeric_c.o(locale$$data)
    __lcnum_c_grouping                       0x0800df87   Data           0  lc_numeric_c.o(locale$$data)
    locale$$data                             0x0800df88   Section      272  lc_ctype_c.o(locale$$data)
    __lcnum_c_end                            0x0800df88   Data           0  lc_numeric_c.o(locale$$data)
    __lcctype_c_name                         0x0800df8c   Data           2  lc_ctype_c.o(locale$$data)
    __lcctype_c_start                        0x0800df94   Data           0  lc_ctype_c.o(locale$$data)
    __lcctype_c_end                          0x0800e098   Data           0  lc_ctype_c.o(locale$$data)
    .data                                    0x20000000   Section       88  main.o(.data)
    .data                                    0x20000058   Section       20  system_stm32f10x.o(.data)
    .data                                    0x2000006c   Section        8  adc.o(.data)
    iLastData                                0x20000070   Data           4  adc.o(.data)
    .data                                    0x20000074   Section        4  timer.o(.data)
    .data                                    0x20000078   Section        2  bsp_ec11.o(.data)
    .data                                    0x2000007a   Section        4  delay.o(.data)
    fac_us                                   0x2000007a   Data           1  delay.o(.data)
    fac_ms                                   0x2000007c   Data           2  delay.o(.data)
    .data                                    0x20000080   Section        6  usart.o(.data)
    .data                                    0x20000086   Section       45  main_menu.o(.data)
    .data                                    0x200000b3   Section      113  cw_menu.o(.data)
    .data                                    0x20000124   Section       22  power_menu.o(.data)
    .data                                    0x2000013a   Section        4  key_s1_process.o(.data)
    .data                                    0x20000140   Section       16  all_lo_init.o(.data)
    .data                                    0x20000150   Section       40  lo_lmx2592_freq_set.o(.data)
    .data                                    0x20000178   Section       24  ad9912_drive.o(.data)
    .data                                    0x20000190   Section       20  adl5513.o(.data)
    .data                                    0x200001a4   Section       36  amp_set.o(.data)
    .data                                    0x200001c8   Section       20  malloc.o(.data)
    .data                                    0x200001dc   Section       20  stm32f10x_rcc.o(.data)
    APBAHBPrescTable                         0x200001dc   Data          16  stm32f10x_rcc.o(.data)
    ADCPrescTable                            0x200001ec   Data           4  stm32f10x_rcc.o(.data)
    .bss                                     0x200001f0   Section       93  matrix_key.o(.bss)
    s_tBtn                                   0x200001f0   Data          80  matrix_key.o(.bss)
    s_tKey                                   0x20000240   Data          13  matrix_key.o(.bss)
    .bss                                     0x2000024d   Section       64  cw_menu.o(.bss)
    .bss                                     0x20000290   Section    38080  malloc.o(.bss)
    .bss                                     0x20009750   Section       96  libspace.o(.bss)
    HEAP                                     0x200097b0   Section     1024  startup_stm32f10x_hd.o(HEAP)
    Heap_Mem                                 0x200097b0   Data        1024  startup_stm32f10x_hd.o(HEAP)
    STACK                                    0x20009bb0   Section     2048  startup_stm32f10x_hd.o(STACK)
    Stack_Mem                                0x20009bb0   Data        2048  startup_stm32f10x_hd.o(STACK)
    __initial_sp                             0x2000a3b0   Data           0  startup_stm32f10x_hd.o(STACK)

    Global Symbols

    Symbol Name                              Value     Ov Type        Size  Object(Section)

    BuildAttributes$$THM_ISAv4$P$D$K$B$S$PE$A:L22UL41UL21$X:L11$S22US41US21$IEEE1$IW$USESV6$~STKCKD$USESV7$~SHL$OTIME$ROPI$IEEEX$EBA8$UX$STANDARDLIB$REQ8$PRES8$EABIv2 0x00000000   Number         0  anon$$obj.o ABSOLUTE
    __ARM_use_no_argv                        0x00000000   Number         0  main.o ABSOLUTE
    _printf_flags                            0x00000000   Number         0  printf_stubs.o ABSOLUTE
    _printf_return_value                     0x00000000   Number         0  printf_stubs.o ABSOLUTE
    _printf_sizespec                         0x00000000   Number         0  printf_stubs.o ABSOLUTE
    _printf_widthprec                        0x00000000   Number         0  printf_stubs.o ABSOLUTE
    __ARM_exceptions_init                     - Undefined Weak Reference
    __alloca_initialize                       - Undefined Weak Reference
    __arm_preinit_                            - Undefined Weak Reference
    __cpp_initialize__aeabi_                  - Undefined Weak Reference
    __cxa_finalize                            - Undefined Weak Reference
    __sigvec_lookup                           - Undefined Weak Reference
    _atexit_init                              - Undefined Weak Reference
    _call_atexit_fns                          - Undefined Weak Reference
    _clock_init                               - Undefined Weak Reference
    _fp_trap_init                             - Undefined Weak Reference
    _fp_trap_shutdown                         - Undefined Weak Reference
    _get_lc_collate                           - Undefined Weak Reference
    _get_lc_monetary                          - Undefined Weak Reference
    _get_lc_time                              - Undefined Weak Reference
    _getenv_init                              - Undefined Weak Reference
    _handle_redirection                       - Undefined Weak Reference
    _init_alloc                               - Undefined Weak Reference
    _init_user_alloc                          - Undefined Weak Reference
    _initio                                   - Undefined Weak Reference
    _mutex_acquire                            - Undefined Weak Reference
    _mutex_release                            - Undefined Weak Reference
    _printf_truncate_signed                   - Undefined Weak Reference
    _printf_truncate_unsigned                 - Undefined Weak Reference
    _rand_init                                - Undefined Weak Reference
    _signal_finish                            - Undefined Weak Reference
    _signal_init                              - Undefined Weak Reference
    _terminate_alloc                          - Undefined Weak Reference
    _terminate_user_alloc                     - Undefined Weak Reference
    _terminateio                              - Undefined Weak Reference
    __Vectors_Size                           0x00000130   Number         0  startup_stm32f10x_hd.o ABSOLUTE
    __Vectors                                0x08000000   Data           4  startup_stm32f10x_hd.o(RESET)
    __Vectors_End                            0x08000130   Data           0  startup_stm32f10x_hd.o(RESET)
    __main                                   0x08000131   Thumb Code     8  __main.o(!!!main)
    __scatterload                            0x08000139   Thumb Code     0  __scatter.o(!!!scatter)
    __scatterload_rt2                        0x08000139   Thumb Code    44  __scatter.o(!!!scatter)
    __scatterload_rt2_thumb_only             0x08000139   Thumb Code     0  __scatter.o(!!!scatter)
    __scatterload_null                       0x08000147   Thumb Code     0  __scatter.o(!!!scatter)
    __decompress                             0x0800016d   Thumb Code    90  __dczerorl2.o(!!dczerorl2)
    __decompress1                            0x0800016d   Thumb Code     0  __dczerorl2.o(!!dczerorl2)
    __scatterload_zeroinit                   0x080001c9   Thumb Code    28  __scatter_zi.o(!!handler_zi)
    _printf_f                                0x080001e5   Thumb Code     0  _printf_f.o(.ARM.Collect$$_printf_percent$$00000003)
    _printf_percent                          0x080001e5   Thumb Code     0  _printf_percent.o(.ARM.Collect$$_printf_percent$$00000000)
    _printf_ll                               0x080001eb   Thumb Code     0  _printf_ll.o(.ARM.Collect$$_printf_percent$$00000007)
    _printf_u                                0x080001f5   Thumb Code     0  _printf_u.o(.ARM.Collect$$_printf_percent$$0000000A)
    _printf_llu                              0x080001fb   Thumb Code     0  _printf_llu.o(.ARM.Collect$$_printf_percent$$0000000F)
    _printf_percent_end                      0x08000201   Thumb Code     0  _printf_percent_end.o(.ARM.Collect$$_printf_percent$$00000017)
    __rt_lib_init                            0x08000205   Thumb Code     0  libinit.o(.ARM.Collect$$libinit$$00000000)
    __rt_lib_init_fp_1                       0x08000207   Thumb Code     0  libinit2.o(.ARM.Collect$$libinit$$00000002)
    __rt_lib_init_heap_1                     0x08000207   Thumb Code     0  libinit2.o(.ARM.Collect$$libinit$$0000000A)
    __rt_lib_init_lc_common                  0x08000207   Thumb Code     0  libinit2.o(.ARM.Collect$$libinit$$0000000F)
    __rt_lib_init_preinit_1                  0x08000207   Thumb Code     0  libinit2.o(.ARM.Collect$$libinit$$00000004)
    __rt_lib_init_rand_1                     0x08000207   Thumb Code     0  libinit2.o(.ARM.Collect$$libinit$$0000000E)
    __rt_lib_init_user_alloc_1               0x08000207   Thumb Code     0  libinit2.o(.ARM.Collect$$libinit$$0000000C)
    __rt_lib_init_lc_collate_1               0x0800020d   Thumb Code     0  libinit2.o(.ARM.Collect$$libinit$$00000011)
    __rt_lib_init_lc_ctype_2                 0x0800020d   Thumb Code     0  libinit2.o(.ARM.Collect$$libinit$$00000012)
    __rt_lib_init_lc_ctype_1                 0x08000219   Thumb Code     0  libinit2.o(.ARM.Collect$$libinit$$00000013)
    __rt_lib_init_lc_monetary_1              0x08000219   Thumb Code     0  libinit2.o(.ARM.Collect$$libinit$$00000015)
    __rt_lib_init_lc_numeric_2               0x08000219   Thumb Code     0  libinit2.o(.ARM.Collect$$libinit$$00000016)
    __rt_lib_init_alloca_1                   0x08000223   Thumb Code     0  libinit2.o(.ARM.Collect$$libinit$$0000002E)
    __rt_lib_init_argv_1                     0x08000223   Thumb Code     0  libinit2.o(.ARM.Collect$$libinit$$0000002C)
    __rt_lib_init_atexit_1                   0x08000223   Thumb Code     0  libinit2.o(.ARM.Collect$$libinit$$0000001B)
    __rt_lib_init_clock_1                    0x08000223   Thumb Code     0  libinit2.o(.ARM.Collect$$libinit$$00000021)
    __rt_lib_init_cpp_1                      0x08000223   Thumb Code     0  libinit2.o(.ARM.Collect$$libinit$$00000032)
    __rt_lib_init_exceptions_1               0x08000223   Thumb Code     0  libinit2.o(.ARM.Collect$$libinit$$00000030)
    __rt_lib_init_fp_trap_1                  0x08000223   Thumb Code     0  libinit2.o(.ARM.Collect$$libinit$$0000001F)
    __rt_lib_init_getenv_1                   0x08000223   Thumb Code     0  libinit2.o(.ARM.Collect$$libinit$$00000023)
    __rt_lib_init_lc_numeric_1               0x08000223   Thumb Code     0  libinit2.o(.ARM.Collect$$libinit$$00000017)
    __rt_lib_init_lc_time_1                  0x08000223   Thumb Code     0  libinit2.o(.ARM.Collect$$libinit$$00000019)
    __rt_lib_init_return                     0x08000223   Thumb Code     0  libinit2.o(.ARM.Collect$$libinit$$00000033)
    __rt_lib_init_signal_1                   0x08000223   Thumb Code     0  libinit2.o(.ARM.Collect$$libinit$$0000001D)
    __rt_lib_init_stdio_1                    0x08000223   Thumb Code     0  libinit2.o(.ARM.Collect$$libinit$$00000025)
    __rt_lib_shutdown                        0x08000225   Thumb Code     0  libshutdown.o(.ARM.Collect$$libshutdown$$00000000)
    __rt_lib_shutdown_cpp_1                  0x08000227   Thumb Code     0  libshutdown2.o(.ARM.Collect$$libshutdown$$00000002)
    __rt_lib_shutdown_fp_trap_1              0x08000227   Thumb Code     0  libshutdown2.o(.ARM.Collect$$libshutdown$$00000007)
    __rt_lib_shutdown_heap_1                 0x08000227   Thumb Code     0  libshutdown2.o(.ARM.Collect$$libshutdown$$0000000F)
    __rt_lib_shutdown_return                 0x08000227   Thumb Code     0  libshutdown2.o(.ARM.Collect$$libshutdown$$00000010)
    __rt_lib_shutdown_signal_1               0x08000227   Thumb Code     0  libshutdown2.o(.ARM.Collect$$libshutdown$$0000000A)
    __rt_lib_shutdown_stdio_1                0x08000227   Thumb Code     0  libshutdown2.o(.ARM.Collect$$libshutdown$$00000004)
    __rt_lib_shutdown_user_alloc_1           0x08000227   Thumb Code     0  libshutdown2.o(.ARM.Collect$$libshutdown$$0000000C)
    __rt_entry                               0x08000229   Thumb Code     0  __rtentry.o(.ARM.Collect$$rtentry$$00000000)
    __rt_entry_presh_1                       0x08000229   Thumb Code     0  __rtentry2.o(.ARM.Collect$$rtentry$$00000002)
    __rt_entry_sh                            0x08000229   Thumb Code     0  __rtentry4.o(.ARM.Collect$$rtentry$$00000004)
    __rt_entry_li                            0x0800022f   Thumb Code     0  __rtentry2.o(.ARM.Collect$$rtentry$$0000000A)
    __rt_entry_postsh_1                      0x0800022f   Thumb Code     0  __rtentry2.o(.ARM.Collect$$rtentry$$00000009)
    __rt_entry_main                          0x08000233   Thumb Code     0  __rtentry2.o(.ARM.Collect$$rtentry$$0000000D)
    __rt_entry_postli_1                      0x08000233   Thumb Code     0  __rtentry2.o(.ARM.Collect$$rtentry$$0000000C)
    __rt_exit                                0x0800023b   Thumb Code     0  rtexit.o(.ARM.Collect$$rtexit$$00000000)
    __rt_exit_ls                             0x0800023d   Thumb Code     0  rtexit2.o(.ARM.Collect$$rtexit$$00000003)
    __rt_exit_prels_1                        0x0800023d   Thumb Code     0  rtexit2.o(.ARM.Collect$$rtexit$$00000002)
    __rt_exit_exit                           0x08000241   Thumb Code     0  rtexit2.o(.ARM.Collect$$rtexit$$00000004)
    main                                     0x08000249   Thumb Code   762  main.o(.text)
    NMI_Handler                              0x08000759   Thumb Code     2  stm32f10x_it.o(.text)
    HardFault_Handler                        0x0800075b   Thumb Code     4  stm32f10x_it.o(.text)
    MemManage_Handler                        0x0800075f   Thumb Code     4  stm32f10x_it.o(.text)
    BusFault_Handler                         0x08000763   Thumb Code     4  stm32f10x_it.o(.text)
    UsageFault_Handler                       0x08000767   Thumb Code     4  stm32f10x_it.o(.text)
    SVC_Handler                              0x0800076b   Thumb Code     2  stm32f10x_it.o(.text)
    DebugMon_Handler                         0x0800076d   Thumb Code     2  stm32f10x_it.o(.text)
    PendSV_Handler                           0x0800076f   Thumb Code     2  stm32f10x_it.o(.text)
    SysTick_Handler                          0x08000771   Thumb Code     2  stm32f10x_it.o(.text)
    SystemInit                               0x08000853   Thumb Code    78  system_stm32f10x.o(.text)
    SystemCoreClockUpdate                    0x080008a1   Thumb Code   142  system_stm32f10x.o(.text)
    LED_Init                                 0x08000955   Thumb Code    92  led.o(.text)
    Adc_Init                                 0x080009b9   Thumb Code   202  adc.o(.text)
    Get_Adc                                  0x08000a83   Thumb Code    46  adc.o(.text)
    Get_Adc_Average                          0x08000ab1   Thumb Code    42  adc.o(.text)
    Get_Adc_Rms                              0x08000adb   Thumb Code   140  adc.o(.text)
    Get_Adc_LPF                              0x08000b67   Thumb Code   114  adc.o(.text)
    ADC1_2_IRQHandler                        0x08000bd9   Thumb Code    38  adc.o(.text)
    TIM3_Int_Init                            0x08000c19   Thumb Code    88  timer.o(.text)
    TIM2_Int_Init                            0x08000c71   Thumb Code    92  timer.o(.text)
    TIM5_Int_Init                            0x08000ccd   Thumb Code    88  timer.o(.text)
    TIM6_Int_Init                            0x08000d25   Thumb Code    88  timer.o(.text)
    TIM8_Init                                0x08000d7d   Thumb Code   116  timer.o(.text)
    TIM3_IRQHandler                          0x08000df1   Thumb Code    78  timer.o(.text)
    TIM2_IRQHandler                          0x08000e3f   Thumb Code    44  timer.o(.text)
    TIM6_IRQHandler                          0x08000e6b   Thumb Code    22  timer.o(.text)
    TIM5_IRQHandler                          0x08000e81   Thumb Code    36  timer.o(.text)
    TIM8_UP_IRQHandler                       0x08000ea5   Thumb Code    24  timer.o(.text)
    bsp_InitEC11Hard                         0x08000ee9   Thumb Code    66  bsp_ec11.o(.text)
    SPI2_Init                                0x08000f31   Thumb Code   124  spi.o(.text)
    SPI2_WriteByte                           0x08000fad   Thumb Code    44  spi.o(.text)
    SPI2_ReadByte                            0x08000fd9   Thumb Code    40  spi.o(.text)
    SPI2_ReadWriteByte                       0x08001001   Thumb Code    78  spi.o(.text)
    SPI2_ReadTwoByte                         0x0800104f   Thumb Code    44  spi.o(.text)
    SPI2_WriteTwoByte                        0x0800107b   Thumb Code    44  spi.o(.text)
    OLED_WR_Byte                             0x080010b1   Thumb Code   108  oled.o(.text)
    Set_Write_RAM                            0x0800111d   Thumb Code    12  oled.o(.text)
    Set_Row_Address                          0x08001129   Thumb Code    32  oled.o(.text)
    Set_Column_Address                       0x08001149   Thumb Code    32  oled.o(.text)
    Draw_Rectangle                           0x08001169   Thumb Code   632  oled.o(.text)
    Fill_RAM                                 0x080013e1   Thumb Code    66  oled.o(.text)
    OLED_Init                                0x08001423   Thumb Code   526  oled.o(.text)
    Set_Read_RAM                             0x08001631   Thumb Code    12  oled.o(.text)
    Set_Remap_Format                         0x0800163d   Thumb Code    30  oled.o(.text)
    Set_Partial_Display                      0x0800165b   Thumb Code    38  oled.o(.text)
    Set_Display_Offset                       0x08001681   Thumb Code    22  oled.o(.text)
    Set_Start_Line                           0x08001697   Thumb Code    22  oled.o(.text)
    Set_Master_Current                       0x080016ad   Thumb Code    22  oled.o(.text)
    Set_Gray_Scale_Table                     0x080016c3   Thumb Code   140  oled.o(.text)
    Set_Linear_Gray_Scale_Table              0x0800174f   Thumb Code    12  oled.o(.text)
    Vertical_Scroll                          0x0800175b   Thumb Code   132  oled.o(.text)
    Fill_Part_RAM                            0x080017df   Thumb Code   182  oled.o(.text)
    Fill_Block                               0x08001895   Thumb Code   106  oled.o(.text)
    Show_Pattern                             0x080018ff   Thumb Code   116  oled.o(.text)
    Con_4_byte                               0x08001973   Thumb Code   174  oled.o(.text)
    Asc5_8                                   0x08001a21   Thumb Code   150  oled.o(.text)
    Asc5_8_advant                            0x08001ab7   Thumb Code   184  oled.o(.text)
    Asc5_8_Single                            0x08001b6f   Thumb Code   120  oled.o(.text)
    Asc12_24_advant                          0x08001be7   Thumb Code   190  oled.o(.text)
    Grayscale                                0x08001ca5   Thumb Code   132  oled.o(.text)
    Dac1_Init                                0x08001d31   Thumb Code    94  dac.o(.text)
    Dac1_Set_Vol                             0x08001d8f   Thumb Code    60  dac.o(.text)
    bsp_InitKey                              0x08001f29   Thumb Code    12  matrix_key.o(.text)
    bsp_PutKey                               0x08001f35   Thumb Code    28  matrix_key.o(.text)
    bsp_GetKey                               0x08001f51   Thumb Code    46  matrix_key.o(.text)
    bsp_GetKey2                              0x08001f7f   Thumb Code    46  matrix_key.o(.text)
    bsp_GetKeyState                          0x08001fad   Thumb Code    12  matrix_key.o(.text)
    bsp_SetKeyParam                          0x08001fb9   Thumb Code    30  matrix_key.o(.text)
    bsp_ClearKey                             0x08001fd7   Thumb Code    10  matrix_key.o(.text)
    bsp_KeyScan                              0x080020a7   Thumb Code    22  matrix_key.o(.text)
    PLL_Freq_Amp_Init                        0x080020e1   Thumb Code    46  bsp.o(.text)
    bsp_init                                 0x0800210f   Thumb Code   194  bsp.o(.text)
    DDS_Freq_Amp_Init                        0x080021d1   Thumb Code    88  bsp.o(.text)
    Key_Scan_Process                         0x080022a1   Thumb Code   228  key_scan.o(.text)
    delay_init                               0x0800243d   Thumb Code    50  delay.o(.text)
    delay_us                                 0x0800246f   Thumb Code    72  delay.o(.text)
    delay_ms                                 0x080024b7   Thumb Code    72  delay.o(.text)
    _sys_exit                                0x08002511   Thumb Code     6  usart.o(.text)
    fputc                                    0x08002517   Thumb Code    24  usart.o(.text)
    uart_init                                0x0800252f   Thumb Code   154  usart.o(.text)
    Reset_Handler                            0x080025d1   Thumb Code     8  startup_stm32f10x_hd.o(.text)
    ADC3_IRQHandler                          0x080025eb   Thumb Code     0  startup_stm32f10x_hd.o(.text)
    CAN1_RX1_IRQHandler                      0x080025eb   Thumb Code     0  startup_stm32f10x_hd.o(.text)
    CAN1_SCE_IRQHandler                      0x080025eb   Thumb Code     0  startup_stm32f10x_hd.o(.text)
    DMA1_Channel1_IRQHandler                 0x080025eb   Thumb Code     0  startup_stm32f10x_hd.o(.text)
    DMA1_Channel2_IRQHandler                 0x080025eb   Thumb Code     0  startup_stm32f10x_hd.o(.text)
    DMA1_Channel3_IRQHandler                 0x080025eb   Thumb Code     0  startup_stm32f10x_hd.o(.text)
    DMA1_Channel4_IRQHandler                 0x080025eb   Thumb Code     0  startup_stm32f10x_hd.o(.text)
    DMA1_Channel5_IRQHandler                 0x080025eb   Thumb Code     0  startup_stm32f10x_hd.o(.text)
    DMA1_Channel6_IRQHandler                 0x080025eb   Thumb Code     0  startup_stm32f10x_hd.o(.text)
    DMA1_Channel7_IRQHandler                 0x080025eb   Thumb Code     0  startup_stm32f10x_hd.o(.text)
    DMA2_Channel1_IRQHandler                 0x080025eb   Thumb Code     0  startup_stm32f10x_hd.o(.text)
    DMA2_Channel2_IRQHandler                 0x080025eb   Thumb Code     0  startup_stm32f10x_hd.o(.text)
    DMA2_Channel3_IRQHandler                 0x080025eb   Thumb Code     0  startup_stm32f10x_hd.o(.text)
    DMA2_Channel4_5_IRQHandler               0x080025eb   Thumb Code     0  startup_stm32f10x_hd.o(.text)
    EXTI0_IRQHandler                         0x080025eb   Thumb Code     0  startup_stm32f10x_hd.o(.text)
    EXTI15_10_IRQHandler                     0x080025eb   Thumb Code     0  startup_stm32f10x_hd.o(.text)
    EXTI1_IRQHandler                         0x080025eb   Thumb Code     0  startup_stm32f10x_hd.o(.text)
    EXTI2_IRQHandler                         0x080025eb   Thumb Code     0  startup_stm32f10x_hd.o(.text)
    EXTI3_IRQHandler                         0x080025eb   Thumb Code     0  startup_stm32f10x_hd.o(.text)
    EXTI4_IRQHandler                         0x080025eb   Thumb Code     0  startup_stm32f10x_hd.o(.text)
    EXTI9_5_IRQHandler                       0x080025eb   Thumb Code     0  startup_stm32f10x_hd.o(.text)
    FLASH_IRQHandler                         0x080025eb   Thumb Code     0  startup_stm32f10x_hd.o(.text)
    FSMC_IRQHandler                          0x080025eb   Thumb Code     0  startup_stm32f10x_hd.o(.text)
    I2C1_ER_IRQHandler                       0x080025eb   Thumb Code     0  startup_stm32f10x_hd.o(.text)
    I2C1_EV_IRQHandler                       0x080025eb   Thumb Code     0  startup_stm32f10x_hd.o(.text)
    I2C2_ER_IRQHandler                       0x080025eb   Thumb Code     0  startup_stm32f10x_hd.o(.text)
    I2C2_EV_IRQHandler                       0x080025eb   Thumb Code     0  startup_stm32f10x_hd.o(.text)
    PVD_IRQHandler                           0x080025eb   Thumb Code     0  startup_stm32f10x_hd.o(.text)
    RCC_IRQHandler                           0x080025eb   Thumb Code     0  startup_stm32f10x_hd.o(.text)
    RTCAlarm_IRQHandler                      0x080025eb   Thumb Code     0  startup_stm32f10x_hd.o(.text)
    RTC_IRQHandler                           0x080025eb   Thumb Code     0  startup_stm32f10x_hd.o(.text)
    SDIO_IRQHandler                          0x080025eb   Thumb Code     0  startup_stm32f10x_hd.o(.text)
    SPI1_IRQHandler                          0x080025eb   Thumb Code     0  startup_stm32f10x_hd.o(.text)
    SPI2_IRQHandler                          0x080025eb   Thumb Code     0  startup_stm32f10x_hd.o(.text)
    SPI3_IRQHandler                          0x080025eb   Thumb Code     0  startup_stm32f10x_hd.o(.text)
    TAMPER_IRQHandler                        0x080025eb   Thumb Code     0  startup_stm32f10x_hd.o(.text)
    TIM1_BRK_IRQHandler                      0x080025eb   Thumb Code     0  startup_stm32f10x_hd.o(.text)
    TIM1_CC_IRQHandler                       0x080025eb   Thumb Code     0  startup_stm32f10x_hd.o(.text)
    TIM1_TRG_COM_IRQHandler                  0x080025eb   Thumb Code     0  startup_stm32f10x_hd.o(.text)
    TIM1_UP_IRQHandler                       0x080025eb   Thumb Code     0  startup_stm32f10x_hd.o(.text)
    TIM4_IRQHandler                          0x080025eb   Thumb Code     0  startup_stm32f10x_hd.o(.text)
    TIM7_IRQHandler                          0x080025eb   Thumb Code     0  startup_stm32f10x_hd.o(.text)
    TIM8_BRK_IRQHandler                      0x080025eb   Thumb Code     0  startup_stm32f10x_hd.o(.text)
    TIM8_CC_IRQHandler                       0x080025eb   Thumb Code     0  startup_stm32f10x_hd.o(.text)
    TIM8_TRG_COM_IRQHandler                  0x080025eb   Thumb Code     0  startup_stm32f10x_hd.o(.text)
    UART4_IRQHandler                         0x080025eb   Thumb Code     0  startup_stm32f10x_hd.o(.text)
    UART5_IRQHandler                         0x080025eb   Thumb Code     0  startup_stm32f10x_hd.o(.text)
    USART1_IRQHandler                        0x080025eb   Thumb Code     0  startup_stm32f10x_hd.o(.text)
    USART2_IRQHandler                        0x080025eb   Thumb Code     0  startup_stm32f10x_hd.o(.text)
    USART3_IRQHandler                        0x080025eb   Thumb Code     0  startup_stm32f10x_hd.o(.text)
    USBWakeUp_IRQHandler                     0x080025eb   Thumb Code     0  startup_stm32f10x_hd.o(.text)
    USB_HP_CAN1_TX_IRQHandler                0x080025eb   Thumb Code     0  startup_stm32f10x_hd.o(.text)
    USB_LP_CAN1_RX0_IRQHandler               0x080025eb   Thumb Code     0  startup_stm32f10x_hd.o(.text)
    WWDG_IRQHandler                          0x080025eb   Thumb Code     0  startup_stm32f10x_hd.o(.text)
    __user_initial_stackheap                 0x080025ed   Thumb Code     0  startup_stm32f10x_hd.o(.text)
    Fun_KEY_Display                          0x08002611   Thumb Code   234  main_menu.o(.text)
    Device_name_Display                      0x080026fb   Thumb Code    14  main_menu.o(.text)
    Main_menu_Win                            0x08002709   Thumb Code    14  main_menu.o(.text)
    CW_Menu_Parameters_Init                  0x08002759   Thumb Code    44  cw_menu.o(.text)
    CW_menu_Amp_Unit_Lable                   0x08002785   Thumb Code    18  cw_menu.o(.text)
    CW_menu_Freq_Unit_Lable                  0x08002797   Thumb Code    84  cw_menu.o(.text)
    CW_menu_Out_Type                         0x080027eb   Thumb Code   100  cw_menu.o(.text)
    CW_menu_Amp_show                         0x0800284f   Thumb Code   170  cw_menu.o(.text)
    CW_menu_Freq_show                        0x080028f9   Thumb Code   184  cw_menu.o(.text)
    CW_menu_Out_Lable                        0x080029b1   Thumb Code    18  cw_menu.o(.text)
    CW_menu_Amp_Lable                        0x080029c3   Thumb Code    18  cw_menu.o(.text)
    CW_menu_Freq_Lable                       0x080029d5   Thumb Code    18  cw_menu.o(.text)
    CW_Menu_Read_Only_Win                    0x080029e7   Thumb Code    58  cw_menu.o(.text)
    CW_Menu_Lable_Select_Win                 0x08002a21   Thumb Code   174  cw_menu.o(.text)
    CW_Menu_Edit_Select_Win                  0x08002acf   Thumb Code    60  cw_menu.o(.text)
    CW_menu_Fix_Display                      0x08002b0b   Thumb Code   216  cw_menu.o(.text)
    CW_menu_Win                              0x08002be3   Thumb Code    96  cw_menu.o(.text)
    Power_menu_dBm_show                      0x08002c4d   Thumb Code   106  power_menu.o(.text)
    Power_menu_Fix_Display                   0x08002cb7   Thumb Code    52  power_menu.o(.text)
    Power_menu_Win                           0x08002ceb   Thumb Code    38  power_menu.o(.text)
    Oled_Main_Task                           0x08002d2d   Thumb Code   226  oled_task.o(.text)
    Key_S1_Down_Process_Other                0x08002e2d   Thumb Code    76  key_s1_process.o(.text)
    Key_S2_Down_Process                      0x08002e91   Thumb Code     4  key_s2_process.o(.text)
    Key_S3_Down_Process                      0x08002e95   Thumb Code   124  key_s3_process.o(.text)
    EC11_Key_Down                            0x08002f4d   Thumb Code   108  ec11_key_process.o(.text)
    EC11_Key_LONG                            0x08002fb9   Thumb Code    50  ec11_key_process.o(.text)
    _EC11_Spin_LableSel_Count                0x08002ffd   Thumb Code    84  ec11_spin_process.o(.text)
    _EC11_Spin_LableSel_Process              0x08003051   Thumb Code    76  ec11_spin_process.o(.text)
    _EC11_Spin_EditSel_Count                 0x0800309d   Thumb Code    84  ec11_spin_process.o(.text)
    _EC11_Spin_EditSel_Process               0x080030f1   Thumb Code   484  ec11_spin_process.o(.text)
    _EC11_Spin_Edit_Count                    0x080032d5   Thumb Code    84  ec11_spin_process.o(.text)
    _EC11_Amp_Step_Up                        0x08003329   Thumb Code   154  ec11_spin_process.o(.text)
    _EC11_Freq_Step_Up                       0x080033c3   Thumb Code   778  ec11_spin_process.o(.text)
    _EC11_Amp_Step_Down                      0x080036cd   Thumb Code   158  ec11_spin_process.o(.text)
    _EC11_Freq_Step_Down                     0x0800376b   Thumb Code   976  ec11_spin_process.o(.text)
    _EC11_Spin_Edit_Process                  0x08003b3b   Thumb Code    76  ec11_spin_process.o(.text)
    Soft_SPI_Init                            0x08003bb5   Thumb Code   124  pll_spi_init.o(.text)
    Soft_SPI_WriteByte                       0x08003c31   Thumb Code   218  pll_spi_init.o(.text)
    Soft_SPI_Read_Reg                        0x08003d0b   Thumb Code   348  pll_spi_init.o(.text)
    LO_LMX2582_Init_Config                   0x08003ed5   Thumb Code    70  all_lo_init.o(.text)
    ALL_PLL_Init                             0x08003f1b   Thumb Code    30  all_lo_init.o(.text)
    PLL_Out_Ctr                              0x08003f39   Thumb Code   178  all_lo_init.o(.text)
    LO_LMX2592_Init_Config                   0x08003feb   Thumb Code   104  all_lo_init.o(.text)
    LMX2592_OUT_VCO                          0x080040a9   Thumb Code   268  lo_lmx2592_freq_set.o(.text)
    LMX2592_OUT_DIV                          0x080041b5   Thumb Code   852  lo_lmx2592_freq_set.o(.text)
    LMX2592_DIV                              0x08004509   Thumb Code   466  lo_lmx2592_freq_set.o(.text)
    Set_LMX2592_Freq_RealTime                0x080046db   Thumb Code   138  lo_lmx2592_freq_set.o(.text)
    AD9912_GPIO_init                         0x08004785   Thumb Code    80  ad9912_drive.o(.text)
    AD9912_Soft_Spi_Init                     0x080047d5   Thumb Code    40  ad9912_drive.o(.text)
    AD9912_Soft_WriteByte                    0x080047fd   Thumb Code   126  ad9912_drive.o(.text)
    AD9912_Soft_ReadByte                     0x0800487b   Thumb Code   232  ad9912_drive.o(.text)
    AD9912_Read_Part_ID                      0x08004963   Thumb Code    44  ad9912_drive.o(.text)
    AD9912_Soft_RESET                        0x0800498f   Thumb Code    34  ad9912_drive.o(.text)
    AD9912_Soft_UPDATE                       0x080049b1   Thumb Code    18  ad9912_drive.o(.text)
    AD9912_Soft_Clear_UPDATE                 0x080049c3   Thumb Code    18  ad9912_drive.o(.text)
    AD9912_IO_update                         0x080049d5   Thumb Code    26  ad9912_drive.o(.text)
    AD9912_Default_Config                    0x080049ef   Thumb Code    72  ad9912_drive.o(.text)
    AD9912_Default_FTW_config                0x08004a37   Thumb Code    74  ad9912_drive.o(.text)
    AD9912_Default_Phase_config              0x08004a81   Thumb Code    74  ad9912_drive.o(.text)
    AD9912_Freq_Convert                      0x08004acb   Thumb Code    86  ad9912_drive.o(.text)
    AD9912_Freq_Convert_Hz                   0x08004b21   Thumb Code    90  ad9912_drive.o(.text)
    AD9912_Phase_Convert                     0x08004b7b   Thumb Code    96  ad9912_drive.o(.text)
    AD9912_SetFreq                           0x08004bdb   Thumb Code    70  ad9912_drive.o(.text)
    AD9912_SetFreq_Hz                        0x08004c21   Thumb Code    70  ad9912_drive.o(.text)
    AD9912_SetPhase                          0x08004c67   Thumb Code    84  ad9912_drive.o(.text)
    AD9912_SetFreq_Test                      0x08004cbb   Thumb Code    72  ad9912_drive.o(.text)
    AD9912_SetPhase_Test                     0x08004d03   Thumb Code    84  ad9912_drive.o(.text)
    AD9912_Power_Ctr                         0x08004d57   Thumb Code   158  ad9912_drive.o(.text)
    AD9912_HSTL_Set                          0x08004df5   Thumb Code   124  ad9912_drive.o(.text)
    AD9912_CMOS_Set                          0x08004e71   Thumb Code   148  ad9912_drive.o(.text)
    PE4302_GPIO_Init                         0x08004f21   Thumb Code    96  pe4302.o(.text)
    PE4302_Set                               0x08004f81   Thumb Code   122  pe4302.o(.text)
    HMC241_GPIO_Init                         0x08005019   Thumb Code    80  hmc241.o(.text)
    HMC241_Set                               0x08005069   Thumb Code   122  hmc241.o(.text)
    ADL5513_dBm_Out                          0x080050fd   Thumb Code   358  adl5513.o(.text)
    DDS_Out_Amp                              0x080052b9   Thumb Code   580  amp_set.o(.text)
    PLL_Out_Amp                              0x080054fd   Thumb Code   400  amp_set.o(.text)
    Amp_ASC_to_Value                         0x0800568d   Thumb Code   310  amp_set.o(.text)
    Amp_Value_to_ASCII                       0x080057c3   Thumb Code    54  amp_set.o(.text)
    Freq_ASC_to_Value                        0x08005805   Thumb Code    94  ch2_freq_set.o(.text)
    Freq_ASC_to_Value_PLL                    0x08005863   Thumb Code   136  ch2_freq_set.o(.text)
    Freq_Value_to_ASCII                      0x080058eb   Thumb Code    98  ch2_freq_set.o(.text)
    Freq_Value_to_ASCII_PLL                  0x0800594d   Thumb Code   112  ch2_freq_set.o(.text)
    CH2_Freq_Set                             0x080059bd   Thumb Code    94  ch2_freq_set.o(.text)
    mymemcpy                                 0x08005a41   Thumb Code    26  malloc.o(.text)
    mymemset                                 0x08005a5b   Thumb Code    20  malloc.o(.text)
    mem_init                                 0x08005a6f   Thumb Code    38  malloc.o(.text)
    mem_perused                              0x08005a95   Thumb Code    42  malloc.o(.text)
    mem_malloc                               0x08005abf   Thumb Code   116  malloc.o(.text)
    mem_free                                 0x08005b33   Thumb Code    66  malloc.o(.text)
    myfree                                   0x08005b75   Thumb Code    24  malloc.o(.text)
    mymalloc                                 0x08005b8d   Thumb Code    28  malloc.o(.text)
    myrealloc                                0x08005ba9   Thumb Code    50  malloc.o(.text)
    GPIO_DeInit                              0x08005be1   Thumb Code   172  stm32f10x_gpio.o(.text)
    GPIO_AFIODeInit                          0x08005c8d   Thumb Code    20  stm32f10x_gpio.o(.text)
    GPIO_Init                                0x08005ca1   Thumb Code   278  stm32f10x_gpio.o(.text)
    GPIO_StructInit                          0x08005db7   Thumb Code    16  stm32f10x_gpio.o(.text)
    GPIO_ReadInputDataBit                    0x08005dc7   Thumb Code    18  stm32f10x_gpio.o(.text)
    GPIO_ReadInputData                       0x08005dd9   Thumb Code     8  stm32f10x_gpio.o(.text)
    GPIO_ReadOutputDataBit                   0x08005de1   Thumb Code    18  stm32f10x_gpio.o(.text)
    GPIO_ReadOutputData                      0x08005df3   Thumb Code     8  stm32f10x_gpio.o(.text)
    GPIO_SetBits                             0x08005dfb   Thumb Code     4  stm32f10x_gpio.o(.text)
    GPIO_ResetBits                           0x08005dff   Thumb Code     4  stm32f10x_gpio.o(.text)
    GPIO_WriteBit                            0x08005e03   Thumb Code    10  stm32f10x_gpio.o(.text)
    GPIO_Write                               0x08005e0d   Thumb Code     4  stm32f10x_gpio.o(.text)
    GPIO_PinLockConfig                       0x08005e11   Thumb Code    18  stm32f10x_gpio.o(.text)
    GPIO_EventOutputConfig                   0x08005e23   Thumb Code    26  stm32f10x_gpio.o(.text)
    GPIO_EventOutputCmd                      0x08005e3d   Thumb Code     6  stm32f10x_gpio.o(.text)
    GPIO_PinRemapConfig                      0x08005e43   Thumb Code   138  stm32f10x_gpio.o(.text)
    GPIO_EXTILineConfig                      0x08005ecd   Thumb Code    66  stm32f10x_gpio.o(.text)
    GPIO_ETH_MediaInterfaceConfig            0x08005f0f   Thumb Code     8  stm32f10x_gpio.o(.text)
    RCC_DeInit                               0x08005f3d   Thumb Code    64  stm32f10x_rcc.o(.text)
    RCC_HSEConfig                            0x08005f7d   Thumb Code    70  stm32f10x_rcc.o(.text)
    RCC_GetFlagStatus                        0x08005fc3   Thumb Code    56  stm32f10x_rcc.o(.text)
    RCC_WaitForHSEStartUp                    0x08005ffb   Thumb Code    56  stm32f10x_rcc.o(.text)
    RCC_AdjustHSICalibrationValue            0x08006033   Thumb Code    20  stm32f10x_rcc.o(.text)
    RCC_HSICmd                               0x08006047   Thumb Code     6  stm32f10x_rcc.o(.text)
    RCC_PLLConfig                            0x0800604d   Thumb Code    24  stm32f10x_rcc.o(.text)
    RCC_PLLCmd                               0x08006065   Thumb Code     6  stm32f10x_rcc.o(.text)
    RCC_SYSCLKConfig                         0x0800606b   Thumb Code    18  stm32f10x_rcc.o(.text)
    RCC_GetSYSCLKSource                      0x0800607d   Thumb Code    10  stm32f10x_rcc.o(.text)
    RCC_HCLKConfig                           0x08006087   Thumb Code    18  stm32f10x_rcc.o(.text)
    RCC_PCLK1Config                          0x08006099   Thumb Code    18  stm32f10x_rcc.o(.text)
    RCC_PCLK2Config                          0x080060ab   Thumb Code    20  stm32f10x_rcc.o(.text)
    RCC_ITConfig                             0x080060bf   Thumb Code    26  stm32f10x_rcc.o(.text)
    RCC_USBCLKConfig                         0x080060d9   Thumb Code     8  stm32f10x_rcc.o(.text)
    RCC_ADCCLKConfig                         0x080060e1   Thumb Code    18  stm32f10x_rcc.o(.text)
    RCC_LSEConfig                            0x080060f3   Thumb Code    50  stm32f10x_rcc.o(.text)
    RCC_LSICmd                               0x08006125   Thumb Code     6  stm32f10x_rcc.o(.text)
    RCC_RTCCLKConfig                         0x0800612b   Thumb Code    12  stm32f10x_rcc.o(.text)
    RCC_RTCCLKCmd                            0x08006137   Thumb Code     8  stm32f10x_rcc.o(.text)
    RCC_GetClocksFreq                        0x0800613f   Thumb Code   192  stm32f10x_rcc.o(.text)
    RCC_AHBPeriphClockCmd                    0x080061ff   Thumb Code    26  stm32f10x_rcc.o(.text)
    RCC_APB2PeriphClockCmd                   0x08006219   Thumb Code    26  stm32f10x_rcc.o(.text)
    RCC_APB1PeriphClockCmd                   0x08006233   Thumb Code    26  stm32f10x_rcc.o(.text)
    RCC_APB2PeriphResetCmd                   0x0800624d   Thumb Code    26  stm32f10x_rcc.o(.text)
    RCC_APB1PeriphResetCmd                   0x08006267   Thumb Code    26  stm32f10x_rcc.o(.text)
    RCC_BackupResetCmd                       0x08006281   Thumb Code     8  stm32f10x_rcc.o(.text)
    RCC_ClockSecuritySystemCmd               0x08006289   Thumb Code     6  stm32f10x_rcc.o(.text)
    RCC_MCOConfig                            0x0800628f   Thumb Code     6  stm32f10x_rcc.o(.text)
    RCC_ClearFlag                            0x08006295   Thumb Code    14  stm32f10x_rcc.o(.text)
    RCC_GetITStatus                          0x080062a3   Thumb Code    20  stm32f10x_rcc.o(.text)
    RCC_ClearITPendingBit                    0x080062b7   Thumb Code     6  stm32f10x_rcc.o(.text)
    USART_DeInit                             0x080062e1   Thumb Code   134  stm32f10x_usart.o(.text)
    USART_Init                               0x08006367   Thumb Code   210  stm32f10x_usart.o(.text)
    USART_StructInit                         0x08006439   Thumb Code    24  stm32f10x_usart.o(.text)
    USART_ClockInit                          0x08006451   Thumb Code    34  stm32f10x_usart.o(.text)
    USART_ClockStructInit                    0x08006473   Thumb Code    12  stm32f10x_usart.o(.text)
    USART_Cmd                                0x0800647f   Thumb Code    24  stm32f10x_usart.o(.text)
    USART_ITConfig                           0x08006497   Thumb Code    74  stm32f10x_usart.o(.text)
    USART_DMACmd                             0x080064e1   Thumb Code    18  stm32f10x_usart.o(.text)
    USART_SetAddress                         0x080064f3   Thumb Code    18  stm32f10x_usart.o(.text)
    USART_WakeUpConfig                       0x08006505   Thumb Code    18  stm32f10x_usart.o(.text)
    USART_ReceiverWakeUpCmd                  0x08006517   Thumb Code    24  stm32f10x_usart.o(.text)
    USART_LINBreakDetectLengthConfig         0x0800652f   Thumb Code    18  stm32f10x_usart.o(.text)
    USART_LINCmd                             0x08006541   Thumb Code    24  stm32f10x_usart.o(.text)
    USART_SendData                           0x08006559   Thumb Code     8  stm32f10x_usart.o(.text)
    USART_ReceiveData                        0x08006561   Thumb Code    10  stm32f10x_usart.o(.text)
    USART_SendBreak                          0x0800656b   Thumb Code    10  stm32f10x_usart.o(.text)
    USART_SetGuardTime                       0x08006575   Thumb Code    16  stm32f10x_usart.o(.text)
    USART_SetPrescaler                       0x08006585   Thumb Code    16  stm32f10x_usart.o(.text)
    USART_SmartCardCmd                       0x08006595   Thumb Code    24  stm32f10x_usart.o(.text)
    USART_SmartCardNACKCmd                   0x080065ad   Thumb Code    24  stm32f10x_usart.o(.text)
    USART_HalfDuplexCmd                      0x080065c5   Thumb Code    24  stm32f10x_usart.o(.text)
    USART_OverSampling8Cmd                   0x080065dd   Thumb Code    22  stm32f10x_usart.o(.text)
    USART_OneBitMethodCmd                    0x080065f3   Thumb Code    24  stm32f10x_usart.o(.text)
    USART_IrDAConfig                         0x0800660b   Thumb Code    18  stm32f10x_usart.o(.text)
    USART_IrDACmd                            0x0800661d   Thumb Code    24  stm32f10x_usart.o(.text)
    USART_GetFlagStatus                      0x08006635   Thumb Code    26  stm32f10x_usart.o(.text)
    USART_ClearFlag                          0x0800664f   Thumb Code    18  stm32f10x_usart.o(.text)
    USART_GetITStatus                        0x08006661   Thumb Code    84  stm32f10x_usart.o(.text)
    USART_ClearITPendingBit                  0x080066b5   Thumb Code    52  stm32f10x_usart.o(.text)
    NVIC_PriorityGroupConfig                 0x080066e9   Thumb Code    10  misc.o(.text)
    NVIC_Init                                0x080066f3   Thumb Code   100  misc.o(.text)
    NVIC_SetVectorTable                      0x08006757   Thumb Code    14  misc.o(.text)
    NVIC_SystemLPConfig                      0x08006765   Thumb Code    34  misc.o(.text)
    SysTick_CLKSourceConfig                  0x08006787   Thumb Code    40  misc.o(.text)
    ADC_DeInit                               0x080067c5   Thumb Code    78  stm32f10x_adc.o(.text)
    ADC_Init                                 0x08006813   Thumb Code    70  stm32f10x_adc.o(.text)
    ADC_StructInit                           0x08006859   Thumb Code    18  stm32f10x_adc.o(.text)
    ADC_Cmd                                  0x0800686b   Thumb Code    22  stm32f10x_adc.o(.text)
    ADC_DMACmd                               0x08006881   Thumb Code    22  stm32f10x_adc.o(.text)
    ADC_ITConfig                             0x08006897   Thumb Code    24  stm32f10x_adc.o(.text)
    ADC_ResetCalibration                     0x080068af   Thumb Code    10  stm32f10x_adc.o(.text)
    ADC_GetResetCalibrationStatus            0x080068b9   Thumb Code    20  stm32f10x_adc.o(.text)
    ADC_StartCalibration                     0x080068cd   Thumb Code    10  stm32f10x_adc.o(.text)
    ADC_GetCalibrationStatus                 0x080068d7   Thumb Code    20  stm32f10x_adc.o(.text)
    ADC_SoftwareStartConvCmd                 0x080068eb   Thumb Code    22  stm32f10x_adc.o(.text)
    ADC_GetSoftwareStartConvStatus           0x08006901   Thumb Code    20  stm32f10x_adc.o(.text)
    ADC_DiscModeChannelCountConfig           0x08006915   Thumb Code    24  stm32f10x_adc.o(.text)
    ADC_DiscModeCmd                          0x0800692d   Thumb Code    22  stm32f10x_adc.o(.text)
    ADC_RegularChannelConfig                 0x08006943   Thumb Code   184  stm32f10x_adc.o(.text)
    ADC_ExternalTrigConvCmd                  0x080069fb   Thumb Code    22  stm32f10x_adc.o(.text)
    ADC_GetConversionValue                   0x08006a11   Thumb Code     8  stm32f10x_adc.o(.text)
    ADC_GetDualModeConversionValue           0x08006a19   Thumb Code     8  stm32f10x_adc.o(.text)
    ADC_AutoInjectedConvCmd                  0x08006a21   Thumb Code    22  stm32f10x_adc.o(.text)
    ADC_InjectedDiscModeCmd                  0x08006a37   Thumb Code    22  stm32f10x_adc.o(.text)
    ADC_ExternalTrigInjectedConvConfig       0x08006a4d   Thumb Code    16  stm32f10x_adc.o(.text)
    ADC_ExternalTrigInjectedConvCmd          0x08006a5d   Thumb Code    22  stm32f10x_adc.o(.text)
    ADC_SoftwareStartInjectedConvCmd         0x08006a73   Thumb Code    22  stm32f10x_adc.o(.text)
    ADC_GetSoftwareStartInjectedConvCmdStatus 0x08006a89   Thumb Code    20  stm32f10x_adc.o(.text)
    ADC_InjectedChannelConfig                0x08006a9d   Thumb Code   130  stm32f10x_adc.o(.text)
    ADC_InjectedSequencerLengthConfig        0x08006b1f   Thumb Code    24  stm32f10x_adc.o(.text)
    ADC_SetInjectedOffset                    0x08006b37   Thumb Code    20  stm32f10x_adc.o(.text)
    ADC_GetInjectedConversionValue           0x08006b4b   Thumb Code    28  stm32f10x_adc.o(.text)
    ADC_AnalogWatchdogCmd                    0x08006b67   Thumb Code    16  stm32f10x_adc.o(.text)
    ADC_AnalogWatchdogThresholdsConfig       0x08006b77   Thumb Code     6  stm32f10x_adc.o(.text)
    ADC_AnalogWatchdogSingleChannelConfig    0x08006b7d   Thumb Code    16  stm32f10x_adc.o(.text)
    ADC_TempSensorVrefintCmd                 0x08006b8d   Thumb Code    64  stm32f10x_adc.o(.text)
    ADC_GetFlagStatus                        0x08006bcd   Thumb Code    18  stm32f10x_adc.o(.text)
    ADC_ClearFlag                            0x08006bdf   Thumb Code     6  stm32f10x_adc.o(.text)
    ADC_GetITStatus                          0x08006be5   Thumb Code    36  stm32f10x_adc.o(.text)
    ADC_ClearITPendingBit                    0x08006c09   Thumb Code    10  stm32f10x_adc.o(.text)
    TIM_DeInit                               0x08006c15   Thumb Code   424  stm32f10x_tim.o(.text)
    TIM_TimeBaseInit                         0x08006dbd   Thumb Code   122  stm32f10x_tim.o(.text)
    TIM_OC1Init                              0x08006e37   Thumb Code   132  stm32f10x_tim.o(.text)
    TIM_OC2Init                              0x08006ebb   Thumb Code   154  stm32f10x_tim.o(.text)
    TIM_OC3Init                              0x08006f55   Thumb Code   150  stm32f10x_tim.o(.text)
    TIM_OC4Init                              0x08006feb   Thumb Code   182  stm32f10x_tim.o(.text)
    TIM_SetIC4Prescaler                      0x080070a1   Thumb Code    26  stm32f10x_tim.o(.text)
    TIM_SetIC3Prescaler                      0x0800713d   Thumb Code    18  stm32f10x_tim.o(.text)
    TIM_SetIC2Prescaler                      0x080071c9   Thumb Code    26  stm32f10x_tim.o(.text)
    TIM_SetIC1Prescaler                      0x08007265   Thumb Code    18  stm32f10x_tim.o(.text)
    TIM_ICInit                               0x080072e3   Thumb Code   150  stm32f10x_tim.o(.text)
    TIM_PWMIConfig                           0x08007379   Thumb Code   124  stm32f10x_tim.o(.text)
    TIM_BDTRConfig                           0x080073f5   Thumb Code    32  stm32f10x_tim.o(.text)
    TIM_TimeBaseStructInit                   0x08007415   Thumb Code    18  stm32f10x_tim.o(.text)
    TIM_OCStructInit                         0x08007427   Thumb Code    20  stm32f10x_tim.o(.text)
    TIM_ICStructInit                         0x0800743b   Thumb Code    18  stm32f10x_tim.o(.text)
    TIM_BDTRStructInit                       0x0800744d   Thumb Code    40  stm32f10x_tim.o(.text)
    TIM_Cmd                                  0x08007475   Thumb Code    24  stm32f10x_tim.o(.text)
    TIM_CtrlPWMOutputs                       0x0800748d   Thumb Code    30  stm32f10x_tim.o(.text)
    TIM_ITConfig                             0x080074ab   Thumb Code    18  stm32f10x_tim.o(.text)
    TIM_GenerateEvent                        0x080074bd   Thumb Code     4  stm32f10x_tim.o(.text)
    TIM_DMAConfig                            0x080074c1   Thumb Code    10  stm32f10x_tim.o(.text)
    TIM_DMACmd                               0x080074cb   Thumb Code    18  stm32f10x_tim.o(.text)
    TIM_InternalClockConfig                  0x080074dd   Thumb Code    12  stm32f10x_tim.o(.text)
    TIM_SelectInputTrigger                   0x080074e9   Thumb Code    18  stm32f10x_tim.o(.text)
    TIM_ITRxExternalClockConfig              0x080074fb   Thumb Code    24  stm32f10x_tim.o(.text)
    TIM_TIxExternalClockConfig               0x08007513   Thumb Code    62  stm32f10x_tim.o(.text)
    TIM_ETRConfig                            0x08007551   Thumb Code    28  stm32f10x_tim.o(.text)
    TIM_ETRClockMode1Config                  0x0800756d   Thumb Code    54  stm32f10x_tim.o(.text)
    TIM_ETRClockMode2Config                  0x080075a3   Thumb Code    32  stm32f10x_tim.o(.text)
    TIM_PrescalerConfig                      0x080075c3   Thumb Code     6  stm32f10x_tim.o(.text)
    TIM_CounterModeConfig                    0x080075c9   Thumb Code    18  stm32f10x_tim.o(.text)
    TIM_EncoderInterfaceConfig               0x080075db   Thumb Code    66  stm32f10x_tim.o(.text)
    TIM_ForcedOC1Config                      0x0800761d   Thumb Code    18  stm32f10x_tim.o(.text)
    TIM_ForcedOC2Config                      0x0800762f   Thumb Code    26  stm32f10x_tim.o(.text)
    TIM_ForcedOC3Config                      0x08007649   Thumb Code    18  stm32f10x_tim.o(.text)
    TIM_ForcedOC4Config                      0x0800765b   Thumb Code    26  stm32f10x_tim.o(.text)
    TIM_ARRPreloadConfig                     0x08007675   Thumb Code    24  stm32f10x_tim.o(.text)
    TIM_SelectCOM                            0x0800768d   Thumb Code    24  stm32f10x_tim.o(.text)
    TIM_SelectCCDMA                          0x080076a5   Thumb Code    24  stm32f10x_tim.o(.text)
    TIM_CCPreloadControl                     0x080076bd   Thumb Code    24  stm32f10x_tim.o(.text)
    TIM_OC1PreloadConfig                     0x080076d5   Thumb Code    18  stm32f10x_tim.o(.text)
    TIM_OC2PreloadConfig                     0x080076e7   Thumb Code    26  stm32f10x_tim.o(.text)
    TIM_OC3PreloadConfig                     0x08007701   Thumb Code    18  stm32f10x_tim.o(.text)
    TIM_OC4PreloadConfig                     0x08007713   Thumb Code    26  stm32f10x_tim.o(.text)
    TIM_OC1FastConfig                        0x0800772d   Thumb Code    18  stm32f10x_tim.o(.text)
    TIM_OC2FastConfig                        0x0800773f   Thumb Code    26  stm32f10x_tim.o(.text)
    TIM_OC3FastConfig                        0x08007759   Thumb Code    18  stm32f10x_tim.o(.text)
    TIM_OC4FastConfig                        0x0800776b   Thumb Code    26  stm32f10x_tim.o(.text)
    TIM_ClearOC1Ref                          0x08007785   Thumb Code    18  stm32f10x_tim.o(.text)
    TIM_ClearOC2Ref                          0x08007797   Thumb Code    24  stm32f10x_tim.o(.text)
    TIM_ClearOC3Ref                          0x080077af   Thumb Code    18  stm32f10x_tim.o(.text)
    TIM_ClearOC4Ref                          0x080077c1   Thumb Code    24  stm32f10x_tim.o(.text)
    TIM_OC1PolarityConfig                    0x080077d9   Thumb Code    18  stm32f10x_tim.o(.text)
    TIM_OC1NPolarityConfig                   0x080077eb   Thumb Code    18  stm32f10x_tim.o(.text)
    TIM_OC2PolarityConfig                    0x080077fd   Thumb Code    26  stm32f10x_tim.o(.text)
    TIM_OC2NPolarityConfig                   0x08007817   Thumb Code    26  stm32f10x_tim.o(.text)
    TIM_OC3PolarityConfig                    0x08007831   Thumb Code    26  stm32f10x_tim.o(.text)
    TIM_OC3NPolarityConfig                   0x0800784b   Thumb Code    26  stm32f10x_tim.o(.text)
    TIM_OC4PolarityConfig                    0x08007865   Thumb Code    26  stm32f10x_tim.o(.text)
    TIM_CCxCmd                               0x0800787f   Thumb Code    30  stm32f10x_tim.o(.text)
    TIM_CCxNCmd                              0x0800789d   Thumb Code    30  stm32f10x_tim.o(.text)
    TIM_SelectOCxM                           0x080078bb   Thumb Code    82  stm32f10x_tim.o(.text)
    TIM_UpdateDisableConfig                  0x0800790d   Thumb Code    24  stm32f10x_tim.o(.text)
    TIM_UpdateRequestConfig                  0x08007925   Thumb Code    24  stm32f10x_tim.o(.text)
    TIM_SelectHallSensor                     0x0800793d   Thumb Code    24  stm32f10x_tim.o(.text)
    TIM_SelectOnePulseMode                   0x08007955   Thumb Code    18  stm32f10x_tim.o(.text)
    TIM_SelectOutputTrigger                  0x08007967   Thumb Code    18  stm32f10x_tim.o(.text)
    TIM_SelectSlaveMode                      0x08007979   Thumb Code    18  stm32f10x_tim.o(.text)
    TIM_SelectMasterSlaveMode                0x0800798b   Thumb Code    18  stm32f10x_tim.o(.text)
    TIM_SetCounter                           0x0800799d   Thumb Code     4  stm32f10x_tim.o(.text)
    TIM_SetAutoreload                        0x080079a1   Thumb Code     4  stm32f10x_tim.o(.text)
    TIM_SetCompare1                          0x080079a5   Thumb Code     4  stm32f10x_tim.o(.text)
    TIM_SetCompare2                          0x080079a9   Thumb Code     4  stm32f10x_tim.o(.text)
    TIM_SetCompare3                          0x080079ad   Thumb Code     4  stm32f10x_tim.o(.text)
    TIM_SetCompare4                          0x080079b1   Thumb Code     6  stm32f10x_tim.o(.text)
    TIM_SetClockDivision                     0x080079b7   Thumb Code    18  stm32f10x_tim.o(.text)
    TIM_GetCapture1                          0x080079c9   Thumb Code     6  stm32f10x_tim.o(.text)
    TIM_GetCapture2                          0x080079cf   Thumb Code     6  stm32f10x_tim.o(.text)
    TIM_GetCapture3                          0x080079d5   Thumb Code     6  stm32f10x_tim.o(.text)
    TIM_GetCapture4                          0x080079db   Thumb Code     8  stm32f10x_tim.o(.text)
    TIM_GetCounter                           0x080079e3   Thumb Code     6  stm32f10x_tim.o(.text)
    TIM_GetPrescaler                         0x080079e9   Thumb Code     6  stm32f10x_tim.o(.text)
    TIM_GetFlagStatus                        0x080079ef   Thumb Code    18  stm32f10x_tim.o(.text)
    TIM_ClearFlag                            0x08007a01   Thumb Code     6  stm32f10x_tim.o(.text)
    TIM_GetITStatus                          0x08007a07   Thumb Code    34  stm32f10x_tim.o(.text)
    TIM_ClearITPendingBit                    0x08007a29   Thumb Code     6  stm32f10x_tim.o(.text)
    SPI_I2S_DeInit                           0x08007a31   Thumb Code    76  stm32f10x_spi.o(.text)
    SPI_Init                                 0x08007a7d   Thumb Code    60  stm32f10x_spi.o(.text)
    I2S_Init                                 0x08007ab9   Thumb Code   226  stm32f10x_spi.o(.text)
    SPI_StructInit                           0x08007b9b   Thumb Code    24  stm32f10x_spi.o(.text)
    I2S_StructInit                           0x08007bb3   Thumb Code    20  stm32f10x_spi.o(.text)
    SPI_Cmd                                  0x08007bc7   Thumb Code    24  stm32f10x_spi.o(.text)
    I2S_Cmd                                  0x08007bdf   Thumb Code    24  stm32f10x_spi.o(.text)
    SPI_I2S_ITConfig                         0x08007bf7   Thumb Code    32  stm32f10x_spi.o(.text)
    SPI_I2S_DMACmd                           0x08007c17   Thumb Code    18  stm32f10x_spi.o(.text)
    SPI_I2S_SendData                         0x08007c29   Thumb Code     4  stm32f10x_spi.o(.text)
    SPI_I2S_ReceiveData                      0x08007c2d   Thumb Code     6  stm32f10x_spi.o(.text)
    SPI_NSSInternalSoftwareConfig            0x08007c33   Thumb Code    30  stm32f10x_spi.o(.text)
    SPI_SSOutputCmd                          0x08007c51   Thumb Code    24  stm32f10x_spi.o(.text)
    SPI_DataSizeConfig                       0x08007c69   Thumb Code    18  stm32f10x_spi.o(.text)
    SPI_TransmitCRC                          0x08007c7b   Thumb Code    10  stm32f10x_spi.o(.text)
    SPI_CalculateCRC                         0x08007c85   Thumb Code    24  stm32f10x_spi.o(.text)
    SPI_GetCRC                               0x08007c9d   Thumb Code    16  stm32f10x_spi.o(.text)
    SPI_GetCRCPolynomial                     0x08007cad   Thumb Code     6  stm32f10x_spi.o(.text)
    SPI_BiDirectionalLineConfig              0x08007cb3   Thumb Code    28  stm32f10x_spi.o(.text)
    SPI_I2S_GetFlagStatus                    0x08007ccf   Thumb Code    18  stm32f10x_spi.o(.text)
    SPI_I2S_ClearFlag                        0x08007ce1   Thumb Code     6  stm32f10x_spi.o(.text)
    SPI_I2S_GetITStatus                      0x08007ce7   Thumb Code    52  stm32f10x_spi.o(.text)
    SPI_I2S_ClearITPendingBit                0x08007d1b   Thumb Code    20  stm32f10x_spi.o(.text)
    DAC_DeInit                               0x08007d3d   Thumb Code    22  stm32f10x_dac.o(.text)
    DAC_Init                                 0x08007d53   Thumb Code    46  stm32f10x_dac.o(.text)
    DAC_StructInit                           0x08007d81   Thumb Code    12  stm32f10x_dac.o(.text)
    DAC_Cmd                                  0x08007d8d   Thumb Code    34  stm32f10x_dac.o(.text)
    DAC_DMACmd                               0x08007daf   Thumb Code    38  stm32f10x_dac.o(.text)
    DAC_SoftwareTriggerCmd                   0x08007dd5   Thumb Code    48  stm32f10x_dac.o(.text)
    DAC_DualSoftwareTriggerCmd               0x08007e05   Thumb Code    38  stm32f10x_dac.o(.text)
    DAC_WaveGenerationCmd                    0x08007e2b   Thumb Code    36  stm32f10x_dac.o(.text)
    DAC_SetChannel1Data                      0x08007e4f   Thumb Code    26  stm32f10x_dac.o(.text)
    DAC_SetChannel2Data                      0x08007e69   Thumb Code    26  stm32f10x_dac.o(.text)
    DAC_SetDualChannelData                   0x08007e83   Thumb Code    32  stm32f10x_dac.o(.text)
    DAC_GetDataOutputValue                   0x08007ea3   Thumb Code    32  stm32f10x_dac.o(.text)
    __use_no_semihosting                     0x08007ec9   Thumb Code     2  use_no_semi_2.o(.text)
    __2printf                                0x08007ecd   Thumb Code    20  noretval__2printf.o(.text)
    __2sprintf                               0x08007ee5   Thumb Code    34  noretval__2sprintf.o(.text)
    _printf_pre_padding                      0x08007f0d   Thumb Code    44  _printf_pad.o(.text)
    _printf_post_padding                     0x08007f39   Thumb Code    34  _printf_pad.o(.text)
    _printf_int_dec                          0x08007f5d   Thumb Code   104  _printf_dec.o(.text)
    _printf_longlong_dec                     0x08007fd5   Thumb Code   108  _printf_longlong_dec.o(.text)
    __printf                                 0x08008051   Thumb Code   388  __printf_flags_ss_wp.o(.text)
    atoi                                     0x080081d9   Thumb Code    26  atoi.o(.text)
    __use_two_region_memory                  0x080081f3   Thumb Code     2  heapauxi.o(.text)
    __rt_heap_escrow$2region                 0x080081f5   Thumb Code     2  heapauxi.o(.text)
    __rt_heap_expand$2region                 0x080081f7   Thumb Code     2  heapauxi.o(.text)
    __I$use$semihosting                      0x080081f9   Thumb Code     0  use_no_semi.o(.text)
    __use_no_semihosting_swi                 0x080081f9   Thumb Code     2  use_no_semi.o(.text)
    __aeabi_errno_addr                       0x080081fd   Thumb Code     8  rt_errno_addr_intlibspace.o(.text)
    __errno$intlibspace                      0x080081fd   Thumb Code     0  rt_errno_addr_intlibspace.o(.text)
    __rt_errno_addr$intlibspace              0x080081fd   Thumb Code     0  rt_errno_addr_intlibspace.o(.text)
    _ll_udiv10                               0x08008205   Thumb Code   138  lludiv10.o(.text)
    __read_errno                             0x0800828f   Thumb Code    10  _rserrno.o(.text)
    __set_errno                              0x08008299   Thumb Code    12  _rserrno.o(.text)
    _printf_int_common                       0x080082a5   Thumb Code   178  _printf_intcommon.o(.text)
    __lib_sel_fp_printf                      0x08008357   Thumb Code     2  _printf_fp_dec.o(.text)
    _printf_fp_dec_real                      0x08008505   Thumb Code   620  _printf_fp_dec.o(.text)
    _printf_char_common                      0x0800877b   Thumb Code    32  _printf_char_common.o(.text)
    _sputc                                   0x080087a1   Thumb Code    10  _sputc.o(.text)
    _printf_char_file                        0x080087ad   Thumb Code    32  _printf_char_file.o(.text)
    __strtod_int                             0x0800880d   Thumb Code    90  strtod.o(.text)
    strtol                                   0x08008875   Thumb Code   112  strtol.o(.text)
    __user_libspace                          0x080088e5   Thumb Code     8  libspace.o(.text)
    __user_perproc_libspace                  0x080088e5   Thumb Code     0  libspace.o(.text)
    __user_perthread_libspace                0x080088e5   Thumb Code     0  libspace.o(.text)
    __rt_ctype_table                         0x080088ed   Thumb Code    16  rt_ctype_table.o(.text)
    __rt_locale                              0x080088fd   Thumb Code     8  rt_locale_intlibspace.o(.text)
    isspace                                  0x08008905   Thumb Code    18  isspace.o(.text)
    _printf_fp_infnan                        0x08008919   Thumb Code   112  _printf_fp_infnan.o(.text)
    _sgetc                                   0x08008999   Thumb Code    30  _sgetc.o(.text)
    _sbackspace                              0x080089b7   Thumb Code    34  _sgetc.o(.text)
    _strtoul                                 0x080089d9   Thumb Code   158  _strtoul.o(.text)
    _btod_etento                             0x08008a79   Thumb Code   216  bigflt0.o(.text)
    ferror                                   0x08008b55   Thumb Code     8  ferror.o(.text)
    __user_setup_stackheap                   0x08008b5d   Thumb Code    74  sys_stackheap_outer.o(.text)
    _chval                                   0x08008ba7   Thumb Code    28  _chval.o(.text)
    _scanf_really_real                       0x08008dc1   Thumb Code   668  scanf_fp.o(.text)
    exit                                     0x08009069   Thumb Code    18  exit.o(.text)
    strcmp                                   0x0800907d   Thumb Code   128  strcmpv7m.o(.text)
    _scanf_really_hex_real                   0x080090fd   Thumb Code   786  scanf_hexfp.o(.text)
    _scanf_really_infnan                     0x0800941d   Thumb Code   292  scanf_infnan.o(.text)
    __aeabi_llsl                             0x08009551   Thumb Code     0  llshl.o(.text)
    _ll_shift_l                              0x08009551   Thumb Code    38  llshl.o(.text)
    _btod_d2e                                0x08009577   Thumb Code    62  btod.o(CL$$btod_d2e)
    _d2e_denorm_low                          0x080095b5   Thumb Code    70  btod.o(CL$$btod_d2e_denorm_low)
    _d2e_norm_op1                            0x080095fb   Thumb Code    96  btod.o(CL$$btod_d2e_norm_op1)
    __btod_div_common                        0x0800965b   Thumb Code   696  btod.o(CL$$btod_div_common)
    _e2d                                     0x08009995   Thumb Code    80  btod.o(CL$$btod_e2d)
    _e2e                                     0x080099e9   Thumb Code   198  btod.o(CL$$btod_e2e)
    _btod_ediv                               0x08009aaf   Thumb Code    40  btod.o(CL$$btod_ediv)
    _btod_edivd                              0x08009ad7   Thumb Code    40  btod.o(CL$$btod_edivd)
    _btod_emul                               0x08009aff   Thumb Code    40  btod.o(CL$$btod_emul)
    _btod_emuld                              0x08009b27   Thumb Code    40  btod.o(CL$$btod_emuld)
    __btod_mult_common                       0x08009b4f   Thumb Code   580  btod.o(CL$$btod_mult_common)
    __ARM_fpclassify                         0x08009d93   Thumb Code    40  fpclassify.o(i.__ARM_fpclassify)
    __kernel_poly                            0x08009dbb   Thumb Code   170  poly.o(i.__kernel_poly)
    __mathlib_dbl_divzero                    0x08009e65   Thumb Code    12  dunder.o(i.__mathlib_dbl_divzero)
    __mathlib_dbl_infnan2                    0x08009e75   Thumb Code     4  dunder.o(i.__mathlib_dbl_infnan2)
    __mathlib_dbl_invalid                    0x08009e79   Thumb Code    12  dunder.o(i.__mathlib_dbl_invalid)
    __mathlib_dbl_overflow                   0x08009e85   Thumb Code    14  dunder.o(i.__mathlib_dbl_overflow)
    __mathlib_dbl_underflow                  0x08009e95   Thumb Code    10  dunder.o(i.__mathlib_dbl_underflow)
    __mathlib_narrow                         0x08009ea5   Thumb Code    16  narrow.o(i.__mathlib_narrow)
    __mathlib_tofloat                        0x08009eb5   Thumb Code   132  narrow.o(i.__mathlib_tofloat)
    __support_ldexp                          0x08009f3d   Thumb Code    22  ldexp.o(i.__support_ldexp)
    _is_digit                                0x08009f53   Thumb Code    14  __printf_wp.o(i._is_digit)
    atof                                     0x08009f61   Thumb Code    42  atof.o(i.atof)
    frexp                                    0x08009f8d   Thumb Code    80  frexp.o(i.frexp)
    ldexp                                    0x08009fe5   Thumb Code   116  ldexp.o(i.ldexp)
    pow                                      0x0800a059   Thumb Code  2512  pow.o(i.pow)
    sqrt                                     0x0800aa31   Thumb Code    76  sqrt.o(i.sqrt)
    _get_lc_numeric                          0x0800aa7d   Thumb Code    44  lc_numeric_c.o(locale$$code)
    _get_lc_ctype                            0x0800aaa9   Thumb Code    44  lc_ctype_c.o(locale$$code)
    __aeabi_d2f                              0x0800aad5   Thumb Code     0  d2f.o(x$fpl$d2f)
    _d2f                                     0x0800aad5   Thumb Code    98  d2f.o(x$fpl$d2f)
    __aeabi_dadd                             0x0800ab39   Thumb Code     0  daddsub_clz.o(x$fpl$dadd)
    _dadd                                    0x0800ab39   Thumb Code   332  daddsub_clz.o(x$fpl$dadd)
    __fpl_dcheck_NaN1                        0x0800ac89   Thumb Code    10  dcheck1.o(x$fpl$dcheck1)
    __fpl_dcmp_Inf                           0x0800ac99   Thumb Code    24  dcmpi.o(x$fpl$dcmpinf)
    __aeabi_ddiv                             0x0800acb1   Thumb Code     0  ddiv.o(x$fpl$ddiv)
    _ddiv                                    0x0800acb1   Thumb Code   552  ddiv.o(x$fpl$ddiv)
    __aeabi_cdcmpeq                          0x0800af61   Thumb Code     0  deqf.o(x$fpl$deqf)
    _dcmpeq                                  0x0800af61   Thumb Code   120  deqf.o(x$fpl$deqf)
    __aeabi_d2uiz                            0x0800afd9   Thumb Code     0  dfixu.o(x$fpl$dfixu)
    _dfixu                                   0x0800afd9   Thumb Code    90  dfixu.o(x$fpl$dfixu)
    __aeabi_i2d                              0x0800b033   Thumb Code     0  dflt_clz.o(x$fpl$dflt)
    _dflt                                    0x0800b033   Thumb Code    46  dflt_clz.o(x$fpl$dflt)
    __aeabi_ui2d                             0x0800b061   Thumb Code     0  dflt_clz.o(x$fpl$dfltu)
    _dfltu                                   0x0800b061   Thumb Code    38  dflt_clz.o(x$fpl$dfltu)
    __aeabi_ul2d                             0x0800b089   Thumb Code     0  dfltll_clz.o(x$fpl$dfltull)
    _ll_uto_d                                0x0800b089   Thumb Code   138  dfltll_clz.o(x$fpl$dfltull)
    __aeabi_cdcmple                          0x0800b115   Thumb Code     0  dleqf.o(x$fpl$dleqf)
    _dcmple                                  0x0800b115   Thumb Code   120  dleqf.o(x$fpl$dleqf)
    __fpl_dcmple_InfNaN                      0x0800b177   Thumb Code     0  dleqf.o(x$fpl$dleqf)
    __aeabi_dmul                             0x0800b18d   Thumb Code     0  dmul.o(x$fpl$dmul)
    _dmul                                    0x0800b18d   Thumb Code   332  dmul.o(x$fpl$dmul)
    __fpl_dnaninf                            0x0800b2e1   Thumb Code   156  dnaninf.o(x$fpl$dnaninf)
    __fpl_dretinf                            0x0800b37d   Thumb Code    12  dretinf.o(x$fpl$dretinf)
    __aeabi_cdrcmple                         0x0800b389   Thumb Code     0  drleqf.o(x$fpl$drleqf)
    _drcmple                                 0x0800b389   Thumb Code   108  drleqf.o(x$fpl$drleqf)
    __aeabi_drsub                            0x0800b3f5   Thumb Code     0  daddsub_clz.o(x$fpl$drsb)
    _drsb                                    0x0800b3f5   Thumb Code    22  daddsub_clz.o(x$fpl$drsb)
    _dsqrt                                   0x0800b40d   Thumb Code   456  dsqrt_noumaal.o(x$fpl$dsqrt)
    __aeabi_dsub                             0x0800b5d9   Thumb Code     0  daddsub_clz.o(x$fpl$dsub)
    _dsub                                    0x0800b5d9   Thumb Code   464  daddsub_clz.o(x$fpl$dsub)
    __aeabi_f2d                              0x0800b7ad   Thumb Code     0  f2d.o(x$fpl$f2d)
    _f2d                                     0x0800b7ad   Thumb Code    86  f2d.o(x$fpl$f2d)
    __aeabi_fadd                             0x0800b805   Thumb Code     0  faddsub_clz.o(x$fpl$fadd)
    _fadd                                    0x0800b805   Thumb Code   196  faddsub_clz.o(x$fpl$fadd)
    __fpl_fcmp_Inf                           0x0800b8c9   Thumb Code    24  fcmpi.o(x$fpl$fcmpinf)
    __aeabi_fdiv                             0x0800b8e1   Thumb Code     0  fdiv.o(x$fpl$fdiv)
    _fdiv                                    0x0800b8e1   Thumb Code   384  fdiv.o(x$fpl$fdiv)
    __aeabi_cfcmpeq                          0x0800ba65   Thumb Code     0  feqf.o(x$fpl$feqf)
    _fcmpeq                                  0x0800ba65   Thumb Code   104  feqf.o(x$fpl$feqf)
    __aeabi_f2uiz                            0x0800bacd   Thumb Code     0  ffixu.o(x$fpl$ffixu)
    _ffixu                                   0x0800bacd   Thumb Code    62  ffixu.o(x$fpl$ffixu)
    __aeabi_ui2f                             0x0800bb0d   Thumb Code     0  fflt_clz.o(x$fpl$ffltu)
    _ffltu                                   0x0800bb0d   Thumb Code    38  fflt_clz.o(x$fpl$ffltu)
    __aeabi_cfcmple                          0x0800bb35   Thumb Code     0  fleqf.o(x$fpl$fleqf)
    _fcmple                                  0x0800bb35   Thumb Code   104  fleqf.o(x$fpl$fleqf)
    __fpl_fcmple_InfNaN                      0x0800bb87   Thumb Code     0  fleqf.o(x$fpl$fleqf)
    __aeabi_fmul                             0x0800bb9d   Thumb Code     0  fmul.o(x$fpl$fmul)
    _fmul                                    0x0800bb9d   Thumb Code   258  fmul.o(x$fpl$fmul)
    __fpl_fnaninf                            0x0800bc9f   Thumb Code   140  fnaninf.o(x$fpl$fnaninf)
    __fpl_fretinf                            0x0800bd2b   Thumb Code    10  fretinf.o(x$fpl$fretinf)
    __aeabi_cfrcmple                         0x0800bd35   Thumb Code     0  frleqf.o(x$fpl$frleqf)
    _frcmple                                 0x0800bd35   Thumb Code    98  frleqf.o(x$fpl$frleqf)
    __aeabi_frsub                            0x0800bd97   Thumb Code     0  faddsub_clz.o(x$fpl$frsb)
    _frsb                                    0x0800bd97   Thumb Code    20  faddsub_clz.o(x$fpl$frsb)
    __aeabi_fsub                             0x0800bdad   Thumb Code     0  faddsub_clz.o(x$fpl$fsub)
    _fsub                                    0x0800bdad   Thumb Code   234  faddsub_clz.o(x$fpl$fsub)
    __aeabi_d2ulz                            0x0800be99   Thumb Code     0  dfixull.o(x$fpl$llufromd)
    _ll_ufrom_d                              0x0800be99   Thumb Code   120  dfixull.o(x$fpl$llufromd)
    _printf_fp_dec                           0x0800bf11   Thumb Code     4  printf1.o(x$fpl$printf1)
    __fpl_return_NaN                         0x0800bf15   Thumb Code   100  retnan.o(x$fpl$retnan)
    __ARM_scalbn                             0x0800bf79   Thumb Code    92  scalbn.o(x$fpl$scalbn)
    _scanf_real                              0x0800bfd5   Thumb Code     4  scanf1.o(x$fpl$scanf1)
    _scanf_hex_real                          0x0800bfd9   Thumb Code     4  scanf2.o(x$fpl$scanf2)
    _scanf_infnan                            0x0800bfdd   Thumb Code     4  scanf2.o(x$fpl$scanf2)
    __fpl_cmpreturn                          0x0800bfe1   Thumb Code    48  trapv.o(x$fpl$trapveneer)
    ASC5X8                                   0x0800c010   Data         768  oled.o(.constdata)
    __I$use$fp                               0x0800c010   Number         0  usenofp.o(x$fpl$usenofp)
    ASC12X24                                 0x0800c310   Data        4608  oled.o(.constdata)
    LO_LMX2582_Default_Reg1                  0x0800d510   Data         172  all_lo_init.o(.constdata)
    LO_LMX2582_Default_Reg2                  0x0800d5bc   Data         172  all_lo_init.o(.constdata)
    LO_LMX2582_Default_Reg3                  0x0800d668   Data         172  all_lo_init.o(.constdata)
    LO_LMX2582_Default_Reg4                  0x0800d714   Data         172  all_lo_init.o(.constdata)
    LO_LMX2582_Default_Reg5                  0x0800d7c0   Data         172  all_lo_init.o(.constdata)
    LO_LMX2592_Default_Reg1                  0x0800d86c   Data         172  all_lo_init.o(.constdata)
    LO_LMX2592_Default_Reg2                  0x0800d918   Data         172  all_lo_init.o(.constdata)
    LO_LMX2592_Default_Reg3                  0x0800d9c4   Data         172  all_lo_init.o(.constdata)
    Cal_Bypass_ATT0                          0x0800da70   Data         920  amp_set.o(.constdata)
    __mathlib_zero                           0x0800dea8   Data           8  qnan.o(.constdata)
    Region$$Table$$Base                      0x0800df44   Number         0  anon$$obj.o(Region$$Table)
    Region$$Table$$Limit                     0x0800df64   Number         0  anon$$obj.o(Region$$Table)
    __aeabi_HUGE_VAL                         0x0800df64   Data           0  fpconst.o(c$$dinf)
    __aeabi_HUGE_VALL                        0x0800df64   Data           0  fpconst.o(c$$dinf)
    __aeabi_INFINITY                         0x0800df64   Data           0  fpconst.o(c$$dinf)
    __dInf                                   0x0800df64   Data           0  fpconst.o(c$$dinf)
    __huge_val                               0x0800df64   Data           0  fpconst.o(c$$dinf)
    __ctype                                  0x0800df95   Data           0  lc_ctype_c.o(locale$$data)
    NVIC_InitStructure                       0x20000000   Data           4  main.o(.data)
    BEEP_SW                                  0x20000004   Data           1  main.o(.data)
    DDS_Freq_Hz                              0x20000008   Data           4  main.o(.data)
    DDS_Freq_Hz_Buf                          0x2000000c   Data           4  main.o(.data)
    PLL_Freq_Hz                              0x20000010   Data           8  main.o(.data)
    PLL_Freq_Hz_Buf                          0x20000018   Data           8  main.o(.data)
    DDS_Amp_dBm                              0x20000020   Data           4  main.o(.data)
    DDS_Amp_dBm_Buf                          0x20000024   Data           4  main.o(.data)
    PLL_Amp_dBm                              0x20000028   Data           4  main.o(.data)
    PLL_Amp_dBm_Buf                          0x2000002c   Data           4  main.o(.data)
    Sweep_Start                              0x20000030   Data           4  main.o(.data)
    Sweep_Step                               0x20000034   Data           4  main.o(.data)
    temp_u8                                  0x20000038   Data           1  main.o(.data)
    t                                        0x20000039   Data           1  main.o(.data)
    i                                        0x2000003a   Data           1  main.o(.data)
    temp_u16                                 0x2000003c   Data           2  main.o(.data)
    EC11_Direct                              0x2000003e   Data           1  main.o(.data)
    EC11_Ent_Count                           0x2000003f   Data           1  main.o(.data)
    Enc0Pos                                  0x20000040   Data           2  main.o(.data)
    Enc_PinDATLast                           0x20000042   Data           2  main.o(.data)
    EC11_Count_LableSel                      0x20000044   Data           2  main.o(.data)
    EC11_Count_LableSel_Reg                  0x20000046   Data           2  main.o(.data)
    EC11_Count_EditSel                       0x20000048   Data           2  main.o(.data)
    EC11_Count_EditSel_Reg                   0x2000004a   Data           2  main.o(.data)
    EC11_Count_EditNum                       0x2000004c   Data           2  main.o(.data)
    EC11_Count_EditNum_Reg                   0x2000004e   Data           2  main.o(.data)
    uKeyCode                                 0x20000050   Data           1  main.o(.data)
    Key_ON                                   0x20000051   Data           1  main.o(.data)
    Menu_Type                                0x20000052   Data           1  main.o(.data)
    Menu_Type_buf                            0x20000053   Data           1  main.o(.data)
    TIM3_tick                                0x20000054   Data           4  main.o(.data)
    SystemCoreClock                          0x20000058   Data           4  system_stm32f10x.o(.data)
    AHBPrescTable                            0x2000005c   Data          16  system_stm32f10x.o(.data)
    adcx1                                    0x2000006c   Data           2  adc.o(.data)
    oled_refresh                             0x20000074   Data           1  timer.o(.data)
    oled_key_refresh                         0x20000075   Data           1  timer.o(.data)
    beep_count                               0x20000076   Data           1  timer.o(.data)
    tim_1s_count                             0x20000077   Data           1  timer.o(.data)
    Out_Process                              0x20000078   Data           1  bsp_ec11.o(.data)
    EC11_Lock                                0x20000079   Data           1  bsp_ec11.o(.data)
    __stdout                                 0x20000080   Data           4  usart.o(.data)
    USART_RX_STA                             0x20000084   Data           2  usart.o(.data)
    Device_Info                              0x20000086   Data          23  main_menu.o(.data)
    Main_menu_S1_Name                        0x2000009d   Data           3  main_menu.o(.data)
    Main_menu_S2_Name                        0x200000a0   Data           6  main_menu.o(.data)
    Main_menu_S3_Name                        0x200000a6   Data           6  main_menu.o(.data)
    Main_menu_S4_Name                        0x200000ac   Data           7  main_menu.o(.data)
    CW_menu_S1_Name0                         0x200000b3   Data           5  cw_menu.o(.data)
    CW_menu_S1_Name1                         0x200000b8   Data           5  cw_menu.o(.data)
    CW_menu_S1_Name2                         0x200000bd   Data           5  cw_menu.o(.data)
    CW_menu_S2_Name                          0x200000c2   Data           6  cw_menu.o(.data)
    CW_menu_S3_Name                          0x200000c8   Data           8  cw_menu.o(.data)
    CW_menu_S4_Name                          0x200000d0   Data           5  cw_menu.o(.data)
    Freq_Label                               0x200000d5   Data           5  cw_menu.o(.data)
    Amp_Label                                0x200000da   Data           5  cw_menu.o(.data)
    Out_Label                                0x200000df   Data           5  cw_menu.o(.data)
    GHz_Label                                0x200000e4   Data           4  cw_menu.o(.data)
    MHz_Label                                0x200000e8   Data           4  cw_menu.o(.data)
    KHz_Label                                0x200000ec   Data           4  cw_menu.o(.data)
    Hz_Label                                 0x200000f0   Data           4  cw_menu.o(.data)
    dBm_Label                                0x200000f4   Data           4  cw_menu.o(.data)
    Vpp_Label                                0x200000f8   Data           4  cw_menu.o(.data)
    Rms_Label                                0x200000fc   Data           4  cw_menu.o(.data)
    DDS_Label                                0x20000100   Data           4  cw_menu.o(.data)
    RFLabel                                  0x20000104   Data           4  cw_menu.o(.data)
    CW_Amp_Show_Buf                          0x20000108   Data           8  cw_menu.o(.data)
    CW_Amp_Show_Last_buf                     0x20000110   Data           8  cw_menu.o(.data)
    CW_Display_flag                          0x20000118   Data           1  cw_menu.o(.data)
    CW_Edit_Sel                              0x20000119   Data           1  cw_menu.o(.data)
    CW_Freq_Show_Point                       0x2000011a   Data           1  cw_menu.o(.data)
    CW_Freq_Uint                             0x2000011b   Data           1  cw_menu.o(.data)
    CW_Freq_Uint_Reg                         0x2000011c   Data           1  cw_menu.o(.data)
    CW_Amp_Uint                              0x2000011d   Data           1  cw_menu.o(.data)
    CW_Amp_Uint_Reg                          0x2000011e   Data           1  cw_menu.o(.data)
    CW_Amp_Sign                              0x2000011f   Data           1  cw_menu.o(.data)
    CW_Out_Type                              0x20000120   Data           1  cw_menu.o(.data)
    CW_Freq_Show_Position                    0x20000121   Data           1  cw_menu.o(.data)
    CW_Amp_Show_Position                     0x20000122   Data           1  cw_menu.o(.data)
    CW_Freq_Show_Count                       0x20000123   Data           1  cw_menu.o(.data)
    POWER_menu_S1_Name                       0x20000124   Data           5  power_menu.o(.data)
    POWER_menu_S2_Name                       0x20000129   Data           4  power_menu.o(.data)
    POWER_menu_S3_Name                       0x2000012d   Data           7  power_menu.o(.data)
    POWER_menu_S4_Name                       0x20000134   Data           5  power_menu.o(.data)
    Power_Display_flag                       0x20000139   Data           1  power_menu.o(.data)
    Out_State                                0x2000013a   Data           1  key_s1_process.o(.data)
    Out_State_Buf                            0x2000013b   Data           1  key_s1_process.o(.data)
    Key_S1_Down_Count                        0x2000013c   Data           2  key_s1_process.o(.data)
    LMX2592_R0_Value                         0x20000140   Data           4  all_lo_init.o(.data)
    LMX2592_R0_Value_Reg                     0x20000144   Data           4  all_lo_init.o(.data)
    LMX2592_R23_Value                        0x20000148   Data           4  all_lo_init.o(.data)
    LMX2592_R23_Value_Reg                    0x2000014c   Data           4  all_lo_init.o(.data)
    LMX2592_VCO_SEL                          0x20000150   Data           1  lo_lmx2592_freq_set.o(.data)
    LMX2592_VCO_SEL_Buf                      0x20000151   Data           1  lo_lmx2592_freq_set.o(.data)
    LMX2592_FCAL_HPFD_ADJ                    0x20000152   Data           1  lo_lmx2592_freq_set.o(.data)
    LMX2592_FCAL_HPFD_ADJ_Buf                0x20000153   Data           1  lo_lmx2592_freq_set.o(.data)
    LMX2592_FCAL_VCO_SEL_STRT                0x20000154   Data           1  lo_lmx2592_freq_set.o(.data)
    LMX2592_Fpfd                             0x20000158   Data           8  lo_lmx2592_freq_set.o(.data)
    LMX2592_OSC                              0x20000160   Data           8  lo_lmx2592_freq_set.o(.data)
    LMX2592_VCO                              0x20000168   Data           8  lo_lmx2592_freq_set.o(.data)
    LMX2592_N                                0x20000170   Data           4  lo_lmx2592_freq_set.o(.data)
    LMX2592_SEG1                             0x20000174   Data           1  lo_lmx2592_freq_set.o(.data)
    LMX2592_SEG2                             0x20000175   Data           1  lo_lmx2592_freq_set.o(.data)
    LMX2592_SEG3                             0x20000176   Data           1  lo_lmx2592_freq_set.o(.data)
    LMX2592_Total_Div                        0x20000177   Data           1  lo_lmx2592_freq_set.o(.data)
    AD9912_fre                               0x20000178   Data           4  ad9912_drive.o(.data)
    AD9912_Pha                               0x2000017c   Data           4  ad9912_drive.o(.data)
    AD9912_Freq_step                         0x20000180   Data           4  ad9912_drive.o(.data)
    AD9912_Freq                              0x20000184   Data           6  ad9912_drive.o(.data)
    AD9912_Phase                             0x2000018a   Data           2  ad9912_drive.o(.data)
    AD9912_Part_ID                           0x2000018c   Data           2  ad9912_drive.o(.data)
    AD9912_Power_Flag                        0x2000018e   Data           1  ad9912_drive.o(.data)
    AD9912_Power_Flag_Reg                    0x2000018f   Data           1  ad9912_drive.o(.data)
    ADL5513_dBm                              0x20000190   Data           4  adl5513.o(.data)
    ADL5513_dBm_buf                          0x20000194   Data           4  adl5513.o(.data)
    ADL5513_Voltage                          0x20000198   Data           4  adl5513.o(.data)
    ADC_Ref                                  0x2000019c   Data           4  adl5513.o(.data)
    Ext_ATT                                  0x200001a0   Data           4  adl5513.o(.data)
    DATT_Set                                 0x200001a4   Data           4  amp_set.o(.data)
    Amp_10MHz_offset                         0x200001a8   Data           4  amp_set.o(.data)
    Amp_100MHz_offset                        0x200001ac   Data           4  amp_set.o(.data)
    Amp_500MHz_offset                        0x200001b0   Data           4  amp_set.o(.data)
    Amp_1500MHz_offset                       0x200001b4   Data           4  amp_set.o(.data)
    Amp_2000MHz_offset                       0x200001b8   Data           4  amp_set.o(.data)
    Amp_2500MHz_offset                       0x200001bc   Data           4  amp_set.o(.data)
    Amp_2800MHz_offset                       0x200001c0   Data           4  amp_set.o(.data)
    ATT_60dB_offset                          0x200001c4   Data           4  amp_set.o(.data)
    mallco_dev                               0x200001c8   Data          20  malloc.o(.data)
    CW_Freq_Show_Buf                         0x2000024d   Data          16  cw_menu.o(.bss)
    CW_Freq_Show_Position_Anti               0x2000025d   Data          16  cw_menu.o(.bss)
    CW_DDS_Freq_Show_Buf                     0x2000026d   Data          16  cw_menu.o(.bss)
    CW_PLL_Freq_Show_Buf                     0x2000027d   Data          16  cw_menu.o(.bss)
    membase                                  0x20000290   Data       35840  malloc.o(.bss)
    memmapbase                               0x20008e90   Data        2240  malloc.o(.bss)
    __libspace_start                         0x20009750   Data          96  libspace.o(.bss)
    __temporary_stack_top$libspace           0x200097b0   Data           0  libspace.o(.bss)



==============================================================================

Memory Map of the image

  Image Entry point : 0x08000131

  Load Region LR_IROM1 (Base: 0x08000000, Size: 0x0000e288, Max: 0x00040000, ABSOLUTE, COMPRESSED[0x0000e17c])

    Execution Region ER_IROM1 (Base: 0x08000000, Size: 0x0000e098, Max: 0x00040000, ABSOLUTE)

    Base Addr    Size         Type   Attr      Idx    E Section Name        Object

    0x08000000   0x00000130   Data   RO          492    RESET               startup_stm32f10x_hd.o
    0x08000130   0x00000008   Code   RO         1029  * !!!main             c_w.l(__main.o)
    0x08000138   0x00000034   Code   RO         1444    !!!scatter          c_w.l(__scatter.o)
    0x0800016c   0x0000005a   Code   RO         1442    !!dczerorl2         c_w.l(__dczerorl2.o)
    0x080001c6   0x00000002   PAD
    0x080001c8   0x0000001c   Code   RO         1446    !!handler_zi        c_w.l(__scatter_zi.o)
    0x080001e4   0x00000000   Code   RO         1023    .ARM.Collect$$_printf_percent$$00000000  c_w.l(_printf_percent.o)
    0x080001e4   0x00000006   Code   RO         1022    .ARM.Collect$$_printf_percent$$00000003  c_w.l(_printf_f.o)
    0x080001ea   0x0000000a   Code   RO         1144    .ARM.Collect$$_printf_percent$$00000007  c_w.l(_printf_ll.o)
    0x080001f4   0x00000006   Code   RO         1021    .ARM.Collect$$_printf_percent$$0000000A  c_w.l(_printf_u.o)
    0x080001fa   0x00000006   Code   RO         1024    .ARM.Collect$$_printf_percent$$0000000F  c_w.l(_printf_llu.o)
    0x08000200   0x00000004   Code   RO         1143    .ARM.Collect$$_printf_percent$$00000017  c_w.l(_printf_percent_end.o)
    0x08000204   0x00000002   Code   RO         1276    .ARM.Collect$$libinit$$00000000  c_w.l(libinit.o)
    0x08000206   0x00000000   Code   RO         1278    .ARM.Collect$$libinit$$00000002  c_w.l(libinit2.o)
    0x08000206   0x00000000   Code   RO         1280    .ARM.Collect$$libinit$$00000004  c_w.l(libinit2.o)
    0x08000206   0x00000000   Code   RO         1283    .ARM.Collect$$libinit$$0000000A  c_w.l(libinit2.o)
    0x08000206   0x00000000   Code   RO         1285    .ARM.Collect$$libinit$$0000000C  c_w.l(libinit2.o)
    0x08000206   0x00000000   Code   RO         1287    .ARM.Collect$$libinit$$0000000E  c_w.l(libinit2.o)
    0x08000206   0x00000006   Code   RO         1288    .ARM.Collect$$libinit$$0000000F  c_w.l(libinit2.o)
    0x0800020c   0x00000000   Code   RO         1290    .ARM.Collect$$libinit$$00000011  c_w.l(libinit2.o)
    0x0800020c   0x0000000c   Code   RO         1291    .ARM.Collect$$libinit$$00000012  c_w.l(libinit2.o)
    0x08000218   0x00000000   Code   RO         1292    .ARM.Collect$$libinit$$00000013  c_w.l(libinit2.o)
    0x08000218   0x00000000   Code   RO         1294    .ARM.Collect$$libinit$$00000015  c_w.l(libinit2.o)
    0x08000218   0x0000000a   Code   RO         1295    .ARM.Collect$$libinit$$00000016  c_w.l(libinit2.o)
    0x08000222   0x00000000   Code   RO         1296    .ARM.Collect$$libinit$$00000017  c_w.l(libinit2.o)
    0x08000222   0x00000000   Code   RO         1298    .ARM.Collect$$libinit$$00000019  c_w.l(libinit2.o)
    0x08000222   0x00000000   Code   RO         1300    .ARM.Collect$$libinit$$0000001B  c_w.l(libinit2.o)
    0x08000222   0x00000000   Code   RO         1302    .ARM.Collect$$libinit$$0000001D  c_w.l(libinit2.o)
    0x08000222   0x00000000   Code   RO         1304    .ARM.Collect$$libinit$$0000001F  c_w.l(libinit2.o)
    0x08000222   0x00000000   Code   RO         1306    .ARM.Collect$$libinit$$00000021  c_w.l(libinit2.o)
    0x08000222   0x00000000   Code   RO         1308    .ARM.Collect$$libinit$$00000023  c_w.l(libinit2.o)
    0x08000222   0x00000000   Code   RO         1310    .ARM.Collect$$libinit$$00000025  c_w.l(libinit2.o)
    0x08000222   0x00000000   Code   RO         1314    .ARM.Collect$$libinit$$0000002C  c_w.l(libinit2.o)
    0x08000222   0x00000000   Code   RO         1316    .ARM.Collect$$libinit$$0000002E  c_w.l(libinit2.o)
    0x08000222   0x00000000   Code   RO         1318    .ARM.Collect$$libinit$$00000030  c_w.l(libinit2.o)
    0x08000222   0x00000000   Code   RO         1320    .ARM.Collect$$libinit$$00000032  c_w.l(libinit2.o)
    0x08000222   0x00000002   Code   RO         1321    .ARM.Collect$$libinit$$00000033  c_w.l(libinit2.o)
    0x08000224   0x00000002   Code   RO         1380    .ARM.Collect$$libshutdown$$00000000  c_w.l(libshutdown.o)
    0x08000226   0x00000000   Code   RO         1401    .ARM.Collect$$libshutdown$$00000002  c_w.l(libshutdown2.o)
    0x08000226   0x00000000   Code   RO         1403    .ARM.Collect$$libshutdown$$00000004  c_w.l(libshutdown2.o)
    0x08000226   0x00000000   Code   RO         1406    .ARM.Collect$$libshutdown$$00000007  c_w.l(libshutdown2.o)
    0x08000226   0x00000000   Code   RO         1409    .ARM.Collect$$libshutdown$$0000000A  c_w.l(libshutdown2.o)
    0x08000226   0x00000000   Code   RO         1411    .ARM.Collect$$libshutdown$$0000000C  c_w.l(libshutdown2.o)
    0x08000226   0x00000000   Code   RO         1414    .ARM.Collect$$libshutdown$$0000000F  c_w.l(libshutdown2.o)
    0x08000226   0x00000002   Code   RO         1415    .ARM.Collect$$libshutdown$$00000010  c_w.l(libshutdown2.o)
    0x08000228   0x00000000   Code   RO         1123    .ARM.Collect$$rtentry$$00000000  c_w.l(__rtentry.o)
    0x08000228   0x00000000   Code   RO         1189    .ARM.Collect$$rtentry$$00000002  c_w.l(__rtentry2.o)
    0x08000228   0x00000006   Code   RO         1201    .ARM.Collect$$rtentry$$00000004  c_w.l(__rtentry4.o)
    0x0800022e   0x00000000   Code   RO         1191    .ARM.Collect$$rtentry$$00000009  c_w.l(__rtentry2.o)
    0x0800022e   0x00000004   Code   RO         1192    .ARM.Collect$$rtentry$$0000000A  c_w.l(__rtentry2.o)
    0x08000232   0x00000000   Code   RO         1194    .ARM.Collect$$rtentry$$0000000C  c_w.l(__rtentry2.o)
    0x08000232   0x00000008   Code   RO         1195    .ARM.Collect$$rtentry$$0000000D  c_w.l(__rtentry2.o)
    0x0800023a   0x00000002   Code   RO         1324    .ARM.Collect$$rtexit$$00000000  c_w.l(rtexit.o)
    0x0800023c   0x00000000   Code   RO         1348    .ARM.Collect$$rtexit$$00000002  c_w.l(rtexit2.o)
    0x0800023c   0x00000004   Code   RO         1349    .ARM.Collect$$rtexit$$00000003  c_w.l(rtexit2.o)
    0x08000240   0x00000006   Code   RO         1350    .ARM.Collect$$rtexit$$00000004  c_w.l(rtexit2.o)
    0x08000246   0x00000002   PAD
    0x08000248   0x00000510   Code   RO            1    .text               main.o
    0x08000758   0x0000001a   Code   RO          187    .text               stm32f10x_it.o
    0x08000772   0x00000002   PAD
    0x08000774   0x000001e0   Code   RO          228    .text               system_stm32f10x.o
    0x08000954   0x00000064   Code   RO          246    .text               led.o
    0x080009b8   0x00000260   Code   RO          261    .text               adc.o
    0x08000c18   0x000002d0   Code   RO          283    .text               timer.o
    0x08000ee8   0x00000048   Code   RO          302    .text               bsp_ec11.o
    0x08000f30   0x00000180   Code   RO          321    .text               spi.o
    0x080010b0   0x00000c80   Code   RO          336    .text               oled.o
    0x08001d30   0x000000a8   Code   RO          359    .text               dac.o
    0x08001dd8   0x00000308   Code   RO          374    .text               matrix_key.o
    0x080020e0   0x000001c0   Code   RO          388    .text               bsp.o
    0x080022a0   0x0000019c   Code   RO          410    .text               key_scan.o
    0x0800243c   0x000000d4   Code   RO          426    .text               delay.o
    0x08002510   0x000000c0   Code   RO          457    .text               usart.o
    0x080025d0   0x00000040   Code   RO          493    .text               startup_stm32f10x_hd.o
    0x08002610   0x00000148   Code   RO          497    .text               main_menu.o
    0x08002758   0x000004f4   Code   RO          516    .text               cw_menu.o
    0x08002c4c   0x000000e0   Code   RO          536    .text               power_menu.o
    0x08002d2c   0x00000100   Code   RO          555    .text               oled_task.o
    0x08002e2c   0x00000064   Code   RO          570    .text               key_s1_process.o
    0x08002e90   0x00000004   Code   RO          589    .text               key_s2_process.o
    0x08002e94   0x000000b8   Code   RO          601    .text               key_s3_process.o
    0x08002f4c   0x000000b0   Code   RO          613    .text               ec11_key_process.o
    0x08002ffc   0x00000bb8   Code   RO          625    .text               ec11_spin_process.o
    0x08003bb4   0x00000320   Code   RO          637    .text               pll_spi_init.o
    0x08003ed4   0x000001d4   Code   RO          649    .text               all_lo_init.o
    0x080040a8   0x000006dc   Code   RO          675    .text               lo_lmx2592_freq_set.o
    0x08004784   0x0000079c   Code   RO          693    .text               ad9912_drive.o
    0x08004f20   0x000000f8   Code   RO          712    .text               pe4302.o
    0x08005018   0x000000e4   Code   RO          724    .text               hmc241.o
    0x080050fc   0x000001bc   Code   RO          751    .text               adl5513.o
    0x080052b8   0x0000054c   Code   RO          766    .text               amp_set.o
    0x08005804   0x0000023c   Code   RO          785    .text               ch2_freq_set.o
    0x08005a40   0x000001a0   Code   RO          815    .text               malloc.o
    0x08005be0   0x0000035c   Code   RO          835    .text               stm32f10x_gpio.o
    0x08005f3c   0x000003a4   Code   RO          847    .text               stm32f10x_rcc.o
    0x080062e0   0x00000408   Code   RO          861    .text               stm32f10x_usart.o
    0x080066e8   0x000000dc   Code   RO          873    .text               misc.o
    0x080067c4   0x0000044e   Code   RO          885    .text               stm32f10x_adc.o
    0x08006c12   0x00000002   PAD
    0x08006c14   0x00000e1a   Code   RO          921    .text               stm32f10x_tim.o
    0x08007a2e   0x00000002   PAD
    0x08007a30   0x0000030c   Code   RO          933    .text               stm32f10x_spi.o
    0x08007d3c   0x0000018c   Code   RO          957    .text               stm32f10x_dac.o
    0x08007ec8   0x00000002   Code   RO          983    .text               c_w.l(use_no_semi_2.o)
    0x08007eca   0x00000002   PAD
    0x08007ecc   0x00000018   Code   RO          989    .text               c_w.l(noretval__2printf.o)
    0x08007ee4   0x00000028   Code   RO          991    .text               c_w.l(noretval__2sprintf.o)
    0x08007f0c   0x0000004e   Code   RO          995    .text               c_w.l(_printf_pad.o)
    0x08007f5a   0x00000002   PAD
    0x08007f5c   0x00000078   Code   RO          997    .text               c_w.l(_printf_dec.o)
    0x08007fd4   0x0000007c   Code   RO          999    .text               c_w.l(_printf_longlong_dec.o)
    0x08008050   0x00000188   Code   RO         1018    .text               c_w.l(__printf_flags_ss_wp.o)
    0x080081d8   0x0000001a   Code   RO         1025    .text               c_w.l(atoi.o)
    0x080081f2   0x00000006   Code   RO         1027    .text               c_w.l(heapauxi.o)
    0x080081f8   0x00000002   Code   RO         1121    .text               c_w.l(use_no_semi.o)
    0x080081fa   0x00000002   PAD
    0x080081fc   0x00000008   Code   RO         1127    .text               c_w.l(rt_errno_addr_intlibspace.o)
    0x08008204   0x0000008a   Code   RO         1129    .text               c_w.l(lludiv10.o)
    0x0800828e   0x00000016   Code   RO         1131    .text               c_w.l(_rserrno.o)
    0x080082a4   0x000000b2   Code   RO         1133    .text               c_w.l(_printf_intcommon.o)
    0x08008356   0x0000041a   Code   RO         1135    .text               c_w.l(_printf_fp_dec.o)
    0x08008770   0x00000030   Code   RO         1137    .text               c_w.l(_printf_char_common.o)
    0x080087a0   0x0000000a   Code   RO         1139    .text               c_w.l(_sputc.o)
    0x080087aa   0x00000002   PAD
    0x080087ac   0x00000024   Code   RO         1141    .text               c_w.l(_printf_char_file.o)
    0x080087d0   0x000000a4   Code   RO         1145    .text               c_w.l(strtod.o)
    0x08008874   0x00000070   Code   RO         1147    .text               c_w.l(strtol.o)
    0x080088e4   0x00000008   Code   RO         1185    .text               c_w.l(libspace.o)
    0x080088ec   0x00000010   Code   RO         1203    .text               c_w.l(rt_ctype_table.o)
    0x080088fc   0x00000008   Code   RO         1208    .text               c_w.l(rt_locale_intlibspace.o)
    0x08008904   0x00000012   Code   RO         1210    .text               c_w.l(isspace.o)
    0x08008916   0x00000002   PAD
    0x08008918   0x00000080   Code   RO         1212    .text               c_w.l(_printf_fp_infnan.o)
    0x08008998   0x00000040   Code   RO         1216    .text               c_w.l(_sgetc.o)
    0x080089d8   0x0000009e   Code   RO         1218    .text               c_w.l(_strtoul.o)
    0x08008a76   0x00000002   PAD
    0x08008a78   0x000000dc   Code   RO         1220    .text               c_w.l(bigflt0.o)
    0x08008b54   0x00000008   Code   RO         1245    .text               c_w.l(ferror.o)
    0x08008b5c   0x0000004a   Code   RO         1258    .text               c_w.l(sys_stackheap_outer.o)
    0x08008ba6   0x0000001c   Code   RO         1260    .text               c_w.l(_chval.o)
    0x08008bc2   0x00000002   PAD
    0x08008bc4   0x000004a4   Code   RO         1262    .text               c_w.l(scanf_fp.o)
    0x08009068   0x00000012   Code   RO         1267    .text               c_w.l(exit.o)
    0x0800907a   0x00000002   PAD
    0x0800907c   0x00000080   Code   RO         1269    .text               c_w.l(strcmpv7m.o)
    0x080090fc   0x00000320   Code   RO         1354    .text               c_w.l(scanf_hexfp.o)
    0x0800941c   0x00000134   Code   RO         1356    .text               c_w.l(scanf_infnan.o)
    0x08009550   0x00000026   Code   RO         1372    .text               c_w.l(llshl.o)
    0x08009576   0x0000003e   Code   RO         1223    CL$$btod_d2e        c_w.l(btod.o)
    0x080095b4   0x00000046   Code   RO         1225    CL$$btod_d2e_denorm_low  c_w.l(btod.o)
    0x080095fa   0x00000060   Code   RO         1224    CL$$btod_d2e_norm_op1  c_w.l(btod.o)
    0x0800965a   0x00000338   Code   RO         1233    CL$$btod_div_common  c_w.l(btod.o)
    0x08009992   0x00000002   PAD
    0x08009994   0x00000054   Code   RO         1231    CL$$btod_e2d        c_w.l(btod.o)
    0x080099e8   0x000000c6   Code   RO         1230    CL$$btod_e2e        c_w.l(btod.o)
    0x08009aae   0x00000028   Code   RO         1227    CL$$btod_ediv       c_w.l(btod.o)
    0x08009ad6   0x00000028   Code   RO         1229    CL$$btod_edivd      c_w.l(btod.o)
    0x08009afe   0x00000028   Code   RO         1226    CL$$btod_emul       c_w.l(btod.o)
    0x08009b26   0x00000028   Code   RO         1228    CL$$btod_emuld      c_w.l(btod.o)
    0x08009b4e   0x00000244   Code   RO         1232    CL$$btod_mult_common  c_w.l(btod.o)
    0x08009d92   0x00000028   Code   RO         1180    i.__ARM_fpclassify  m_ws.l(fpclassify.o)
    0x08009dba   0x000000aa   Code   RO         1182    i.__kernel_poly     m_ws.l(poly.o)
    0x08009e64   0x00000010   Code   RO         1166    i.__mathlib_dbl_divzero  m_ws.l(dunder.o)
    0x08009e74   0x00000004   Code   RO         1168    i.__mathlib_dbl_infnan2  m_ws.l(dunder.o)
    0x08009e78   0x0000000c   Code   RO         1169    i.__mathlib_dbl_invalid  m_ws.l(dunder.o)
    0x08009e84   0x0000000e   Code   RO         1170    i.__mathlib_dbl_overflow  m_ws.l(dunder.o)
    0x08009e92   0x00000002   PAD
    0x08009e94   0x00000010   Code   RO         1172    i.__mathlib_dbl_underflow  m_ws.l(dunder.o)
    0x08009ea4   0x00000010   Code   RO         1341    i.__mathlib_narrow  m_ws.l(narrow.o)
    0x08009eb4   0x00000088   Code   RO         1342    i.__mathlib_tofloat  m_ws.l(narrow.o)
    0x08009f3c   0x00000016   Code   RO         1382    i.__support_ldexp   m_ws.l(ldexp.o)
    0x08009f52   0x0000000e   Code   RO         1011    i._is_digit         c_w.l(__printf_wp.o)
    0x08009f60   0x0000002a   Code   RO         1100    i.atof              m_ws.l(atof.o)
    0x08009f8a   0x00000002   PAD
    0x08009f8c   0x00000058   Code   RO         1365    i.frexp             m_ws.l(frexp.o)
    0x08009fe4   0x00000074   Code   RO         1383    i.ldexp             m_ws.l(ldexp.o)
    0x0800a058   0x000009d8   Code   RO         1104    i.pow               m_ws.l(pow.o)
    0x0800aa30   0x0000004c   Code   RO         1114    i.sqrt              m_ws.l(sqrt.o)
    0x0800aa7c   0x0000002c   Code   RO         1250    locale$$code        c_w.l(lc_numeric_c.o)
    0x0800aaa8   0x0000002c   Code   RO         1265    locale$$code        c_w.l(lc_ctype_c.o)
    0x0800aad4   0x00000062   Code   RO         1031    x$fpl$d2f           fz_ws.l(d2f.o)
    0x0800ab36   0x00000002   PAD
    0x0800ab38   0x00000150   Code   RO         1033    x$fpl$dadd          fz_ws.l(daddsub_clz.o)
    0x0800ac88   0x00000010   Code   RO         1252    x$fpl$dcheck1       fz_ws.l(dcheck1.o)
    0x0800ac98   0x00000018   Code   RO         1149    x$fpl$dcmpinf       fz_ws.l(dcmpi.o)
    0x0800acb0   0x000002b0   Code   RO         1040    x$fpl$ddiv          fz_ws.l(ddiv.o)
    0x0800af60   0x00000078   Code   RO         1362    x$fpl$deqf          fz_ws.l(deqf.o)
    0x0800afd8   0x0000005a   Code   RO         1043    x$fpl$dfixu         fz_ws.l(dfixu.o)
    0x0800b032   0x0000002e   Code   RO         1052    x$fpl$dflt          fz_ws.l(dflt_clz.o)
    0x0800b060   0x00000026   Code   RO         1051    x$fpl$dfltu         fz_ws.l(dflt_clz.o)
    0x0800b086   0x00000002   PAD
    0x0800b088   0x0000008a   Code   RO         1058    x$fpl$dfltull       fz_ws.l(dfltll_clz.o)
    0x0800b112   0x00000002   PAD
    0x0800b114   0x00000078   Code   RO         1061    x$fpl$dleqf         fz_ws.l(dleqf.o)
    0x0800b18c   0x00000154   Code   RO         1063    x$fpl$dmul          fz_ws.l(dmul.o)
    0x0800b2e0   0x0000009c   Code   RO         1151    x$fpl$dnaninf       fz_ws.l(dnaninf.o)
    0x0800b37c   0x0000000c   Code   RO         1153    x$fpl$dretinf       fz_ws.l(dretinf.o)
    0x0800b388   0x0000006c   Code   RO         1065    x$fpl$drleqf        fz_ws.l(drleqf.o)
    0x0800b3f4   0x00000016   Code   RO         1034    x$fpl$drsb          fz_ws.l(daddsub_clz.o)
    0x0800b40a   0x00000002   PAD
    0x0800b40c   0x000001cc   Code   RO         1155    x$fpl$dsqrt         fz_ws.l(dsqrt_noumaal.o)
    0x0800b5d8   0x000001d4   Code   RO         1035    x$fpl$dsub          fz_ws.l(daddsub_clz.o)
    0x0800b7ac   0x00000056   Code   RO         1067    x$fpl$f2d           fz_ws.l(f2d.o)
    0x0800b802   0x00000002   PAD
    0x0800b804   0x000000c4   Code   RO         1069    x$fpl$fadd          fz_ws.l(faddsub_clz.o)
    0x0800b8c8   0x00000018   Code   RO         1157    x$fpl$fcmpinf       fz_ws.l(fcmpi.o)
    0x0800b8e0   0x00000184   Code   RO         1076    x$fpl$fdiv          fz_ws.l(fdiv.o)
    0x0800ba64   0x00000068   Code   RO         1079    x$fpl$feqf          fz_ws.l(feqf.o)
    0x0800bacc   0x0000003e   Code   RO         1081    x$fpl$ffixu         fz_ws.l(ffixu.o)
    0x0800bb0a   0x00000002   PAD
    0x0800bb0c   0x00000026   Code   RO         1085    x$fpl$ffltu         fz_ws.l(fflt_clz.o)
    0x0800bb32   0x00000002   PAD
    0x0800bb34   0x00000068   Code   RO         1091    x$fpl$fleqf         fz_ws.l(fleqf.o)
    0x0800bb9c   0x00000102   Code   RO         1093    x$fpl$fmul          fz_ws.l(fmul.o)
    0x0800bc9e   0x0000008c   Code   RO         1159    x$fpl$fnaninf       fz_ws.l(fnaninf.o)
    0x0800bd2a   0x0000000a   Code   RO         1161    x$fpl$fretinf       fz_ws.l(fretinf.o)
    0x0800bd34   0x00000062   Code   RO         1095    x$fpl$frleqf        fz_ws.l(frleqf.o)
    0x0800bd96   0x00000014   Code   RO         1070    x$fpl$frsb          fz_ws.l(faddsub_clz.o)
    0x0800bdaa   0x00000002   PAD
    0x0800bdac   0x000000ea   Code   RO         1071    x$fpl$fsub          fz_ws.l(faddsub_clz.o)
    0x0800be96   0x00000002   PAD
    0x0800be98   0x00000078   Code   RO         1047    x$fpl$llufromd      fz_ws.l(dfixull.o)
    0x0800bf10   0x00000004   Code   RO         1097    x$fpl$printf1       fz_ws.l(printf1.o)
    0x0800bf14   0x00000064   Code   RO         1322    x$fpl$retnan        fz_ws.l(retnan.o)
    0x0800bf78   0x0000005c   Code   RO         1163    x$fpl$scalbn        fz_ws.l(scalbn.o)
    0x0800bfd4   0x00000004   Code   RO         1256    x$fpl$scanf1        fz_ws.l(scanf1.o)
    0x0800bfd8   0x00000008   Code   RO         1333    x$fpl$scanf2        fz_ws.l(scanf2.o)
    0x0800bfe0   0x00000030   Code   RO         1339    x$fpl$trapveneer    fz_ws.l(trapv.o)
    0x0800c010   0x00000000   Code   RO         1165    x$fpl$usenofp       fz_ws.l(usenofp.o)
    0x0800c010   0x00001500   Data   RO          337    .constdata          oled.o
    0x0800d510   0x00000560   Data   RO          650    .constdata          all_lo_init.o
    0x0800da70   0x00000398   Data   RO          767    .constdata          amp_set.o
    0x0800de08   0x00000011   Data   RO         1019    .constdata          c_w.l(__printf_flags_ss_wp.o)
    0x0800de19   0x00000007   PAD
    0x0800de20   0x00000088   Data   RO         1105    .constdata          m_ws.l(pow.o)
    0x0800dea8   0x00000008   Data   RO         1184    .constdata          m_ws.l(qnan.o)
    0x0800deb0   0x00000094   Data   RO         1221    .constdata          c_w.l(bigflt0.o)
    0x0800df44   0x00000020   Data   RO         1440    Region$$Table       anon$$obj.o
    0x0800df64   0x00000008   Data   RO         1328    c$$dinf             fz_ws.l(fpconst.o)
    0x0800df6c   0x0000001c   Data   RO         1249    locale$$data        c_w.l(lc_numeric_c.o)
    0x0800df88   0x00000110   Data   RO         1264    locale$$data        c_w.l(lc_ctype_c.o)


    Execution Region RW_IRAM1 (Base: 0x20000000, Size: 0x0000a3b0, Max: 0x0000c000, ABSOLUTE, COMPRESSED[0x000000e4])

    Base Addr    Size         Type   Attr      Idx    E Section Name        Object

    0x20000000   0x00000058   Data   RW            3    .data               main.o
    0x20000058   0x00000014   Data   RW          229    .data               system_stm32f10x.o
    0x2000006c   0x00000008   Data   RW          262    .data               adc.o
    0x20000074   0x00000004   Data   RW          284    .data               timer.o
    0x20000078   0x00000002   Data   RW          303    .data               bsp_ec11.o
    0x2000007a   0x00000004   Data   RW          427    .data               delay.o
    0x2000007e   0x00000002   PAD
    0x20000080   0x00000006   Data   RW          459    .data               usart.o
    0x20000086   0x0000002d   Data   RW          498    .data               main_menu.o
    0x200000b3   0x00000071   Data   RW          518    .data               cw_menu.o
    0x20000124   0x00000016   Data   RW          537    .data               power_menu.o
    0x2000013a   0x00000004   Data   RW          571    .data               key_s1_process.o
    0x2000013e   0x00000002   PAD
    0x20000140   0x00000010   Data   RW          651    .data               all_lo_init.o
    0x20000150   0x00000028   Data   RW          676    .data               lo_lmx2592_freq_set.o
    0x20000178   0x00000018   Data   RW          694    .data               ad9912_drive.o
    0x20000190   0x00000014   Data   RW          752    .data               adl5513.o
    0x200001a4   0x00000024   Data   RW          768    .data               amp_set.o
    0x200001c8   0x00000014   Data   RW          818    .data               malloc.o
    0x200001dc   0x00000014   Data   RW          848    .data               stm32f10x_rcc.o
    0x200001f0   0x0000005d   Zero   RW          375    .bss                matrix_key.o
    0x2000024d   0x00000040   Zero   RW          517    .bss                cw_menu.o
    0x2000028d   0x00000003   PAD
    0x20000290   0x000094c0   Zero   RW          816    .bss                malloc.o
    0x20009750   0x00000060   Zero   RW         1186    .bss                c_w.l(libspace.o)
    0x200097b0   0x00000400   Zero   RW          491    HEAP                startup_stm32f10x_hd.o
    0x20009bb0   0x00000800   Zero   RW          490    STACK               startup_stm32f10x_hd.o


==============================================================================

Image component sizes


      Code (inc. data)   RO Data    RW Data    ZI Data      Debug   Object Name

      1948         76          0         24          0       7578   ad9912_drive.o
       608         26          0          8          0       2425   adc.o
       444         92          0         20          0       1356   adl5513.o
       468         86       1376         16          0       3197   all_lo_init.o
      1356        272        920         36          0       3058   amp_set.o
       448        120          0          0          0        991   bsp.o
        72          6          0          2          0        899   bsp_ec11.o
       572         38          0          0          0       1727   ch2_freq_set.o
      1268        122          0        113         64       6208   cw_menu.o
       168         14          0          0          0        821   dac.o
       212         18          0          4          0       1143   delay.o
       176         24          0          0          0        710   ec11_key_process.o
      3000        528          0          0          0       3924   ec11_spin_process.o
       228         26          0          0          0        862   hmc241.o
       100         24          0          4          0        944   key_s1_process.o
         4          0          0          0          0        502   key_s2_process.o
       184         60          0          0          0        618   key_s3_process.o
       412        200          0          0          0        763   key_scan.o
       100          8          0          0          0        559   led.o
      1756        126          0         40          0       3416   lo_lmx2592_freq_set.o
      1296        534          0         88          0     278782   main.o
       328         66          0         45          0       2094   main_menu.o
       416          6          0         20      38080       4205   malloc.o
       776         36          0          0         93       3957   matrix_key.o
       220         22          0          0          0       1901   misc.o
      3200         12       5376          0          0       9702   oled.o
       256         36          0          0          0        645   oled_task.o
       248         30          0          0          0        918   pe4302.o
       800        110          0          0          0       1705   pll_spi_init.o
       224         28          0         22          0       2009   power_menu.o
       384         10          0          0          0       1975   spi.o
        64         26        304          0       3072        820   startup_stm32f10x_hd.o
      1102         26          0          0          0      11145   stm32f10x_adc.o
       396          6          0          0          0       3762   stm32f10x_dac.o
       860         38          0          0          0       5833   stm32f10x_gpio.o
        26          0          0          0          0       1230   stm32f10x_it.o
       932         36          0         20          0       9064   stm32f10x_rcc.o
       780         14          0          0          0       6718   stm32f10x_spi.o
      3610         88          0          0          0      22944   stm32f10x_tim.o
      1032         22          0          0          0       8560   stm32f10x_usart.o
         0          0          0          0          0         32   sys.o
       480         38          0         20          0       1891   system_stm32f10x.o
       720         44          0          4          0       3087   timer.o
       192          8          0          6          0       3092   usart.o

    ----------------------------------------------------------------------
     31872       3102       8008        496      41312     427772   Object Totals
         0          0         32          0          0          0   (incl. Generated)
         6          0          0          4          3          0   (incl. Padding)

    ----------------------------------------------------------------------

      Code (inc. data)   RO Data    RW Data    ZI Data      Debug   Library Member Name

        90          0          0          0          0          0   __dczerorl2.o
         8          0          0          0          0         68   __main.o
       392          4         17          0          0         92   __printf_flags_ss_wp.o
        14          0          0          0          0         68   __printf_wp.o
         0          0          0          0          0          0   __rtentry.o
        12          0          0          0          0          0   __rtentry2.o
         6          0          0          0          0          0   __rtentry4.o
        52          8          0          0          0          0   __scatter.o
        28          0          0          0          0          0   __scatter_zi.o
        28          0          0          0          0         68   _chval.o
        48          6          0          0          0         96   _printf_char_common.o
        36          4          0          0          0         80   _printf_char_file.o
       120         16          0          0          0         92   _printf_dec.o
         6          0          0          0          0          0   _printf_f.o
      1050          0          0          0          0        216   _printf_fp_dec.o
       128         16          0          0          0         84   _printf_fp_infnan.o
       178          0          0          0          0         88   _printf_intcommon.o
        10          0          0          0          0          0   _printf_ll.o
         6          0          0          0          0          0   _printf_llu.o
       124         16          0          0          0         92   _printf_longlong_dec.o
        78          0          0          0          0        108   _printf_pad.o
         0          0          0          0          0          0   _printf_percent.o
         4          0          0          0          0          0   _printf_percent_end.o
         6          0          0          0          0          0   _printf_u.o
        22          0          0          0          0        100   _rserrno.o
        64          0          0          0          0         84   _sgetc.o
        10          0          0          0          0         68   _sputc.o
       158          0          0          0          0         92   _strtoul.o
        26          0          0          0          0         80   atoi.o
       220          4        148          0          0         96   bigflt0.o
      2074        132          0          0          0        940   btod.o
        18          0          0          0          0         80   exit.o
         8          0          0          0          0         68   ferror.o
         6          0          0          0          0        152   heapauxi.o
        18          0          0          0          0         76   isspace.o
        44         10        272          0          0         76   lc_ctype_c.o
        44         10         28          0          0         76   lc_numeric_c.o
         2          0          0          0          0          0   libinit.o
        30          0          0          0          0          0   libinit2.o
         2          0          0          0          0          0   libshutdown.o
         2          0          0          0          0          0   libshutdown2.o
         8          4          0          0         96         68   libspace.o
        38          0          0          0          0         68   llshl.o
       138          0          0          0          0         80   lludiv10.o
        24          4          0          0          0         84   noretval__2printf.o
        40          6          0          0          0         84   noretval__2sprintf.o
        16          4          0          0          0         76   rt_ctype_table.o
         8          4          0          0          0         68   rt_errno_addr_intlibspace.o
         8          4          0          0          0         68   rt_locale_intlibspace.o
         2          0          0          0          0          0   rtexit.o
        10          0          0          0          0          0   rtexit2.o
      1188         12          0          0          0        148   scanf_fp.o
       800         14          0          0          0        100   scanf_hexfp.o
       308         16          0          0          0        100   scanf_infnan.o
       128          0          0          0          0         68   strcmpv7m.o
       164         14          0          0          0        120   strtod.o
       112          0          0          0          0         88   strtol.o
        74          0          0          0          0         80   sys_stackheap_outer.o
         2          0          0          0          0         68   use_no_semi.o
         2          0          0          0          0         68   use_no_semi_2.o
        98          4          0          0          0         92   d2f.o
       826         16          0          0          0        348   daddsub_clz.o
        16          4          0          0          0         68   dcheck1.o
        24          0          0          0          0         68   dcmpi.o
       688        140          0          0          0        208   ddiv.o
       120          4          0          0          0         92   deqf.o
        90          4          0          0          0         92   dfixu.o
       120          4          0          0          0        104   dfixull.o
        84          0          0          0          0        136   dflt_clz.o
       138          0          0          0          0         84   dfltll_clz.o
       120          4          0          0          0         92   dleqf.o
       340         12          0          0          0        104   dmul.o
       156          4          0          0          0         92   dnaninf.o
        12          0          0          0          0         68   dretinf.o
       108          0          0          0          0         80   drleqf.o
       460         56          0          0          0        120   dsqrt_noumaal.o
        86          4          0          0          0         84   f2d.o
       450          8          0          0          0        236   faddsub_clz.o
        24          0          0          0          0         68   fcmpi.o
       388         76          0          0          0         96   fdiv.o
       104          4          0          0          0         84   feqf.o
        62          4          0          0          0         84   ffixu.o
        38          0          0          0          0         68   fflt_clz.o
       104          4          0          0          0         84   fleqf.o
       258          4          0          0          0         84   fmul.o
       140          4          0          0          0         84   fnaninf.o
         0          0          8          0          0          0   fpconst.o
        10          0          0          0          0         68   fretinf.o
        98          0          0          0          0         68   frleqf.o
         4          0          0          0          0         68   printf1.o
       100          0          0          0          0         68   retnan.o
        92          0          0          0          0         68   scalbn.o
         4          0          0          0          0         68   scanf1.o
         8          0          0          0          0         84   scanf2.o
        48          0          0          0          0         68   trapv.o
         0          0          0          0          0          0   usenofp.o
        42          0          0          0          0         84   atof.o
        62         10          0          0          0        340   dunder.o
        40          0          0          0          0         68   fpclassify.o
        88          8          0          0          0         76   frexp.o
       138          0          0          0          0        160   ldexp.o
       152          4          0          0          0        168   narrow.o
       170          0          0          0          0         96   poly.o
      2520        190        136          0          0        324   pow.o
         0          0          8          0          0          0   qnan.o
        76          0          0          0          0         84   sqrt.o

    ----------------------------------------------------------------------
     16992        882        624          0         96       9356   Library Totals
        44          2          7          0          0          0   (incl. Padding)

    ----------------------------------------------------------------------

      Code (inc. data)   RO Data    RW Data    ZI Data      Debug   Library Name

      8242        308        465          0         96       4576   c_w.l
      5418        360          8          0          0       3380   fz_ws.l
      3288        212        144          0          0       1400   m_ws.l

    ----------------------------------------------------------------------
     16992        882        624          0         96       9356   Library Totals

    ----------------------------------------------------------------------

==============================================================================


      Code (inc. data)   RO Data    RW Data    ZI Data      Debug   

     48864       3984       8632        496      41408     428700   Grand Totals
     48864       3984       8632        228      41408     428700   ELF Image Totals (compressed)
     48864       3984       8632        228          0          0   ROM Totals

==============================================================================

    Total RO  Size (Code + RO Data)                57496 (  56.15kB)
    Total RW  Size (RW Data + ZI Data)             41904 (  40.92kB)
    Total ROM Size (Code + RO Data + RW Data)      57724 (  56.37kB)

==============================================================================

